:1000000054464953000100008CD00200300A578F3B
:10001000176302162010261342593559176302013F
:100020002010261342593559176302012010261358
:100030004259355903000000000000000000000094
:100040005446435300200000749E0200000000004C
:100050000080011001210000252100000D1F020079
:10006000292100002B2100002D2100003D2100004E
:100070003D2100003D2100003D2100002F21000016
:10008000312100003D21000033210000B56E000049
:100090007F720000372100003D21000079570010D9
:1000A00037210000C34F0000C74F0000AF710000B0
:1000B00037210000F36A0000E5610000CB4F00002B
:1000C000AD6800003721000037210000015D00000D
:1000D0000000000000000000000000000000000020
:1000E0000000000000000000000000000000000010
:1000F0000000000000000000000000000000000000
:1001000000000000000000000000000000000000EF
:1001100000000000000000000000000000000000DF
:1001200000000000000000000000000000000000CF
:1001300000000000000000000000000000000000BF
:1001400000000000000000000000000000000000AF
:1001500000F003F800F020F8FEE70D480168890878
:100160008900002001C101C101C101C17047000027
:1001700060600010FEE7FEE7FEE7FEE7FEE7FEE751
:10018000FEE7FEE7FEE703480047FEE7FEE7000064
:10019000202100003D21000000F002F800F068F886
:1001A0000AA090E8000C82448344AAF10107DA45D2
:1001B00001D100F05DF8AFF2090EBAE80F0013F0BC
:1001C000010F18BFFB1A43F001031847803A0200E1
:1001D000E03A02000A444FF0000C10F8013B13F023
:1001E000070408BF10F8014B1D1108BF10F8015B90
:1001F000641E05D010F8016B641E01F8016BF9D183
:1002000013F0080F1EBF10F8014BAD1C0C1B09D1D9
:100210006D1E58BF01F801CBFAD505E014F8016B4B
:1002200001F8016B6D1EF9D59142D6D370470000DD
:10023000103A24BF78C878C1FAD8520724BF30C812
:1002400030C144BF04680C607047000000230024E4
:1002500000250026103A28BF78C1FBD8520728BFD6
:1002600030C148BF0B6070471FB51FBD10B510BD32
:10027000DFF80CD0FFF7F8FF07F0D8F91FF060FEA9
:100280000080011003B4FFF7F1FF03BC1FF060FE14
:1002900008B500200346024600900121022000F02C
:1002A00051FB08BD38B5FF4D0024FF48AC81EC81FF
:1002B0002C8240698047E861FF202872FB480023B8
:1002C0001A46046044608460C4600461012068725E
:1002D0002C70AC7001460220009400F033FB01202A
:1002E00038BD38B5EF4D02282C7A22460DD00528AE
:1002F00010D0A24208BF38BD002003460246214666
:10030000009000F01FFB2C7238BD022914BF01249D
:100310000224EEE7022914BF04240824E9E708B503
:10032000009313460A460146012000F00BFB08BD6E
:1003300008B50346009103220221012000F002FBD0
:1003400008BD38B500240DF0B5FF002818BF012402
:1003500012F070FC002818BF0224D2480178A14294
:1003600008BF38BD047000200346022100902246D9
:10037000084600F0E7FA38BD38B5CA4D044668783B
:10038000A04208BF38BD07F065F96C70002C0CBFA7
:10039000052106210020034602460090022000F0BD
:1003A000D1FA38BD08B500210B460246009107215D
:1003B000022000F0C7FA08BD08B500210B4602462E
:1003C00000910821022000F0BDFA08BD08B5002107
:1003D0000091002814BF01220022002303210220E3
:1003E00000F0B0FA08BD08B50020034602460090B0
:1003F0000421022000F0A6FA08BDAA4B0028DA78F2
:1004000014BF01210021D9708A4208BF7047021C25
:1004100018BF012208B50020034600900A210220DF
:1004200000F090FA08BD9F4B00289A7814BF012174
:10043000002199708A4208BF7047021C18BF012230
:1004400008B50020034600900921022000F07AFA46
:1004500008BD94488078002818BF0120704701200B
:100460009049087170478F48007970478D49002086
:10047000087170472DE9F04104460127002503F07B
:100480000700884E8846012804BF0020308248D0EB
:10049000022846D1308A844904280BD2002818BF8C
:1004A000B06902D148688047B06110F8011B217023
:1004B000B0612FE0062809D288688047318A80B26F
:1004C000C1F10501C900C840207023E0082808D206
:1004D00008698047318AC1F10701C900C84020700E
:1004E00018E00C2808D248698047318AC1F10B0115
:1004F000C900C84020700DE00E2808D288698047E6
:10050000318AC1F10D01C900C840207002E0FF200E
:1005100020700027308A401C80B230820E2828BF0D
:10052000012588F800503846BDE8F08130B403F06A
:1005300007000024DFF86CC1012804BFACF80C40B0
:10054000ACF810401BD013F0070F18D1554BBCF876
:1005500010009B89022805D2120242EA1322ACF84D
:100560000C2009E003449D1EB5F5806F04DADCF829
:100570001C502B4403F8022C401CACF810000C70EB
:1005800030BC00207047F0B40746002003F0070499
:10059000444D0646012C04BF2E826E6125D0DFF843
:1005A00004C1022CBCF80EC003D013F0070F0DD00D
:1005B0001BE02A8A0CEB0203B3F5806F15D2E869C1
:1005C000C05C3870501C288201200EE0120242EA02
:1005D0001C22EA816B69012B05D1B2F5806F24BF23
:1005E00040F2FF32EA815A1C6A610E70F0BC70471B
:1005F00038B503F0070000240D46012809D1294829
:1006000000231A460482848119460220009400F0D7
:1006100099F92C70002038BD2DE9F04182B01746C1
:100620000C0005464FF0000808BF002608D02678C9
:100630001F49012E18BF022E58D0032E7ED09EB91E
:1006400085F8008085F80180A5F80280A5F804806F
:10065000A5F80680A5F80880A5F80A80A5F80C8002
:10066000A87B20F00100A873012E18BF032E06D02E
:100670000DF060FB002804BF02B0BDE8F08106F079
:10068000E9FF05281CBF02B0BDE8F081012E04BFC0
:10069000C0208DF800000FD0022E0CBFC220C12058
:1006A00008E0000000840010C05A020020890010F9
:1006B0009C8800108DF8000060788DF8010060883B
:1006C0000123000A8DF80200A0788DF80300A088AD
:1006D0000622000A8DF8040020798DF8050069468D
:1006E000072011F0B0F902B0BDE8F0816078421E39
:1006F00005EB001000F8102C607805EB001000F8F6
:100700000F6C08686288438BC08A5A4392FBF0F0F2
:10071000627805EB021222F80E0C0868A288018BA1
:10072000808A514391FBF0F0617805EB011121F8CB
:100730000C0C6178A07905EB011100E022E021F8B2
:100740000A0C6178207A05EB011121F8080C617818
:10075000607A05EB011121F8060C6178A07B05EBAE
:10076000011121F8040CE0790528607805EB0010F0
:1007700010F8021C0CBF41F0010121F0010100F84A
:10078000021C71E76078421E05EB001000F8102C87
:100790006278032005EB021202F80F0C08686288E9
:1007A000438BC08A5A4392FBF0F0627805EB021249
:1007B00022F80E0C0868A288018B808A514391FBB5
:1007C000F0F0617805EB011121F80C0C06F042FF06
:1007D000052821D107B36178B87905EB011121F81B
:1007E0000A0C6178387A05EB011121F8080C617860
:1007F000787A05EB011121F8060CF8790528607864
:1008000005EB001010F8021C0CBF41F0010121F0B3
:10081000010100F8021C17E0607805EB001020F8D9
:100820000A8C607805EB001020F8088C607805EBE6
:10083000001020F8068C607805EB001010F8021C00
:1008400021F0010100F8021C607805EB001020F88F
:10085000048C09E741490020487170473F484079BE
:100860007047002818BF01203C49887170473B48F9
:1008700080797047002818BF01203849C871704737
:100880003648C079704735494881704733484089B8
:1008900070473249012048717047314B03EB8000AB
:1008A0004254704700B583B0002100910191027855
:1008B0008DF8002042788DF8012082788DF8022092
:1008C000C2788DF8032002798DF8042042798DF8E2
:1008D000052080798DF806008DF8071006F0C8FF16
:1008E00001280CD11FF04AFB012801BF9DF8000030
:1008F00046289DF80100012804BF03B000BD6846EA
:100900001FF041FB03B000BD70471449002818BF19
:100910000120487270471148407A7047012818BF7B
:1009200070471048012904BF416841F4007105D0A7
:10093000002906BF416821F400717047416070478B
:100940000948704708B5DDF808C0CDF800C0DFF8E9
:100950001CC0DCF800C0E04708BD000000840010A7
:10096000208900100010004080550200C05A02008B
:100970007047F648D0F8500300F00100704770B59A
:10098000F24D04000AD002F067FA38B9D5F85003E6
:1009900010F0010F1CBF0020A86005D10120A86045
:1009A000002C08BF00202DD0D5F8600310F0010FF7
:1009B0000BD1D5F8600340F00100C5F86003D5F80D
:1009C000600320F00100C5F86003E148016811F000
:1009D000010F07D1016841F001010160016821F0B8
:1009E0000101016004F022FB00281CBFD5F8500370
:1009F00010F0010F05D004F013FB002818BF04F01D
:100A000021FB0120286270BDD048006A002818BF71
:100A100001207047C00000F1804000F5A040416314
:100A20007047C00000F1804000F5A040006B00F46A
:100A3000807070471021C00000F1804000F5A04098
:100A40004163704730B48209C24B00F00F0000EBE5
:100A5000400053F822404FF4847505EB8015D1F81F
:100A600000C044F805C053F822204FF4867303EB0E
:100A700080104968115030BC70478209B54850F861
:100A80002200D0F8402161F30D22C0F840217047C8
:100A9000B049800951F82000D0F84001C0F305208A
:100AA0007047AA49D1F8402160F31742C1F84021AC
:100AB0007047A648D0F84001C0F3074070474FF494
:100AC000A072C0F3011302EB8312DFF888C200F0BA
:100AD0000F03800903EB43035CF82000002900EBBF
:100AE0008310815814BF41F0010121F001018150B0
:100AF0007047984A810952F8212000F00F0101EB5C
:100B0000410102EB8111C0F301104FF4A07202EB1E
:100B10008010085800F0010070478E4A810952F891
:100B20002110D1F8E01100F00F00012201F00701BF
:100B300002FA00F0084018BF012070474FF4A0727D
:100B4000C0F3011302EB8312DFF808C200F00F03B9
:100B5000800903EB43035CF82000002900EB8310BD
:100B6000815814BF41F0020121F002018150704709
:100B7000784A810952F8212000F00F0101EB410170
:100B800002EB8111C0F301104FF4A07202EB801050
:100B90000858C0F34000704781096F4A01EB4101DA
:100BA00002EBC10100F00F0201EBC201C0F3011022
:100BB00051F820007047684982091CD00122B2EB2D
:100BC000901F18BF704765480068C0F3080088612F
:100BD00063480268C2F308420A620068C0F3080072
:100BE000486260480268C2F308428A620068C0F343
:100BF0000800C86270475548D0F82421C2F30802A3
:100C00000A60D0F8E421C2F308428A60D0F8E421F7
:100C1000C2F30802CA60D0F8A422C2F308420A61F3
:100C2000D0F8A402C0F30800486170472DE9F00332
:100C30000122830900F00F01C0F3011CC0F301166B
:100C400022EA0C0C00290BBF02254D1E00224FEAA0
:100C50000C124FF0080404EBCC043F4F03EB430CA1
:100C600007EBCC0C0CEBC101DFF8E88051F82660F3
:100C70004FF4587C58F823100CEBC50551F805C00B
:100C800000F00F001CF0010F00EB40004FF4927CCD
:100C90000CEB801C40F2FF1729D02C48D0F84403FD
:100CA0004FF032090005000D06FB09F60EBF0120CA
:100CB000B6FBF0F0401CFF2888BFFF204E594FF0D4
:100CC000FF0909FA04F9C0B226EA0906A040304338
:100CD000485158F8230050F80C3007FA02F123EA83
:100CE0000102114340F80C10BDE8F003704751F8C1
:100CF0000C0007FA02F39843C6F3080303FA02F262
:100D0000104341F80C00BDE8F003704710B5002017
:100D1000FFF78CFF0120FFF789FF1120FFF786FF07
:100D20000220FFF783FF1220FFF780FF4020FFF72C
:100D30007DFF4120FFF77AFF5120FFF777FF422028
:100D4000FFF774FFBDE8104052206FE700500040ED
:100D5000605B00409C550200D4890010245900407B
:100D6000E4590040A45A00402DE9F04707464FEAF5
:100D70009016FF480D0050F826404FF0000020620A
:100D8000C4F84001C4F80002C4F84002C4F8C0022C
:100D9000C4F8000308BFBDE8F087286820606868D1
:100DA000606061680120002908BF6060F149086047
:100DB000A868A060E868E0602869A0616869E061EF
:100DC000E8696062286AE06221206063E063686A23
:100DD0002064A86A6064E86AA064286BE064686BB9
:100DE0002066A86BA066E86B6067286CA067686CDB
:100DF000E067A86CC4F88000E86CC4F88400286D33
:100E0000C4F88800686DC4F88C00A86DC4F8900020
:100E1000E86DC4F8A400286EC4F8A800686EC4F891
:100E2000AC00A86EC4F8B000E86EC4F8B400286F37
:100E3000C4F8B800686FC4F8BC004FF0FF30C4F8C5
:100E4000E400A86FC4F8F000E86FC4F8F400D5F827
:100E50008000C4F8FC004FF4107205F1840104F521
:100E600080701FF095F8D5F8C40220F48030C4F8E3
:100E70004003D5F8C802C4F84C03D5F8CC02C4F836
:100E80005003D5F8D002C4F85403D5F8D402C4F8FE
:100E90005803D5F8D802C4F85C03002005EBC00263
:100EA000D2F8DC3204EBC001C1F86033D2F8E022A2
:100EB000C1F86423401C0328F0DBD5F8F402C4F821
:100EC0007803D5F8F802C4F87C03D5F8FC02C4F81E
:100ED0000004D5F80003C4F80404D5F80403C4F8EA
:100EE0000804D5F80803C4F80C04D5F80C03C4F8BA
:100EF00010040022002104EBC20805EBC20000EB45
:100F00008103D3F8109308EB810CCCF83094D3F81C
:100F10003893CCF85894D3F86033CCF88034491C1B
:100F20000229ECDB05EB8200D0F8883304EB820168
:100F3000C1F8A834D0F89C33C1F8BC34D0F8B00361
:100F4000C1F8D004521C052AD4DB002E14BF8A48F5
:100F50008A48006830F0FF0105D1D4F8901060F3A2
:100F60000301C4F89010D4F8500320F00100C4F835
:100F70005003D4F8600320F00100C4F86003D4F8F3
:100F8000680320F00100C4F86803D4F8700320F06F
:100F90000100C4F870033846BDE8F0470BE6784816
:100FA0000078704776484078704775498870704778
:100FB0007348807870477349D1F8542360F309026D
:100FC000C1F8542370476F48D0F85403C0F30900A8
:100FD00070476B4948607047694840687047684986
:100FE000886070476648806870476549C860704788
:100FF0002DE9F05F04460027384614F4803F18BFFF
:10100000012014F4003F18BF40F0040014F4802FB6
:1010100018BF40F0020014F4002F18BF40F0100079
:1010200014F4001F18BF40F0400014F4800F18BFE4
:1010300040F0080014F4000F18BF40F02000DFF863
:101040004081DFF8409198F8021010EA0105D9F8C4
:10105000400320F48030C9F8400336D0D8F80C6043
:10106000D9F84803002740F00100C9F84803D9F82F
:10107000480320F00100C9F84803D9F8400340F4C0
:101080008030C9F840034FF0630ADFF8FCB016E087
:1010900004F013F95046D9F8481311F0010F0AD0A3
:1010A000D9F844030005000D1CBFBBFBF0F0C8F8E5
:1010B0000800012703E0011EA0F10100EBDC301E57
:1010C000A6F1010601DD002FE2D0D9F8500320F08F
:1010D0000100C9F85003D9F8600320F00100C9F8F5
:1010E0006003D9F8680320F00100C9F86803D9F853
:1010F000700320F00100C9F87003244A106820F042
:10110000010010602248016821F0010101602149BD
:101110000B6823F001030B60F7B315F0010F05D046
:10112000D9F8503343F00103C9F8503315F0040FD8
:1011300005D0D9F8703343F00103C9F8703315F0C6
:10114000020F05D0D9F8603343F00103C9F86033CA
:1011500015F0100F05D0D9F8683343F00103C9F832
:10116000683315F0400F19D00B6843F0010314E009
:101170009C55020004580040F0FE0400E0FE04000C
:10118000208400100050004080F0FA02605B0040B4
:10119000685B0040705B00401AE00B6015F0080FC0
:1011A00003D0116841F00101116015F0200F03D048
:1011B000016841F00101016088F80150012088F8C0
:1011C0000000D9F8400340F48030C9F8400321E022
:1011D000002088F80100ADB1022088F80000D9F89D
:1011E000400340F48030C9F84003D9F8480340F088
:1011F0000100C9F84803D9F8480320F00100C9F8F4
:10120000480307E0D9F8401321F48031C9F84013AE
:1012100088F80000D9F8400114F0010F20F00D000B
:1012200018BF40F0010014F0040F18BF40F0040094
:1012300014F0020F18BF40F00800C9F84001D9F8B7
:10124000000214F0100F14BF40F0010020F0010064
:10125000C9F80002D9F8400214F0200F14BF40F082
:10126000010020F00100C9F84002D9F8C00214F0D2
:10127000400F14BF40F0010020F00100C9F8C00287
:10128000D9F8000314F0800F14BF40F0010020F0E3
:101290000100C9F80003FF4814F4805F016814BF1F
:1012A00041F0010121F001010160FB4814F4005FED
:1012B000016814BF41F0010121F001010160F7480C
:1012C00014F4804F016814BF41F0010121F00101C5
:1012D0000160F34814F4004F016814BF41F00101AC
:1012E00021F001010160EF49086814F4807F20F0CB
:1012F0000D0018BF40F0010014F4806F18BF40F0DB
:10130000040014F4007F18BF40F0080008600020BB
:10131000FFF78CFC0120FFF789FC1120FFF786FC0A
:101320000220FFF783FC1220FFF780FC4020FFF72C
:101330007DFC4120FFF77AFC5120FFF777FC42202B
:10134000FFF774FCBDE8F05F52206FE42DE9F04F29
:10135000840900F00F0343EA8411D34D4FEA911C36
:10136000C1F3011855F82C6003EB430C06EB8C1706
:101370004FF4A07606EB8818024657F80870002054
:1013800017F0010F10D141F010018F09C1F30111C5
:1013900055F8277006EB811107EB8C17795811F07F
:1013A000010F08BFBDE8F08F55F82410CF6907F092
:1013B000080801EB8C17D7F80011DFF8F0A204EB56
:1013C000440C0AEBCC0C1FFA81F902F00F05002146
:1013D00003EB43060CEBC505C2F3011A43EA011205
:1013E00042EA8412DFF8C0C2C2F3811B5CF82BC052
:1013F000C2F3011B4FF4A0720CEB861C02EB8B12A4
:101400005CF8022012F0010F1AD007EB811C55F88E
:101410002A20DCF844B1B8F1000FCBF3080B0EBF63
:101420004FF0000CDCF844C1CCF3023C02EBC20EDE
:101430000EEB021200EB42000BFA0CF202FB090069
:10144000491C0229CAD3BDE8F08F2DE9F041850976
:10145000AA0195489309002450F82300D0F84011C0
:1014600011F0010F34D0914E03EB430306EBC3039D
:1014700002F00F0603EBC603C2F3011211F0040FD2
:1014800053F82220D0F8003101F0080C9EB2D0F8B9
:101490004431C3F3080318BFC1F30744C769C1F35C
:1014A000052117F0080F1ABFD0F84401C0F302302D
:1014B0000020BCF1000F18BF491C03FA00F001FB2B
:1014C000004002EBC201704301EB021100EB41044A
:1014D000012040EA8510FFF739FF0646022040EA66
:1014E0008510FFF733FFA1190844BDE8F08110B55E
:1014F0000020FFF7AAFF4FF47A7148434CF25031B5
:10150000B0FBF1F010BD6A484068C0F30C007047B2
:1015100070B504460020FFF798FF05464020FFF70E
:1015200094FF35B3624BB0B141F288310844A84210
:1015300011D9421B186800F01F0104FB01F000EBF9
:10154000C00C0CEB0010B2EB400F04D93220484322
:10155000B2FBF0F0441CB4F5005F28BF41F6FF7405
:1015600002D2002C08BF0124586864F30C005860B4
:1015700070BDB4F5005F28BF41F6FF7402D2002CA5
:1015800008BF01244B48016864F30C01016070BD81
:101590002DE9F041464F0646386810F01F0508BF98
:1015A00001250020FFF751FFDFF80C810446002ED3
:1015B00018BF002C3FD0414900204A68002A08BFCC
:1015C00001223309B3FBF2F1D7F850C31CF0010F2D
:1015D0001BD0B3EB420F1DD33949B1FBF2F3B6FB7D
:1015E000F2F10A09B3FBF4F1102928BF0F218A4256
:1015F00098BF114639B1012984BF01FB1430B0FBFB
:10160000F1F007D908E0012109E0B8FBF6F2A242A7
:1016100088BF101B0029F6D0102988BF0F21D7F8EA
:101620005C2361F30302C7F85C2332216943B0FBFA
:10163000F1F0FFF76DFF7868C0F30C00684300EB32
:10164000C00101EB001004EB4000B8FBF0F0BDE876
:10165000F08170B5164D0024D5F8500310F0010F3D
:1016600008D01648D5F85C13406801F00F014843D4
:1016700004012DE00020FFF7E8FE024628686968B3
:1016800000F01F00C1F30C01414301EBC10000EB6E
:10169000011017E0005A0040405A0040C05A004074
:1016A000005B0040405900409C550200D489001066
:1016B00000500040045800400008AF2F2084001064
:1016C00080F0FA0212EB40001CBFFE49B1FBF0F4BF
:1016D000204670BD002818BF0120FB49D1F85C23CB
:1016E00060F30302C1F85C237047F748D0F85C034D
:1016F00000F00F0070478109F44A00F00F0000EB82
:10170000400052F821104FF4807202EB801008580C
:10171000EF4980B2B1FBF0F0401C400870472DE962
:10172000F041EA4B8209DFF8A8C353F8223000F0F9
:101730000F0731B1BCFBF1F1491C4A08B2F5004F6B
:1017400001D347F6FF72BCFBF2F1491C4D08D3F8F8
:1017500080104FEA520C01F00704D3F88010DB4BE5
:101760004FEA9018C1F3031600F00F0153F8283028
:1017700001EB410103EB81112FB3D1F80431F61CC9
:1017800074439BB2A2EB4404D1F8006124F001043D
:1017900062F30F06C1F80061D1F800216CF31F421B
:1017A000C1F80021D1F8042163F30F02C1F804212C
:1017B000D1F8182164F30F02C1F8182101F090F854
:1017C0002846BDE8F081F61CACF10E037443A3EB90
:1017D0004404D9E78109BD4A00F00F0000EB400046
:1017E00052F821104FF4807202EB80100858000C60
:1017F0007047830910F00F02B44850F8230002EB41
:10180000420300EB8313D3F800C161F31F4CC3F80C
:1018100000C118BF7047D0F8802002F00703D0F84D
:101820008020C2F30312D21C5A430E39A1EB4202AC
:10183000D0F8043122F0010261F30F03C0F8043143
:10184000D0F8181162F30F01C0F8181170479F4AC1
:10185000810952F8212000F00F0101EB410102EB58
:101860008111C0F301104FF4A27202EB80100858EE
:10187000C0F308007047F0B4944B840900F00F0CDB
:1018800053F824300CEB4C0503EB8516C0F3011222
:10189000D6F81C5106EB82164D1BD6F8447161F345
:1018A0000807C6F844714CEA021141EA841101F0BC
:1018B0000F02C1F3011101EB4201864A03F5C07327
:1018C00052F821104A08C90753F822C0C90E40F245
:1018D000FF148C402CEA040CAD1EC5F3080404FA76
:1018E00001F14CEA010143F82210F0BC00F0F8BF0E
:1018F000830900F00F01C0F30112744850F823006F
:10190000C36901EB410100EB811013F0100FD0F817
:10191000281100EB8210C9B2D0F84401C0F30800CE
:1019200008BF0021401A0004000C08BF01207047C6
:1019300003091B0203EB810101F1405101F5003164
:101940000007C00E0B6802FA00F0184308607047E9
:101950000209120202EB810101F1405101F500314F
:1019600000070968C00E21FA00F000F0030070477C
:1019700070B4DFF858C1820900F00F035CF8225000
:1019800003EB4303C0F301104FF4A87605EB831576
:1019900006EB80160C68AC515CF82220496802EB1B
:1019A00083124FF4AA7303EB8010115070BC704780
:1019B00030B4DFF818C1820900F00F035CF8224050
:1019C00003EB4303C0F301104FF4A87504EB831439
:1019D00005EB801564590C605CF8222002EB831241
:1019E0004FF4AA7303EB80101058486030BC704766
:1019F000364910B4820983B051F8222000F00F015B
:101A000001EB410102EB8111C0F301104FF4A87208
:101A100002EB80128A5800924FF4AA7202EB8010F7
:101A200008580190002001466A4601234FEA511CE4
:101A300001F01F0452F82CC003FA04F41CEA040F4E
:101A400018BF401C491C2629F0D303B010BC7047B6
:101A500030B4002210F00F0F06D000F00F02C0F3D8
:101A6000011303EB4202521E184B80094FF48665A6
:101A700053F8204005EBC205D1F800C044F805C07A
:101A800053F8200040F2344303EBC202496881500E
:101A900030BC704710B4002210F00F0F06D000F0D9
:101AA0000F02C0F3011303EB4202521E074B8009E1
:101AB0004FF4866453F820C004EBC2045CF804C001
:101AC0000AE000000008AF2F005000409C550200C3
:101AD000A0860100A4550200C1F800C053F8200000
:101AE00040F2344303EBC2028058486010BC704798
:101AF000FE48C06870470022FD49830951F8231051
:101B0000CB6913F0080F0ED000F00F0202EB420277
:101B100001EB8211C0F301104FF4A27202EB8010AE
:101B20000858C0F3023210467047DFF8C4C310B43F
:101B300082095CF82230DC6944F00804DC615CF85E
:101B4000223000F00F0202EB420203EB8212C0F3DC
:101B500001134FF4A27000EB8310135861F30E339E
:101B6000135010BC70470022E149830951F823103B
:101B7000CB6913F0080F0ED000F00F0202EB420207
:101B800001EB8211C0F301104FF4A47202EB80103C
:101B90000858C0F3024210467047D54A830952F8EC
:101BA000233000F00F0202EB420203EB8212C0F37B
:101BB00001134FF4A47000EB8310135861F3124328
:101BC00013507047042988BF70472DE9F0030027A0
:101BD000DFF81C83840958F82430DA69C0F3011C4B
:101BE00012F0080F4FF4A27202EB8C1C00F00F02EF
:101BF00002EB420205D003EB821555F80C50C5F3F9
:101C00000237DD69002615F0080F4FF4A475C0F304
:101C1000011005EB801504D003EB82104059C0F38E
:101C20000246C91B7018042803DD081A011D042090
:101C300003E00028BCBF014400207E18D96941F0B0
:101C40000801D96158F8241001EB821151F80C30C9
:101C500066F30E3341F80C3058F8241001EB821172
:101C60004A5960F312424A51BDE8F0037047A04A56
:101C70008009002952F82000816914BF41F0080151
:101C800021F00801816170479949800951F82000CD
:101C90008069C0F3C0007047954A8009002952F856
:101CA0002000816914BF41F0020121F0020181612D
:101CB00070478F49800951F820008069C0F34000C7
:101CC00070478B4B820953F8223000F00F0202EB71
:101CD000420203EB8212C0F301104FF4A67303EB30
:101CE000801011507047824A810952F8212000F07B
:101CF0000F0101EB410102EB8111C0F301104FF420
:101D0000A67202EB801008587047784A10B4D2F8D7
:101D1000400110F0010F0BD0D2F84C01D2F8441161
:101D20000028C1F302311EBF0029C043C2F84C0194
:101D30000123002003EB43018C0104EB801101F12E
:101D4000804101F5A041D1F8402112F0010F0CD0E3
:101D5000D1F84C21D1F844C1002ACCF3023C1EBF7B
:101D6000BCF1000FD243C1F84C21401C0228E4D33F
:101D70005B1C032BDDD310BC704700225C49830938
:101D800051F82310CB6913F0080F0ED000F00F02AA
:101D900002EB420201EB8211C0F301104FF4A47276
:101DA00002EB80100858C0F3005210467047012023
:101DB00070472DE9F04F82B0022ADDE90B49DDF8CA
:101DC000348026BF921E4FEA520C4FF0000C022BBB
:101DD00026BF9A1E53080023464AA2FB0442170955
:101DE000B8F1000F14BF012200220192B9F1020FD5
:101DF00016BF5FEA09024FF0010B4FF0000B82099A
:101E00003B4C00F00F0606EB460554F822404FF419
:101E1000B27E04EB851AC0F301140EEB841ECDF8DC
:101E200000A05AF80EA061F35C6A6BF3186A05D142
:101E300067F3174A63F3CA1A6CF3C60A019969F388
:101E4000420A61F3000A0099DFF8A49041F80EA05D
:101E500059F822204FF4B471C0F3011A01EB8A1132
:101E600002EB8512B8F1000F555814BF45F08005FC
:101E700025F0800555500125B5EB901F1CBF02B021
:101E8000BDE8F08F04EB46001B4951F820201831C3
:101E900011F8208006EB4600800100EB841000F171
:101EA000804000F5A040D0F850491449FF26A1FB1E
:101EB00002914908A1EB81094A44D2009640FFB241
:101EC00097404FEA8802002003F00F0393400CF084
:101ED0000F0C4FF00F090CFA02FC09FA02F24FEA5C
:101EE000810805FA00F121422DD009E000500040A0
:101EF0009C550200CDCCCCCCBC550200ABAAAAAA02
:101F000008EBC00101F1804101F5A041D1F8809CAE
:101F100029EA060949EA0709C1F8809C810001F114
:101F2000804101F5A041D1F8A89C29EA020949EABB
:101F30000309C1F8A89CD1F8BC9C29EA020949EA26
:101F40000C09C1F8BC9C401C0528CAD302B0BDE8EE
:101F5000F08F2DE9F04F84B0DDE90EA8DDF834C034
:101F6000B8F1000F14BF012400240294BAF1020F4B
:101F700016BF5FEA0A044FF0010B4FF0000B840913
:101F8000FA4D00F00F0707EB470655F824504FF4C1
:101F9000B27E05EB8619C0F301150EEB851ECDE967
:101FA000009E59F80E9061F35C696BF318697CD060
:101FB00002996AF3420961F30009DDE9001BDFF8C9
:101FC000ACA341F80B904FF4B4715AF82440C0F31D
:101FD000011901EB891104EB8614B8F1000F665862
:101FE00014BF46F0800626F0800666500126B6EB48
:101FF000901F1CBF04B0BDE8F08F05EB4700DC4923
:10200000DC4C51F8201054F8204007EB47008001C9
:1020100000EB851000F1804000F5A040D0F8500999
:10202000D54DFF26A5FB01756D08A5EB8507394445
:102030004FEAC109009006FA09FE00200F21A40012
:10204000A1404FEA850B012505FA00F6009D2E42BE
:1020500041D01568022D26BFAD1E6D080025121D4A
:102060001E68022E26BFB61E760800265CF8048B7A
:10207000C24FA7FB08874FEA07580BEBC00707F1D1
:10208000804707F5A047D7F880AC4FEA18682AEADE
:102090000E0A08FA09F84AEA0808C7F8808C87008F
:1020A00007F1804707F5A04700E01AE0D7F8A88CB1
:1020B00006F00F0628EA0108A64048EA0606C7F817
:1020C000A86CD7F8BC6C05F00F058E43A5403543CE
:1020D000C7F8BC5C1B1D401C0528B4D304B0BDE888
:1020E000F08F1168022926BF891E49080021D3F804
:1020F00000B0BBF1020F26BFABF1020B4FEA5B0B46
:102100004FF0000BCDF80CB0DFF870B2DCF800E057
:10211000ABFB0EEB4FEA1B1B6BF31749DDF80CB062
:102120006BF3CA1961F3C60942E72DE9F00F8F4D31
:1021300084094FF4B27955F8244000F00F0505EBFF
:10214000450604EB8614C0F3011609EB8619DDE998
:10215000098754F80940DDF820C0C4F3436BC4F389
:10216000410904F0010A002918BFC1F800B0B8F114
:10217000000F18BFC8F80090002F18BFC7F800A0C4
:1021800081094FF001085BD0B8EB901F1CBFBDE880
:10219000F00F704706EB45007549764C51F820105A
:1021A00054F820B005EB4500800100EB861000F1EB
:1021B000804000F5A040D0F850A96F4C0020A4FB4F
:1021C000015464084FEA8409A4EB84042144CF003D
:1021D0004FEA8B0508FA00F111EA0A0F2AD009EB41
:1021E000C00101F1804101F5A041D1F8801CF94006
:1021F000840004F1804404F5A044C9B2D4F8A86C6A
:10220000D4F8BC4CEE4006F00F06EC4004F00F048E
:102210001AB16400A41C42F8044B1BB17400A41C46
:1022200043F8044BBCF1000F04D001EB810189009D
:102230004CF8041B401C0528CCD3BDE8F00F7047B8
:10224000C4F30740C4F3C311C4F3C30412B1640060
:10225000A41C146013B14900891C1960BCF1000F63
:1022600004BFBDE8F00F704700EB80008000CCF8A1
:102270000000BDE8F00F70473C4A8009002952F881
:102280002000C16914BF41F0200121F02001C1618B
:1022900070473649800951F82000C069C0F34010EA
:1022A000704730B490B000224FF48045EC466C107B
:1022B00001E0082A05D2531C03EB8303B5FBF3F3BB
:1022C00004E0D31F03EB8303B4FBF3F35B1A48BFB3
:1022D0005B424CF82230521C102AEAD30023009CA7
:1022E00001215CF82120A242BCBF14460B46491CC8
:1022F0001029F6D300F00F0202EB42014FEA8111E0
:10230000C0F3011C01EB8C1101F18041840901F53E
:10231000A04135D00124B4EB901F1EBF10B030BCDB
:1023200070470CEB4200D1F850C9124A12F8202035
:102330000F25910000208D4003F00F028A4004FA1F
:1023400000F111EA0C0F0AD0810001F1804101F582
:10235000A041D1F8D03CAB431343C1F8D03C401C62
:102360000528ECD310B030BC704700009C5502002B
:10237000BC550200D4550200ABAAAAAACDCCCCCC45
:10238000D1F8680163F30300C1F86801EAE7810945
:102390001CBF0020704700F00F0101EB41018901D3
:1023A000C0F3011001EB801000F1804000F5A04067
:1023B000D0F8680100F00F00082834BF401CC01F8F
:1023C00000EB800034BF4FF480414FF40051B1FB6B
:1023D000F0F070472DE9F0074FF0010991B0B9EB2B
:1023E000901F1EBF11B0BDE8F007704700F00F024C
:1023F000C0F3011000EB420302EB4202920102EB38
:102400008010DFF83CC500F1804000F5A0405CF88A
:102410002330D0F850A90F204FEA83084FF0000C6A
:102420004FF480466C4600FA08F709FA0CF010EAFF
:102430000A0F36D051F8043B00204FF4005501E05C
:10244000082805D2421C02EB8202B6FBF2F204E03D
:10245000C21F02EB8202B5FBF2F2D21A48BF52420F
:1024600044F82020401C1028EAD30025009B0120BE
:1024700054F820209A42BCBF13460546401C102841
:10248000F6D34FEA8C0000F1804000F5A040D0F870
:10249000D02C05F00F03BA4303FA08F31A43C0F82F
:1024A000D02C0CF1010CBCF1050FBED311B0BDE86E
:1024B000F007704770B40124B4EB901F1CBF70BCD0
:1024C000704700F00F02C0F3011000EB420302EB73
:1024D00042029201DFF868C402EB801000F18040F4
:1024E00000F5A0405CF82330D0F850C900209B00D4
:1024F0004FF480456E1004FA00F212EA0C0F16D069
:10250000820002F1804202F5A042D2F8D02CDA40DB
:1025100002F00F02082A34BF521CD21F02EB8202C3
:1025200034BFB5FBF2F2B6FBF2F241F8042B401CCB
:102530000528E0D370BC704700F00F02C0F3011310
:1025400003EB4202FE4B8009A3F1380C53F8222022
:102550005CF8200001230029D0F8101403FA02F2DD
:1025600014BF11439143C0F81014704700F00F01DD
:10257000C0F3011303EB4101F14B0022800913F872
:102580002110383B53F82000D0F81004012303FA3F
:1025900001F1084218BF01221046704770B410F0D4
:1025A000300F14BF012300238609DFF898C300F021
:1025B0000F024FEA90104FF49A7502EB42025CF85A
:1025C00020004FF0010405EB821214D085584FEA29
:1025D000430C5B420CEB43039B1C04FA03F35B1EAE
:1025E00003FA0CF4194025EA040401FA0CF1214322
:1025F000815070BC70470029815804FA03F31ABF58
:10260000194381509943F3D070BC704730B410F037
:10261000300118BF012184094FEA9013C94D00F021
:102620000F0000EB40004FF49A7202EB801255F855
:1026300023004FF0010C0CD082584800C2404942A0
:1026400000EB4100801C0CFA00F0401E30BC104032
:10265000704780580CFA01F1084018BF012030BCC7
:102660007047B84B800953F820C0CCF8741053F869
:1026700020C01168CCF8781053F820005168C16769
:102680007047B1490028D1F8AC0014BF40F00200F7
:1026900020F00200C1F8AC007047AB490028D1F827
:1026A000AC0014BF40F0010020F00100C1F8AC0004
:1026B0007047A548D0F8E000A4490968084370476E
:1026C000A149C1F8E400A249086070479E48D0F8CB
:1026D0009800A049096840EA4100704770B44FEA89
:1026E0000075860900F00F044FEAD565C0F30110AC
:1026F000A5F1020502F0010C05444FEA8C334FEAC4
:10270000520012D001EB41017CB305EB4502D2002F
:1027100002EB8C3202EB810101EB800000F14050B2
:1027200000F5C030406A70BC704701EB410202EB1B
:1027300001117CB198226A4302EB8C3202EB8101D9
:1027400001EB800000F1405000F58030D0F88C0E95
:1027500070BC704703EB810101EB800000F1405039
:1027600000F58030006870BC7047FFE703EB810123
:1027700001EB800000F1405000F5C030006870BCF3
:102780007047F0B44FEA0076870900F00F044FEA73
:10279000D666C0F30110A6F1020602F0010C064451
:1027A0004FEA8C354FEA520012D001EB41017CB365
:1027B00006EB4602D20002EB8C3202EB810101EB08
:1027C000800000F1405000F5C0304362F0BC70471B
:1027D00001EB410202EB01117CB19822724302EB42
:1027E0008C3202EB810101EB800000F1405000F5DA
:1027F0008030C0F88C3EF0BC704705EB810101EBE6
:10280000800000F1405000F580300360F0BC70475C
:10281000FFE705EB810101EB800000F1405000F57E
:10282000C0300360F0BC7047830900F00F02C0F3B2
:1028300001100CD0002A08BF474805D0012A17D044
:1028400000280CBF4548464800EB81307047002AFD
:1028500008BF4FF04050F7D0012A04D000280CBF29
:1028600040484148F0E7002814BF40484048EBE7A3
:10287000002814BF3F484048E6E710B44FEA007C08
:10288000840900F00F034FEADC6CC0F30110ACF1D7
:10289000020C604410D0002B08BF38481CD000EB5D
:1028A0004000C00000EB813002EB420100EB8100F0
:1028B000334910BC08447047002B08BF31480BD087
:1028C0009823584300EB813002EB420101EB0211E7
:1028D00000EB81002C49ECE710BC00EB8130704725
:1028E0002DE9F0074FEA901C00F00F04154804EBA7
:1028F000440150F82C0000F5C07300EB8110D0F8B3
:1029000000014FF47A7280B2B2FBF0F100FB1120AB
:10291000002818BF01200D181C4F002040F2FF16A0
:1029200044EA001141EA8C1101F00F02C1F30111D8
:1029300001EB420157F821104A08C907C90E27E0E8
:10294000D45502009C55020000500040E058004061
:10295000E45800409858004000800030E481003086
:10296000248300304C1800304C1D0030CC0E003059
:10297000CC090030648100302480003000800130B8
:1029800024800130000001308C0E0130A45502007B
:1029900053F8228003EB820228FA01F8D2F80CA047
:1029A000A8EB050906FA01F8C9F308092AEA080A9A
:1029B00009FA01F14AEA0109C2F80C90D2F818901C
:1029C00029EA080848EA01019161401C0228A7D3BE
:1029D000BDE8F00770470000FEF716B810B5FEF727
:1029E00013F8012818BF10BD0020FDF7C8FF2121F2
:1029F0000020FEF70FF82121BDE810400120FEF76E
:102A000009B810B5FDF7B4FFFDF7FEFF01280AD1A4
:102A10000020FDF7B4FF21210020FDF7FBFF21215D
:102A20000120FDF7F7FF0121052001F03AFE012109
:102A3000052001F036FEF7490020887110BD10B561
:102A40004FF4066001F083FEBDE810404FF40660CD
:102A500001F06EBEEF4A01461079002818BF012030
:102A6000002918BF01211171002151717047E94AF5
:102A7000916A906208467047E6490020C8708870E5
:102A800048707047E3490020C870887048707047EC
:102A900010B5044601468422DF481DF079FA04F19E
:102AA0008401BDE810408422DC481DF071BA70B585
:102AB0000007C00E0D46801E00EB400101EB001424
:102AC000D7484FF4987200EBC40029461DF060FA15
:102AD000D44805F5987100EBC400BDE870404FF490
:102AE00098721DF055BADFF840C348B14A424FF41E
:102AF000806300EB810103EB820260461DF048BA5F
:102B00004FF4806160461DF048BA2DE9F04105465A
:102B10000020FDF7BDFFC54FDFF814830446EDB17B
:102B20004C2004FB00F21646294638461DF030FAC8
:102B3000324605F5BE6140461DF02AFA04EB44001A
:102B400000EB041407EB84004C211DF026FA08EB7F
:102B50008400BDE8F0414C211DF01FBA4C21401CFF
:102B600041430C4638461DF018FA21464046BDE860
:102B7000F0411DF012BA10B5A64C2062FEF738FAEB
:102B8000FEF70DFAA169A269C1F307216FF30F02E5
:102B9000A261A369C2B243EA0222A261022803D160
:102BA000A26942F00102A26181421ABFE269002AD1
:102BB00010BD012918BF0021012818BF0020814243
:102BC00008BF10BDBDE8104010474FF0402081699C
:102BD00041F002018161016941F00301016100F0EE
:102BE000EEBF2DE9F0414FF04022054690690C46BA
:102BF00040F002019161106940F00300106100F0A3
:102C0000DEFF0027002C7CD00020FDF7B8FE00205E
:102C10002168FEF7A9F840206168FEF7A5F828466C
:102C2000FFF7A9FF0020FDF764FF0126002832D03E
:102C3000A068FFF76AFF7C48636953B1E1694FF40C
:102C4000806C4A420CEB820203EB81011DF0A0F97B
:102C50001AE0784D4FF480611DF09FF9002029564D
:102C600000290EDB0A09120202EB800202F1405237
:102C700002F500320907C90E136806FA01F119437B
:102C80001160401C2628EAD36B48A16969B14FF452
:102C900000721DF07DF9E068A0B30120FDF729FF67
:102CA000DFF87C815F4E28B108E04FF400711DF021
:102CB00074F9F0E71120FDF71CFF68B1E5684046A4
:102CC0004FF4987229461DF063F930464FF498721C
:102CD00005F598711DF05CF90220FDF70AFF18B99F
:102CE0001220FDF706FF68B1E56854484FF498726A
:102CF00029461DF04DF952484FF4987205F5987128
:102D000001E017E001E01DF043F94120FDF7F1FE7D
:102D100018B95120FDF7EDFE60B1246954B1842249
:102D200021463D481DF034F9842204F184013B48DA
:102D30001DF02EF93748C770877047708762017998
:102D40000021017147714FF4066001F000FDBDE8FC
:102D5000F0414FF4066001F0EBBC10B50020FDF728
:102D60000EFE00F01CFF2B48406B002808BF10BD72
:102D70004FF04020016921F003010161816921F0D8
:102D80000201816110BD4FF4066001F0D6BC10B5A0
:102D90004FF4066001F0D1FCFDF736FE01280AD1A0
:102DA0000020FDF7ECFD21210020FDF733FE21215D
:102DB0000120FDF72FFE2348D0F8401321F4803185
:102DC000C0F840130020FDF7DAFD00F0E8FE1148DE
:102DD000406B002808BF10BD4FF04020016921F072
:102DE00003010161816921F00201816110BD10B50B
:102DF00001F0A8FC10F0600018BF012010BD054ACA
:102E0000D169D061084670470248006A704701489E
:102E100080697047308400100080013000C00130AC
:102E20008C0E01308C4E0130000002300000013069
:102E300000400130048A001000400230BC0F013015
:102E4000BC4F01300050004072B6FE498A6922EA48
:102E50000000886162B67047FA480078002818BF01
:102E60000120704770B5FDF7CFFD002818BF70BD79
:102E70000024F44DEC70AC706C7021212046FDF7FD
:102E8000C9FD21210120FDF7C5FD2C70BDE8704072
:102E90000120FDF774BD70B50446FDF7B5FD0028AF
:102EA00018BF70BD0021E74DE970A970697021213C
:102EB0000020FDF7AFFD21210120FDF7ABFD022C25
:102EC0003CBF0120FDF7B6FD012028706C62BDE813
:102ED0007040FDF754BD10B5FDF796FD002818BFF2
:102EE00010BD0020D74CE070A07060702121FDF76C
:102EF00091FD21210120FDF78DFD0120FDF79AFDB7
:102F0000012020706062BDE81040FDF738BD002050
:102F1000FDF735BD10B5CB4C0020A07060702121AD
:102F2000FDF778FD21210120FDF774FD20780028B0
:102F30001CBF0120FDF77EFD0120BDE81040FDF71C
:102F40001EBDC049C8627047BE48C06A7047BD49CF
:102F500008637047BB48006B7047BA4A00F00F0027
:102F6000116B21F00F01084310637047B54890F8CA
:102F7000300000F00F00704770B5B24C0546E06AB3
:102F8000421CE262216B11F0800F14BFC1F30211E9
:102F900001F00F0139B1B2FBF1F001FB1020002864
:102FA00008BFFEF7B2FE207850B1606A10B1606AC7
:102FB000401E6062606A002804BF0020FDF7DFFC4D
:102FC00020212846FDF726FDA16A00291CBF2846BE
:102FD0008847FDF7E4FF022815D19B48D0F8481335
:102FE00011F0010F0FD0D0F8481341F00101C0F8E3
:102FF0004813D0F8481321F00101C0F84813A06924
:1030000040F00200A0619148016841F02001016098
:1030100070BD0020B0E70120AEE710B5FFF749FB17
:103020000446FFF74DFB8A48044208BF10BD85489F
:10303000816941F0040181610E2101EAD43104F07B
:1030400001020A43816962F31F4181617F4801687F
:1030500041F02001016010BD002818BF012079490E
:10306000486370477B4870477B4870477548806B62
:1030700070477448C179427A914214BFC06B006CAA
:1030800070477048006C70472DE9F04F0025DFF85D
:10309000C4918DB009F14C04AC466F1E09F805705F
:1030A00004F805C06D1C262DF8DB0025002805DD81
:1030B000565D09F805606D1CA842F9DC0022012666
:1030C000CDF804C06D46CDF800C0002821DD19F907
:1030D00002B0BBF1000F19DBBBF1140FA8BFABF1BD
:1030E000140B04DABBF10A0FA8BF0BF1120BBBF1F2
:1030F000260F0BD24FEA5B180BF01F0B55F828A0D8
:1031000006FA0BFB4AEA0B0A45F828A0521C824239
:10311000DDDB002292460DF108084FEA521B02F057
:103120001F0E55F82BB006FA0EFE1BEA0E0F1ABF43
:1031300008F802A00AF1010A08F80270521C262AB7
:10314000EBDB4FF0000A002816DD19F90A20002AEF
:103150000EDB142AA8BF143A02DA0A2AA8BF1232D8
:10316000262A3ABF18F8022004F80A2004F80A7048
:103170000AF1010A8245E8DBDFF8C8900022002846
:10318000C9F838C009DD14F902A0924502D0C9F887
:10319000384002E0521C8242F5DB304A0020A2F1A6
:1031A0007204A2F1260A27540AF800C002F800C0EF
:1031B000401C2628F7DB0020002906DD13F800B0AC
:1031C00004F800B0401C8142F8DC0020CDF804C0B7
:1031D000CDF800C0002913DD2356002B0DDB262B74
:1031E0000BD24FEA531B03F01F0355F82BE006FAEE
:1031F00003F34EEA030345F82B30401C8842EBDB17
:10320000002003464FEA501B00F01F0E55F82BB06C
:1032100006FA0EFE1BEA0E0F1ABF08F800305B1C00
:1032200008F80070401C2628ECDB0020002919DD7E
:103230002356002B04DB262B3CBF18F80330135415
:10324000401C0DE0308400100050004084840010C9
:1032500001000700048A00102A8A00109C8A0010CE
:103260008842E5DB0020C9F840C0002908DD13567C
:10327000834202D0C9F8402002E0401C8842F6DBBD
:1032800011F0010F18BF252015D0420900F01F03CF
:1032900055F8222006FA03F31A420AD1420900F037
:1032A0001F0055F8223006FA00F0184345F82200B6
:1032B00001E0401EE9D500200246430900F01F0B43
:1032C00055F8233006FA0BFB13EA0B0F1ABF08F868
:1032D0000020521C08F80070401C2628EDDB00205E
:1032E00000290BDD2256002A05DB262A3CBF18F8F0
:1032F00002200AF80020401C8842F3DB0020C9F8B5
:103300003CC00029DCBF0DB0BDE8F08F1AF90020E9
:10331000824204D0C9F83CA00DB0BDE8F08F401C3B
:103320008842F3DB0DB0BDE8F08FFE487047FE48E1
:10333000406C70472DE9F001FA4C002282B0551E16
:1033400004F1050CA5540CF80250521C052AF9DBB7
:1033500000228B5CA354521C052AFADB00230127B0
:10336000194600280AD96256002A04DB052A3CBF08
:1033700007FA02F21343491C8142F4D300210A46A2
:103380006E4607FA01F818EA030F1ABF7254521C6E
:103390007554491C0529F4DB002100280AD962561E
:1033A000002A04DB052A3CBFB25C0CF80120491C52
:1033B0008142F4D3DC4B0021002859649EBF02B047
:1033C000BDE8F00170471CF901208A4205D0C3F81E
:1033D00044C002B0BDE8F0017047491C8142F2D3FD
:1033E00002B0BDE8F001704740F2DB114843CF491D
:1033F00001EB80007047CE49C0EB001001EBC0002C
:103400007047DFF824C3012B8CF807008CF80810F4
:1034100003D9401C20F0010011468CF809008CF8FB
:103420000A1000FB01F24FF6FF7101EA4202ACF80C
:10343000122001EA4000ACF814007047BA48807AC4
:103440007047B948407A7047B74AD07211737047D5
:10345000B548007B7047B448C07A7047B54A1070D1
:1034600051707047B349085C70472DE9F047DFF8A9
:10347000B892044699F80400002804BF99F80100A6
:103480001CF090FD99F80300002808BFBDE8F08704
:103490004FF00008D9F8200047464646454610F050
:1034A000070F1CBFDFF8848210F0020F05D0B9F8B7
:1034B00012109E4A21F001018F1810F0F00F18BF72
:1034C0009B4E10F4774F18BF9B4DD9F82C0020600D
:1034D000FDF768FD10F0010F06D0FEF706F902288F
:1034E00028BF99F8020000D20020E760C4E9010873
:1034F000C4E904650120BDE8F0878B480021C17054
:103500004171704770B505460020FDF7C1FA4C21A6
:1035100000FB01F21446894928461CF039FD224679
:1035200005F5BE60BDE8704085491CF031BDF0B5C1
:1035300083B00020FDF7ACFA044669460020FEF790
:1035400037FA0022002C2AD96E464FF0010C4FF6B4
:10355000F07502EB4200002100EB02104B0901F074
:103560001F0756F823300CFA07F73B4211D0CB0760
:103570005B0C03EB80034F0803EB870303F140531D
:1035800003F580331B889BB2AB4202D903B0002005
:10359000F0BD491C2629E1D3521CA242D9D303B065
:1035A0000120F0BD70B50007C00E0D46801E00EB77
:1035B000400101EB001463484FF4987200EBC40122
:1035C00028461CF0E5FC60484FF4987200EBC401FB
:1035D00005F59870BDE870401CF0DABC2DE9F04F9D
:1035E00007460007C00E83B0801E002527F03F0B62
:1035F000E9464FF001084FF6F0760290384665F341
:103600001F1040EA0B0000F0FF0A5046FDF771FA68
:1036100000283DD05046FEF76EFA08FA00F4022C5E
:1036200088BF022469465046FEF7C2F90022002CEA
:103630002ED902989821284400FB01FA02EB42009F
:10364000002100EB021C480901F01F0359F820007B
:1036500008FA03F3184215D001F001000AEB80309C
:1036600000EB8C004B0800EB830000F1405000F5AC
:103670008030B0F88C0E80B2B04203D903B0002085
:10368000BDE8F08F491C2629DDD3521CA242D5D3B8
:103690006D1C022DB2D303B00120BDE8F08F10B530
:1036A0000446842229491CF073FC04F18400BDE81F
:1036B0001040842226491CF06BBC2DE9F04F83B0EA
:1036C000002002904020FDF714FAE9464FF001086F
:1036D0004FF6F077F0B34020FDF7DAF9044669467B
:1036E0004020FEF765F90022002C3AD9002102EBB8
:1036F000420C480959F8203001F01F0008FA00F088
:1037000003420ED0C807400C00EB8C004B0800EBC6
:10371000830000F1405000F5C030008880B2B8420C
:1037200070D818E078840010308400103C1B011021
:10373000A82201103D8400109823011000000130E0
:10374000004001308C0E01308C4E01300080013081
:1037500000C0013005E0491C0529CAD3521CA24211
:10376000C4D301267000A0F1020B002546EA051023
:10377000C0B240F0400A5046FDF7BBF9C8B350460E
:10378000FEF7B9F908FA00F4022C88BF0224694652
:103790005046FEF70DF90021002C2AD90BEB05004D
:1037A00000EB40004FEAC00A01EB4102002002EBAF
:1037B000011C420900F01F0359F8222008FA03F304
:1037C0001A4210D000F001020AEB823202EB8C02A6
:1037D000430802EB830202F1405202F5C032928CA0
:1037E00092B2BA420ED8401C0528E2D3491CA1422D
:1037F000DAD36D1C022DB9D3701CC6B2022EB1D91A
:1038000001200290029803B0BDE8F08F2DE9F0414D
:1038100000268E4D00280C4645D000F00F01C0F365
:10382000011001290EBF00210229BDE8F081022804
:1038300028BFBDE8F0810F18FDF7E6F85FEA000841
:103840001CBF0020FDF79BF800239820474303EBA3
:103850004300002200EB031C02F0010007EB803064
:10386000510800EB8C0000EB810000F1405000F5A6
:103870008030521CC0F88C4E262AEDD35B1C022BE4
:10388000E5D3B8F1000F08BFBDE8F081AE706E70EF
:1038900021210020FDF7BEF821210120FDF7BAF813
:1038A0002878A0B330E0FDF7AFF807001CBF002078
:1038B000FDF765F8002303EB4300002200EB031043
:1038C000D107490C4FEA520C01EB800101EB8C0C43
:1038D0000CF1405C0CF5803C521CCCF80040262AD0
:1038E000EED35B1C312BE6D3002F08BFBDE8F0817F
:1038F000AE706E7021210020FDF78CF8212101208F
:10390000FDF788F8287810B10120FDF793F8BDE89D
:10391000F0410120FDF733B810B5FDF7E9FF4B4941
:10392000088210BD494B10B4E02101EA102C1B8A1B
:10393000C1B2C0F30422994288BF1946642461438E
:10394000B1FBF3F102EBC20303EB021201EB8201C4
:103950004FF47A723E4B0CFB02F2A3FB0232920848
:10396000521C520810F4803F08BF494210F4003F37
:1039700014BF8818881A00B210BC704710B5354CB7
:103980004FF4806134481CF008FB002001232156CD
:10399000002910DB0A09120202EB800202F14052F8
:1039A00002F500320907C90ED2F800C003FA01F18E
:1039B0004CEA01011160401C2628E8D310BD10B567
:1039C000244C4FF4806124481CF0E7FA00200123C6
:1039D0002156002910DB0A09120202EB800202F1D3
:1039E000405202F500320907C90ED2F800C003FAAE
:1039F00001F14CEA01011160401C2628E8D341F294
:103A0000EC0116481CF0C9FABDE8104041F2EC0187
:103A100013481CF0C2BA0D4810B5006A114908409D
:103A2000FFF7A9F84FF480610B481CF0B6FA40F696
:103A30008C610A481CF0B1FA40F68C6108481CF011
:103A4000ACFABDE810400020FDF762BD30840010E4
:103A5000ABAAAAAA048A00100000023000000130BC
:103A6000004001300100FF0082B04FF4FA62009084
:103A700013E000BF00BF00BF00BF00BF00BF00BF1A
:103A800000BF00BF00BF00BF00BF00BF00BF00BF3E
:103A900000BF0198411E0191EBD20098411E009198
:103AA00028BF0192F5D202B070472DE9F0410027FE
:103AB000634D0126002808BF2E701FD001282F70EB
:103AC00018BF6F701AD04FF04028D8F8100040F09F
:103AD0000400C8F8100029785A4C002914BF49F690
:103AE00008305948E06014BF58484FF0BB70A060E0
:103AF0005748006830F0FF0206D101E06E70E2E73F
:103B0000E26860F30302E26089B1A06840F0180047
:103B1000A0600120FFF7A8FFA06840F48050A060DB
:103B20000120FFF7A1FFA06840F40070A060012011
:103B3000FFF79AFF687870B1E06840F02000E0601D
:103B4000A06820F40070A0600120FFF78DFFE068FE
:103B500040F01000E060D4F8B00040F00100C4F87C
:103B6000B0000120FFF780FFE6674FF4E0602061BE
:103B7000C4F888702878002818BFC4F89460E068FA
:103B800020F03000E060A06820F49050A060D8F8E9
:103B9000100020F00400C8F81000BDE8F0812948AA
:103BA000C16821F03001C160816821F490518160C9
:103BB0004FF04020016921F00401016170474FF08E
:103BC0004020016941F0040101611D491D480A7846
:103BD0003AB1826842F018028260826842F49052E0
:103BE0008260497819B1C16841F03001C160D0F8F4
:103BF000B01041F00101C0F8B0107047B0F5007F7F
:103C000028BF40F2FF10C0F30800124941EA00202B
:103C10000C49086470470B494FF020400864704716
:103C2000084A116C4FF020401064506C11F0FF0FE7
:103C3000C0F308201CBF41F0204111647047000010
:103C4000828400100060004005F4010020009B0009
:103C5000D0FE0400130000A04FF0402000210163BB
:103C600002224263826B02F03C0242F00102826354
:103C7000026922F003020261026A22F0010202627A
:103C8000424A136843F0010313603C2282612822F8
:103C9000C2613F4801603F4801603F4850F88C2FA7
:103CA00042F4805202603D4A481E10603C48016068
:103CB000704710B501F0F9FA39480468002C08BFC4
:103CC00030BFFAD00021016001F0F3FA204610BDA8
:103CD00010B501F0EAFA324B00204FF040210122EA
:103CE0001C6824B1186001F0E4FA204610BD72B6D9
:103CF000D1F838C00CF03C0CC1F838C00A6320BFC2
:103D00000863D1F838C00CF03C0C4CF0010CC1F841
:103D100038C062B6BFF36F8FBFF34F8FE0E710B5C7
:103D200004460F2000F0F8FC0F2000F0DDFC1D49D8
:103D30000A6842EA0400086010BD1A490A6822EACB
:103D4000000008607047164A516850600846704786
:103D500070B51448006814490968114D00EA01045F
:103D6000696800291CBF2046884714F0100F05D051
:103D7000094850F88C1F41F48051016007480460E5
:103D8000286840F40040286070BD000000480040F2
:103D900024480040104800400030004014480040D3
:103DA000848400101C480040184800407047704749
:103DB0000022B2EBD10F26D20368B3F1FF3F04BF5C
:103DC0004368B3F1FF3F17D18368B3F1FF3F04BFEE
:103DD000C368B3F1FF3F0FD10369B3F1FF3F04BFE5
:103DE0004369B3F1FF3F07D18369B3F1FF3F04BFDC
:103DF000C369B3F1FF3F01D0002070472030521C4F
:103E0000B2EBD10FD8D30120704710B40023B3EB2D
:103E1000D20F30D2D0F800C00C68A44522D1D0F81F
:103E200004C04C68A4451DD1D0F808C08C68A445D6
:103E300018D1D0F80CC0CC68A44513D1D0F810C06C
:103E40000C69A4450ED1D0F814C04C69A44509D121
:103E5000D0F818C08C69A44504D1D0F81CC0CC6936
:103E6000A44502D010BC00207047203020315B1CDC
:103E7000B3EBD20FCED310BC012070472DE9F04137
:103E8000054601F01AFA002021264FF48257844695
:103E90004FF4E0221660C5F800C0116841F004013B
:103EA0001160116811F0040FFBD1176080232C46BC
:103EB0000021D4F80080B8F1FF3F04BFD4F804809B
:103EC000B8F1FF3F1DD1D4F80880B8F1FF3F04BF1F
:103ED000D4F80C80B8F1FF3F13D1D4F81080B8F1BA
:103EE000FF3F04BFD4F81480B8F1FF3F09D1D4F8E4
:103EF0001880B8F1FF3F04BFD4F81C80B8F1FF3F31
:103F000008D0C2F800C0401CC0B20828C2D30220AA
:103F1000BDE8F081491C2034B1EBD30FC9D3C2F8FE
:103F200000C00120BDE8F0812DE9F041054601F017
:103F3000C4F90020092684464FF4E0231E60C5F82A
:103F400000C0196841F004011960196811F0040FEC
:103F5000FBD12C464FF4806200212768B7F1FF3F68
:103F600004BF6768B7F1FF3F17D1A768B7F1FF3FFC
:103F700004BFE768B7F1FF3F0FD12769B7F1FF3FF3
:103F800004BF6769B7F1FF3F07D1A769B7F1FF3FEA
:103F900004BFE769B7F1FF3F08D0C3F800C0401C79
:103FA000C0B20328CAD30220BDE8F081491C2034E6
:103FB000B1EBD20FD1D3C3F800C00120BDE8F0812E
:103FC0002DE9F05F8846814604274FF07F0A4FF0C5
:103FD000020B4FF4E02601F070F949464246534681
:103FE0004FF0060CC6F800B052F8040B41F8040B71
:103FF000C6F800C0306810F0040FFBD15B1EF1D290
:10400000002030604C4645461F20D4E900C3D4E967
:104010000221D5F800E0E64504BFD5F804C09C4570
:1040200005D1AB68934204BFEA688A4208D07F1E7C
:1040300003D34846FFF722FFCDE70220BDE8F09FFB
:1040400010341035401EE0D20120BDE8F09F70B55D
:104050000D46044601F031F94FF40072214628461E
:104060001BF096FF012070BD2DE9F0410546C0050B
:10407000ADF5007D14460E46C00D25D0A8466FF361
:1040800008086F4601F019F94FF4007241463846AE
:104090001BF07EFFC5F30800C0F50077A74288BF7C
:1040A000274668443A4631461BF081FF4046FFF7F9
:1040B000E5FE022844D069464046FFF781FF02280A
:1040C00043D03D443E44E41BB4F5007F19D34FF484
:1040D0000072314668461BF06AFF2846FFF7CEFEA5
:1040E00002282DD069462846FFF76AFF02282CD007
:1040F000A4F5007405F5007506F50076B4F5007FAB
:10410000E5D2C4B16F4601F0D8F84FF400722946E9
:1041100038461BF03DFF2246314668461BF047FFFC
:104120002846FFF7ABFE02280AD069462846FFF76B
:1041300047FF022809D00DF5007D0120BDE8F08180
:104140000DF5007D0A20BDE8F0810DF5007D0B2006
:10415000BDE8F08130B4354D2A68002101244FF0CC
:10416000030C04FA01F3034204D04B000CFA03F3EE
:104170009A431A43491C0C29F3DB2A6030BC704770
:10418000F0B42A4D2A68002101244FF0030C0226C6
:1041900004FA01F3034206D04B000CFA03F7BA43CA
:1041A00006FA03F31A43491C0C29F1DB2A60F0BC20
:1041B00070472DE9F001002201251D4C0F2605FA5C
:1041C00002F3034217D0D31702EB537C4FEAEC0300
:1041D00004EB83031F682CF0070CA2EB0C0C4FEAD6
:1041E0008C0C06FA0CF827EA080701FA0CFC47EADF
:1041F0000C0CC3F800C0521C0C2AE0DB0B498A6A85
:1042000022EA00008862BDE8F001704707498A6A27
:104210001043886270470548416821F08001416081
:10422000416821F4007141607047000000100040B7
:1042300020100040704772B64FF04020816941F075
:1042400040018161C16941F04001C16162B6016A0A
:1042500041F00101016270474FF04020016A21F0F6
:104260000101016272B6C16921F04001C161816939
:1042700021F04001816162B6704710B572B64FF00F
:104280004024A06940F04000A061E06940F0400097
:10429000E06162B6206A40F001002062D94843F62E
:1042A0003F71C160002181638164C0F8D010032197
:1042B0000A2000F0F6F90A2000F016FA206A20F031
:1042C0000100206272B6E06920F04000E061A06960
:1042D00020F04000A06162B610BDCA4A1060516073
:1042E000484390607047C74A10605160484310F0DF
:1042F000010F18BF401C90607047C249C1F8D00040
:104300007047C049002818BF012088647047BD4924
:104310008863C86840F00200C8607047DFF8E4C2F4
:10432000CCF82000CCF82410CCF82820CCF82C3085
:104330000120CCF83000DCF8340010F0010F05D07B
:1043400020BFDCF8340010F0010FF9D110F00200AA
:1043500018BF4FF0FF307047AA48C16821F0020132
:10436000C1607047A748C16841F00101C160704752
:10437000A44B186259629A6201201864586C10F0BC
:10438000010F04D020BF586C10F0010FFAD110F0CB
:10439000060018BF4FF0FF3070479A48C16821F0FF
:1043A0000101C16070479748C16841F00401C160D4
:1043B0007047944A8189116701685162416891622E
:1043C0008168D16201211165516D11F0010F04D096
:1043D00020BF516D11F0010FFAD1536F0361936F3C
:1043E0001B148382936FC3F30523C382936F03F07F
:1043F0003F030383D36F1B144383D36FC3F305239E
:104400008383D36F03F03F03C383D2F88030C3F3B9
:1044100009430384D2F88020C2F30902428411F0D8
:10442000020018BF4FF0FF3070477648C16821F096
:104430000401C16070477348C16841F00401C16064
:104440007047027C017B02F03F0241EA02416D4A63
:10445000916501685162416891628168D162012170
:104460001165516D11F0010F04D020BF516D11F095
:10447000010FFAD1D36D8382D36D1B0CC382136EEF
:104480000383136E1B0C4383536E8383526EC2F3FC
:104490000E42C28311F0020018BF4FF0FF30704788
:1044A0005848C16821F00401C16070475548C1688F
:1044B00041F00801C1607047DFF848C1CCF898208E
:1044C000CCF82000CCF82430CCF828100120CCF80F
:1044D0009000DCF8940010F0010F05D020BFDCF84C
:1044E000940010F0010FF9D110F0060018BF4FF042
:1044F000FF3070474348C16821F00801C160704730
:1045000001684FEA31423F49C1F8BC204068C1F818
:10451000C000C86840F02000C860704701684FEADA
:1045200031423849C1F8BC204268C1F8C020027A43
:10453000407A02F0010262F35F00C1F8C400C8686B
:1045400040F02000C86070472E4B18625A62996292
:104550000120C3F8B400D3F8B80010F0010F05D063
:1045600020BFD3F8B80010F0010FF9D110F0060009
:1045700018BF4FF0FF307047224A1062516201208D
:10458000C2F8B000D2F8B80010F0010F05D020BF7B
:10459000D2F8B80010F0010FF9D110F0060018BFE2
:1045A0004FF0FF3070471748C16821F02001C1600B
:1045B00070471448C16841F01001C1607047A3F111
:1045C000050C104BC3F8A8C018625A62996201200A
:1045D000C3F8A000D3F8A40010F0010F05D020BF4D
:1045E000D3F8A40010F0010FF9D110F0060018BFA5
:1045F0004FF0FF3070470348C16821F01001C160DF
:104600007047000000900040234810B5022140F898
:10461000501F012101611021416241F206014161F7
:10462000002181610421816390214163416B41F04C
:1046300001014163C16B21F40021C163C16B41F4ED
:104640000051C163C16B21F00101C163C16B41F035
:104650000101C1634FF4817101610161032000F028
:1046600043F80021032000F01CF8002010BD10B515
:10467000032000F045F808484FF4807101660021DE
:1046800001661021816702214165002010BD0349A8
:104690000020087070470000003000408C8400103B
:1046A000704700F00303DA004FF0FF0C0CFA02F23F
:1046B0004FF0050C0CEBC30301FA03F300F00C01FF
:1046C00001F1E021002807DAD1F8140D90431A40D7
:1046D0001043C1F8140D7047D1F8000490431A40FC
:1046E0001043C1F80004704700F01F01012202FAD4
:1046F00001F14009800000F1E020C0F8001170478E
:1047000000F01F01012202FA01F14009800000F1CE
:10471000E020C0F88011704700F01F01012202FA6A
:1047200001F14009800000F1E020C0F880127047DC
:104730004FF0E021C1F8000170474FF0E021C1F8CF
:10474000800170474FF0E020D0F8000170474FF033
:10475000E021C1F880027047084800687047074AA6
:104760001168106008467047044A126800F110038F
:1047700052F8230042F823107047000008ED00E0D3
:1047800002210C20FFF78DBF72B64FF040208169E7
:1047900041F480518161C16941F48051C16162B6C7
:1047A000704772B64FF04020816921F480518161D9
:1047B000C16921F48051C16162B67047AA4881B0D5
:1047C000016F11F4007FFBD1816E11F0010F1CBF4E
:1047D000D0F88410009104D0D0F88410009A91424F
:1047E000FAD0016F11F4007F04BF4CF27101016631
:1047F00042F24131816601B070479B4981B04FF46C
:104800000D528A660A6FCA66012898BF012005D931
:10481000401EB0F5803F28BF4FF6FF7082B24FF0C8
:104820005C5040EA022048664FF01140C1F8800019
:10483000086F10F4007FFBD1886E10F0010F1CBFD1
:10484000D1F88400009004D0D1F88400009A9042FE
:10485000FAD0086F10F4007F04BF4CF271000866B4
:1048600042F24130886601B070477F4881B0016FE5
:1048700011F4007FFBD1816E11F0010F1CBFD0F845
:104880008410009104D0D0F88410009A9142FAD09C
:104890004FF40D51816601B070474FF040208069A0
:1048A00010F4805008BF70476F48806E00F0010020
:1048B00070476D48406EC0F30F2070476A48D0F8CB
:1048C0008400704710B50C20FFF726FF0C20FFF77F
:1048D0000BFF65490220486710BD634910B50320EE
:1048E00088670C20FFF70CFFBDE810400C20FFF795
:1048F00013BF5E4A11681060084670475A4810B5E9
:10490000016FC16659480068002818BF80475848A1
:10491000016841F48051016010BD544840687047FF
:1049200010B572B64FF04020816941F48051816129
:10493000C16941F48051C16162B603204A49886768
:104940000C20FFF7DDFE0C20FFF7E6FE00F03CF93F
:10495000484B0420C3F888004FF6FF70C3F88C0062
:1049600072B66033FFF749FF4FF40070186062B60B
:1049700010BDF8B572B63C48016F11F4007FFBD151
:10498000816E11F0010F1CBFD0F88410009104D08B
:10499000D0F88410009A9142FAD04FF40D518166FC
:1049A00034494FF400320A6662B6D1F804124FF06F
:1049B0004025002946D02D4C4FF6FF73591AA160AF
:1049C0002A6BD5F834C002F00F020CF00F0C6244D1
:1049D000121D01FA02F2A2F54341DFF89CC05139E1
:1049E00061452FD2D0F88400191AE160B1F5803FFB
:1049F00028D2224B4FF0000CA1FB03070CFB0373E2
:104A000001FB0C3163461BF0D7FA401C40082061C3
:104A1000B0F57A7F38BF4FF47A70194B9968002946
:104A200008BF98605A681A609968C3E901108A4201
:104A300015D9824205D9814201D9616002E06060E6
:104A400000E0626000F0D0F872B6A86920F48050EF
:104A5000A861E86920F48050E86162B6F8BD82423E
:104A6000EFD88142EBD8E8E700C000409084001006
:104A70008484001000A000404F62250000E1F5058D
:104A8000C48A00104FF04020816941F00401816127
:104A90000C48016841F404710160001F016821F0B5
:104AA00004010160016841F010010160704706498E
:104AB00008607047BFF34F8F054904480860BFF393
:104AC0004F8FFEE714ED00E008ED00E00400FA056A
:104AD0000CED00E04FF04020816941F0040181615C
:104AE0000B48016841F0010101600B490948C1F818
:104AF000C40070470948006842F2700108407047DE
:104B0000084807490160084981600021C160704779
:104B1000144C004001005FA00060004000440040D1
:104B2000A0C00E0000100040508A5900022824BF87
:104B300000207047DC4B53F8202043F8201010462B
:104B4000704770B5D94C206FD74D10F0010F05D0CC
:104B50000120E0662868002818BF8047206F10F009
:104B6000020F08BF70BD0220E0666868002808BF19
:104B700070BDBDE87040004710B572B64FF04020E0
:104B8000816941F080018161C16941F08001C161A9
:104B900062B60222C5490A6501230B660323CB6670
:104BA0004A6572B6816921F080018161C16921F095
:104BB0008001C16162B60920FFF796FD0221BDE8C0
:104BC00010400920FFF76DBD72B64FF0402081699B
:104BD00041F080018161C16941F08001C16162B62B
:104BE0000220B24908657047B0490220486572B694
:104BF0004FF04020816921F080018161C16921F07D
:104C00008001C16162B670474FF040208069C0F3F7
:104C1000C0107047A548016F11F4007F14BF4FF416
:104C200040714FF480710166704710B59F4CE06F82
:104C300010F0020F4FF0010018BF0320606700F072
:104C40006DF94FF040210A6B496B02F00F02D04022
:104C500001F00F01C8400521B0FBF1F04FF40571E0
:104C60000009C4F880109249A1FB00104009C4F863
:104C70008400206F10F4007F14BF4FF440704FF495
:104C80008070206610BD8948016F11F4807F14BFC9
:104C90004FF440714FF4007101667047834B30B49C
:104CA000DA6F12F0010F14BF032202225A6700EBE1
:104CB0004005C5EBC010C1EBC0004FF4FA744C4383
:104CC000C0EB001000EB40007A4904EBC000A1FBF0
:104CD00000104FF0402100220C6B4FF0020CC00876
:104CE000496B04F00F0401F00F012144C840052175
:104CF000B0FBF1F0B0F5803F05D3511C4008CAB2BB
:104D0000B0F5803FF9D242EA0C2141F01001C3F81E
:104D10008810C3F88C00186F10F4807F14BF4FF414
:104D200040704FF40070186630BC70475F48016FE8
:104D300011F4003F14BF4FF440314FF4803101664D
:104D400070475A48016F11F4803F14BF4FF440314F
:104D50004FF40031016670475448006FC0F30020E3
:104D600070475248006FC0F3402070474FF0402119
:104D70008969C1F3C011002904BF002070474B4965
:104D800000280CBFD1F80002D1F8040270474FF0A0
:104D900040239A69C2F3C012002A04BF0020704762
:104DA000424A00280CBFD2F88000D2F88800C0F335
:104DB0000A200CBFD2F88020D2F8882002F00F021F
:104DC000D3F830C05B6B0CF00F0C03F00F0363449F
:104DD0001A449140012202EB400048433449A1FBB0
:104DE000001000097047344901200870704770B402
:104DF00032224FF0402351431A6BD3F834C002F0F3
:104E00000F020CF00F0C6244121DD14008BF0121AB
:104E100004D0B1F5803F28BF4FF6FF719A69C2F305
:104E2000C012002A1CBF70BC704772B69A6942F06B
:104E300080029A61DA6942F08002DA6162B6022485
:104E40001A4A1465250415664FF0040CC2F888C090
:104E5000C2F88C10DFF864C0C2F86CC054671849FF
:104E600002283CBF104E46F8201000211248017065
:104E70004FF400711166017819B920BF017800293B
:104E8000FBD01566C2F878C0C2F86CC0546572B623
:104E9000986920F080009861D86920F08000D8617E
:104EA00062B670BC70470000A884001000A00040EB
:104EB0001F85EB51CDCCCCCCA484001002000202A3
:104EC000976D00004FF0E0210020886108612749BC
:104ED0004860704710B54FF0E02460610020A06189
:104EE0000221401EFFF7DDFB07202061BDE81040D6
:104EF00008F0C4BD10B508F0C5FD4FF0E02100205A
:104F0000086110BD10B508F0BDFD4FF0E021002094
:104F1000086116480188491C018010BD134880684B
:104F200070472DE9F041114C002705462780A06805
:104F30004FF47A71B0FBF1F04FF0E026401E706143
:104F4000B7610221C81EFFF7ACFB0720306108F0F3
:104F500095FD2188A942FCD308F094FD3761BDE896
:104F6000F08103494843014988607047B0840010CC
:104F700040420F004FF04020816921F400518161CF
:104F8000C16921F40051C1617047A8490A78824281
:104F900018BF062828BF7047A54AA64B52F830C054
:104FA000C3F808C002EBC0025268DA6008707047AC
:104FB0004FF04020816941F400518161C16941F4A1
:104FC0000051C161704710B501210720FFF769FB4F
:104FD0004FF04020816941F400518161C16941F481
:104FE0000051C161934A0021116093495160DFF87B
:104FF0003CC200219CF800303BB10CF110031C684E
:1050000094605B68D3608CF800108C4911618169F1
:1050100021F400518161C16921F40051C16110BDC9
:105020008248406870478348806970474FF040204D
:10503000806910F4005008BF70477E48006900F096
:10504000010070474FF04020806910F4005F04D0E9
:10505000784B186910F0010F01D10020704710B48F
:1050600072494FF6FE7000248A684AB19A69D1F8F5
:1050700008C0624504D08C604C6010BC01207047B1
:1050800000BF00BF00BF00BF00BF00BF00BF00BF28
:1050900000BF00BF00BF00BF00BF00BF00BF00BF18
:1050A00000BF00BF00BF00BF00BF00BF00BF00BF08
:1050B000401E0028D8DC8C604C6010BC002070477B
:1050C0005A49886070475948806870475948016953
:1050D00041F0010101615549012048607047554880
:1050E000016921F0010101615049002048607047C9
:1050F0000021002808BF4FF0006103D0022808BF3C
:105100004FF080614B48026922F040621143016117
:10511000704748490120096901F04061B1F1806F91
:1051200004BF02207047B1F1006F08BF0020704734
:105130004048406970473D48007870474FF0402034
:10514000806910F4005F38D03A4A106910F0010FFE
:1051500033D03648406801282FD090696FF07F43E4
:10516000984238BF00EB400C27D25169B1EB9C0F3D
:1051700001D30120704700BF00BF00BF00BF00BFC8
:1051800000BF00BF00BF00BF00BF00BF00BF00BF27
:1051900000BF00BF00BF00BF00BF00BF00BF00BF17
:1051A00000BF00BF00BF00BF00BF00BF00BF00BF07
:1051B00000BF00BF00BF9842D7D30020704710B592
:1051C0000720FFF7A9FA0720FFF78EFA19480169AF
:1051D00041F01001016110BD164810B5016921F0C0
:1051E000100101610720FFF78BFABDE8104007208E
:1051F000FFF792BA0D4AD168D0600846704738B5BB
:105200000C4CE069E061094910F0020F1CBFA26973
:105210008A60C96800291CBF00018847E0690090C6
:105220000748016841F08001016038BDBC8400106E
:10523000CC84001000D00040D0121300660F00157F
:1052400084840010704770B505464FF40D50040675
:10525000A0660320E066264860664CF27100206676
:105260002448C4F8800042F24630A06602210020A3
:10527000FFF717FA0020FFF737FA002D08BF70BDBF
:10528000A06E42F241310843A06670BD012110B505
:10529000880781674FF40D5181660020FFF730FACF
:1052A000BDE810400020FFF737BA012081074867AA
:1052B000704701208107886770474CF271008107B1
:1052C000086670470C4A11681060084670470A4823
:1052D00008B5006818B18047002818BF08BD4CF217
:1052E000710188070166016FC166006F009008BDFB
:1052F000075E5F3700AF2F91FC840010FE4900204D
:1053000088717047FC488079704770B5FA4C002569
:105310004FF4E4612570E570F8481AF03EFE4FF452
:10532000E461F7481AF039FEA56025714C21F54873
:105330001AF033FE4C21F4481AF02FFE65717421E7
:10534000F2481AF02AFE7421F1481AF026FEE560B0
:1053500070BDE9480079002818BF01207047E64871
:105360004079002818BF01207047E348C078002822
:1053700018BF01207047E548704770B5E54DE64E0F
:10538000044601462A783078E04B10444200184623
:105390001AF00DFE2A783078DD4B10444200214689
:1053A00018461AF004FED44801214171817941F078
:1053B0000401817170BDD048C0687047CF48704704
:1053C0002DE9F041CC4F80463878002814BFD348EF
:1053D000D348057814BFD348D348047805FB04F6B6
:1053E000FEF729FF21462846FEF777FFC3494346CB
:1053F000C34A0846FEF792FFFEF72EFF72004146B1
:10540000BF481AF0D4FD0120F870B87940F00100CF
:10541000B8710120BDE8F0812DE9F047B64D044692
:1054200001462878DFF8D4C2DFF8F082DFF8F09286
:10543000BC4EBD4F002815BF98F8002099F80020F9
:1054400033783B7802FB03F04FEA400260461AF0E3
:10545000AEFD2878DFF8A8C22146002815BF98F8CD
:10546000002099F8002033783B7802FB03F04FEAE4
:10547000400260461AF09BFD0120E870A87940F0D8
:105480000100A871BDE8F0879B488068704770B53F
:10549000A64C0546014622789A4852001AF087FD2C
:1054A00022782946520098481AF081FD924801213D
:1054B0000171817941F00201817170BD2DE9F04FD8
:1054C000ADF25C7DDFF830920120CDF8440799F809
:1054D0000300CDF8400799F80400CDF83C0799F88F
:1054E0000500CDF8380702F0B5F80446FDF774FA68
:1054F000CDF85807FDF7B0FCCDF85407FCF703F8DA
:10550000CDF85007FBF74EFD0746FBF748FD8046F8
:10551000FDF764FAFCF79DF80830050999F80100D9
:105520000026002804BF0420C9F8140010D002F09F
:10553000A9F88246022C1CBF0920C9F8140011D01A
:10554000BAF1060F04BF0220C9F8140089F80160FF
:10555000FBF728FD10F0010F14D002F0D6F93C281B
:105560000AD00FE015F055F810F4817F14BF3C20ED
:105570001E20C9F81400E3E7FFF758FD002818BF04
:10558000FFF7DCFD4FF0010AB8F1020F14D102F071
:105590006FF988B9022C04D0052C08BF052007D06C
:1055A0000AE04FF47A7068434FF47A7190FBF1F09F
:1055B000C9F8140089F801A0D9F814000428BCBF68
:1055C0000420C9F8140099F80100B9F81410000279
:1055D00040EA014040F001020023912107200CF035
:1055E000A9F917F0010F27D1022C25D00020FBF7D5
:1055F0008FFFFDF770FC37464FF0000B07F036F9D0
:1056000001281FD00DF5E460FDF72FFF002800F002
:10561000D4810DF5E46008F034F8D9F81400C01E08
:105620008642CABF874201250025DDF82C0748B312
:10563000DDF83C0750B144E0FDF714FC0020CDF844
:105640004407D8E74FF0010B00F0A1B96846DDF838
:105650002C171AF0B6FC8046ADB1344C4146207888
:10566000420028481AF0A3FC207841464200264810
:105670001AF09DFC89F804A099F8060040F0020099
:1056800089F806001DE0FEF7D6FD284C01212078A0
:10569000FEF723FE1C4A4346A2F14C010846FEF7E2
:1056A0003DFEFEF7D9FD20784146420016481AF02B
:1056B0007EFC89F804A099F8060040F0020089F801
:1056C0000600DDF8280700287ED0DDF84007002816
:1056D0007AD199F80000DDF8284748BBD9F808804E
:1056E000B8F1000F42D00D480078CDF84C070D48B6
:1056F0000078CDF848071CE000850010D023011089
:10570000D08A001030A000107CA00010F02A0110F8
:10571000C8A000106285001063850010608500102D
:105720005D850010618500105E85001064850010A5
:1057300035E0FEF780FDDDF84817DDF84C07FEF791
:10574000D2FD214642460846FEF712FEFEF784FDD2
:10575000FC480078022804BF404607F0B6FCF94830
:105760000078092804BF204607F0AFFCF64800780F
:10577000012814D9DFF8CC8398F80000042804BF6E
:10578000204607F0A2FC214668461AF01FFC04469A
:1057900098F80000052804BF204607F096FC8DB35A
:1057A000EA4899F800202146002A0CBFE84AE94A55
:1057B000127814BFE84BE94B1B7802FB03F24FEA67
:1057C00042021AF0F4FB00E055E099F80000E44BC7
:1057D0002146002814BFDF48DD48007814BFDE4AA8
:1057E000DE4A127800FB02F04FEA400218461AF037
:1057F000DEFB89F803A099F8060040F0010089F863
:10580000060031E0FFE7CDF8484799F8000000288E
:1058100014BFD048CE4890F8008014BFCE48CF487F
:10582000047808FB04F0CDF84C07FEF704FD214690
:105830004046FEF752FDC549C94A0846DDF84837DB
:10584000FEF76CFDFEF708FDDDF84C07DDF84817A4
:105850004200C3481AF0ABFB89F803A099F8060090
:1058600040F0010089F80600B6480078032804BF1C
:10587000B64807F02AFCDDF8300700287AD0DDF8BA
:105880003807002876D199F80000DDF8304748BB8A
:10589000D9F80C80B8F1000F24D0B2480178B24892
:1058A00000780844401C4008019002200090FEF758
:1058B000C2FCDDE90010FEF716FD2146424608460F
:1058C000FEF756FDFEF7C8FCA8480078022804BF82
:1058D000404607F095FDA5480078092804BF2046FA
:1058E00007F08EFDEDB1A2489E4DDFF87C82214687
:1058F0002B7898F800201A4452001AF058FB2A78A6
:1059000098F800309B481A44214652001AF04FFB89
:1059100089F805A099F8060040F0040089F806000F
:1059200021E09048254601788F4800780C18FEF752
:1059300082FC601C40080221FEF7CFFC8C492B46FC
:105940008C4A0846FEF7EAFCFEF786FC6200294610
:1059500088481AF02CFB89F805A099F8060040F059
:10596000040089F8060081480078032804BF8048B5
:1059700007F046FDFDF7C1FDD9F81400761C7F1C29
:105980008642A8BF874211DBD9F8100070B1FDF73D
:1059900025F8DDF85007FBF7BBFDDDF8580788B1A7
:1059A000DDF8540760B1FDF796FA0BE0DDF8440727
:1059B000002818BFFDF78FFA20E601F0A2FE1DE6D1
:1059C000FDF750FABBF1000F04BF0420C9F8140022
:1059D0000BD0DDF8400789F80300DDF83C0789F8B3
:1059E0000400DDF8380789F80500B9F814104FEA0B
:1059F0000B2040EA01420023912107200BF09AFF7F
:105A00000DF25C7D5846BDE8F08F10B50024FDF71F
:105A1000FBF9594910F0070F0AD0CA78002A08BFCD
:105A2000012410F0020F03D00A79002A08BF0124D4
:105A300010F0F00F03D04879002808BF012400209F
:105A4000002C08BF10BD00200870BDE8104035E5EF
:105A500008B540F20F3101F085FF012804D1FFF7AE
:105A6000D4FF009002F0F2F84348C17800291CBF2F
:105A70004179002904D0007900281CBF012008BD0D
:105A8000002008BD08B540F20F3101F06BFF01287E
:105A900004D1FFF7BAFF009002F0D8F83648C17879
:105AA00000291CBF4179002904D0007900281CBFBF
:105AB000012008BD002008BD70472F4910B5002205
:105AC000CA700A714A7100281CBF012048700CF08E
:105AD000CDFFBDE81040FAF786BC10B54FF4E46185
:105AE0001A481AF05AFABDE810404FF4E4611C4815
:105AF0001AF053BA214870471548017817480078C2
:105B0000484341001D481AF048BA70B5064610488F
:105B1000047812480578FEF78EFB29462046FEF7EA
:105B2000E2FB0A4A31461548FEF722FCFEF794FBD9
:105B300004480078152818BF70BD1048BDE87040B3
:105B400007F0C3BAE58500105F850010D02301106F
:105B50005D85001060850010618500105E85001075
:105B6000D08A00106285001063850010EB8500105C
:105B7000F02A0110C8A0001000850010F09100105C
:105B80002DE9F0470746FB4815460C460678FA48CB
:105B900090F80080FEF74FFB41463046FEF7A3FB2E
:105BA0003A46F6491046FEF7E3FBFEF755FB0020A8
:105BB0000221A8F102092060B9F1020F84BFDFF8C9
:105BC000BC83A6F1020C20D90220BCF1020F19D926
:105BD00001FB060338F9132002F10A0ABAF1140F87
:105BE00006D9D4F800A0002AB8BF5242524422601D
:105BF000B5F900A038F913209245B8BF2A80401C9F
:105C00006045E5D3491C4945DED3DD4800781628B8
:105C100004BF384607F059FA3846BDE8F087002837
:105C200018BF0120D749C870704710B5D54C00285F
:105C300004BFA06010BDDFF850C3D4490B78D4492D
:105C40000A7801465A43520060461AF0B0F9CE482D
:105C5000A06010BD10B54C21CE481AF09EF9BDE8E9
:105C600010404C21CC481AF098B9CA487047002817
:105C700018BF0120C3490871704710B57421C74887
:105C80001AF08BF9BDE810407421C5481AF085B9A7
:105C9000002818BF0120BB494871704710B5B94CA6
:105CA000002804BFE06010BD74220146BD481AF010
:105CB0007EF9BC48E06010BD70B5B24D00210446CD
:105CC000E970297169710CF0D1FEFAF78CFB002C98
:105CD00014BF012000202870BDE87040FFF7EEBB24
:105CE0002DE9F04F89B04FF4E461A7481AF055F957
:105CF0007421AC481AF051F9FDF786F80446FCF718
:105D00006BFE0890FDF7A8F80790FBF7FCFB0690E8
:105D1000FCF764FEFBF746F910F0010F0BD001F021
:105D2000F4FD3C2807D1FFF781F920B10420FFF7EB
:105D30002CF9FFF703FA0020FBF7EAFBFDF7CBF89D
:105D400000252E4606F092FD012853D06846FDF747
:105D50008CFB00285ED0684607F093FC14F0070F18
:105D60001CD08A48DFF820B2DDF8089090F8008057
:105D70008748DA460778FEF75EFA0120FEF7C1FA97
:105D800039464046FEF7AFFA524649465846FEF7B6
:105D9000EFFA0020FEF7B5FAFEF75EFA14F0F00F06
:105DA00020D08148DFF8FCB1022701787F48DA462D
:105DB000DDF8109000780844401C4FEA5008FEF7C8
:105DC0003AFA0120FEF79DFA39464046FEF78BFA73
:105DD000524649465846FEF7CBFA0020FEF791FAA4
:105DE000FEF73AFAFDF789FB6D1C102D03D2FDF783
:105DF00072F8A7E701260520FFF7C7F8FCF7EEFDCC
:105E00000698FBF785FB089848B1079828B1FDF77D
:105E100062F804E001F075FC94E7FDF723F8DEBBBF
:105E2000584F14F0070F1BD05848DFF85CC10178B9
:105E30005748E046007801FB00F210200021002ABC
:105E400088BF03460AD938F9115005EB5005B5FB58
:105E5000F3F52CF81150491C8A42F4D84A48B8602E
:105E600014F0F00F18D050484E4B01784F481C46A4
:105E700000780A184FF010014FF000000AD034F9F2
:105E8000105005EB5105B5FBF1FC23F810C0401C88
:105E90008242F4D84348F86009B03046BDE8F08F3C
:105EA000012070474FF47B3070474FF47B3000681F
:105EB0007047034600209A682C2A88BF2C220021B4
:105EC000B1EB920F28BF704753F821C0491C6044C2
:105ED000B1EB920FF8D37047354A0168914214D163
:105EE0004168B1F5807F10D9836800222C2B88BFD0
:105EF0002C230021B1EB930F09D250F821C0491C8B
:105F00006244B1EB930FF8D30AB10020704701202F
:105F100070474FF47B31264B0A689A425ED191F864
:105F200027300022012B08BF0122052804BF91F869
:105F30002300704713DC012804BF087F7047022844
:105F400004BF91F820007047032804BF91F8210096
:105F50007047042804BF91F82200704751E01428CC
:105F600028D015282CD0162831D0172804BF184661
:105F7000704746E05D8500105E850010D02301105B
:105F8000E585001000850010109900106085001054
:105F90006185001030A000107CA00010F02A0110D4
:105FA000C8A000103CA1001062850010638500109D
:105FB0004353494D002A1CBF91F82400704704E068
:105FC000002A1CBF91F8250070472D207047002A39
:105FD0001CBF91F82600704728207047052812D072
:105FE00007DC01280DD002281CBF032804280AD092
:105FF00007E0142818BF1528E7D01628ECD017287A
:1060000001D0FF207047002070472DE9F047ADF523
:10601000007D00244FF40071684619F0BEFFFF2098
:10602000A04660F307082D20254660F3070560F3BE
:106030000F25282060F317454FF47B37F64E64F3A5
:106040001F654FF481794FF02C0AFF224FF4007145
:10605000684619F0C0FFCDE902A4CDE906480594D1
:106060000A94CDE900690494CDE908453846FDF766
:1060700005FF69463846FDF7A3FF012818BF002039
:106080000DF5007DBDE8F0872DE9F047ADF50C7DFD
:10609000894605461F4690464FF0000A4FF40071AE
:1060A0006846949E19F079FF4FF0000CCDF800C2BD
:1060B0004FF47B34CDF804C2CDF808C2CDF80CC241
:1060C000CDF810C2CDF814C2CDF818C2CDF81CC25C
:1060D000CDF820C2CDF824C2CDF828C2CE49206820
:1060E000884206D0FFF791FF0DF50C7D5046BDE8C4
:1060F000F087D4E901120DF5007AE3688AE80F0011
:1061000004F110010DF5047A0FC98AE80F00D4E9F3
:106110000801A26A8A92CDE9880184988DF82092BC
:106120008DF82182401C8DF822728DF81C528DF85A
:1061300023628490002D14BF8698859800F1010099
:1061400014BF8690859080AB82980021CDF80CC258
:106150002C2894BF02462C220020B0EB920F06D2CE
:1061600053F820C0401C6144B0EB920FF8D3484272
:106170008390FF224FF40071684619F02CFF80AC29
:1061800094E80F008DE80F0084AC94E80F0004AC95
:1061900084E80F00DDE988018A9A4FF47B34CDE969
:1061A00008010A922046FDF769FE69462046FDF780
:1061B00007FF012818BF00200DF50C7DBDE8F08712
:1061C0002DE9F041ADF50C7D0F46804616464FF4A3
:1061D0000071684619F0E1FE002580954FF47B348C
:1061E00081958295839584958595869587958895E3
:1061F00089958A9588492068884218D16068B0F5E9
:10620000807F14D9A06821464FF0000C2C2888BF4D
:106210002C200023B3EB900F11D251F823205B1CEC
:106220009444B3EB900FF8D3BCF1000F07D0FFF705
:10623000ECFE002804BF0DF50C7DBDE8F0810FCC0D
:106240000DF5007C8CE80F000FCC0DF5047C8CE87C
:106250000F00D4E90001A2688A92CDE988018DF887
:1062600024828DF825728DF8266201208DF8270290
:106270008298002180AB83952C2894BF02462C2263
:106280000020B0EB920F06D253F820C0401C6144AE
:10629000B0EB920FF8D348428390FF224FF4007185
:1062A000684619F098FE80AC94E80F008DE80F0066
:1062B00084AC94E80F0004AC84E80F00DDE98801A9
:1062C0008A9A4FF47B34CDE908010A922046FDF703
:1062D000D5FD69462046FDF773FE012818BF002052
:1062E0000DF50C7DBDE8F0812DE9F04F4B4D4FF0E1
:1062F000000885B06C4246461720FFF70AFE4FF4AF
:106300007B32844644491068884217D15068B0F502
:10631000807F13D9936800212C2B88BF2C23002069
:10632000B0EB930F80F0FE8052F82090401C49445F
:10633000B0EB930FF8D3002900F0F480FFF765FE6F
:10634000002804BF05B0BDE8F08F1420FFF7E1FD81
:1063500002901520FFF7DDFD00901620FFF7D9FD14
:1063600040B201901620FFF7D4FD404240B20390A6
:10637000FCF74AFDDFF8A8908246002089F8030068
:1063800089F8040089F805000CF070FBFAF72BF887
:10639000002089F80000FFF791F81AF0F00F05D0FF
:1063A00019F01EFE012808BF48F001081AF0070F77
:1063B0007DD01C481D4A002690F800E01A4803785A
:1063C00099F80200A3EB000984468145C4BFAEEBF7
:1063D0000C01A1F1010B1CDD61468B4516DD01F1BD
:1063E000010A01FB03070AFB030A32F8177032F8AF
:1063F0001AA0A7EB0A073FB2002FB8BF7F423FB2F7
:10640000B742C8BFBEB2491C8B45E8DC401C814581
:10641000E2DC009800280BE04353494DF1D8FFFF20
:10642000008500105E8500105D850010D0230110EE
:1064300018BF864288BF48F002080027E246AEEB4C
:106440000A0000905045C8BFA9F1010B1BDD604652
:10645000834513DD0AFB030132F811E002EB410131
:106460004988AEEB010109B20029B8BF494209B21F
:10647000B942C8BF8FB2401C8345EBDC00980AF1DB
:10648000010A5045E3DC0298002818BF874288BF04
:1064900048F00408E2460098504516DD61468945FB
:1064A0000EDD0AFB031032F91000A84200E016E0EE
:1064B000C8BF0546A042B8BF0446491C8945F0DC68
:1064C00000980AF1010A5045E8DC0198002806DD31
:1064D000854202DC0398844201DA48F00808FF2F65
:1064E00088BFFF27FF2E88BFFF267F2DC8BF7F25CF
:1064F00004DC15F1800FB8BF6FF07F057F2CC8BF9B
:106500007F2404DC14F1800FB8BF6FF07F04E0B289
:106510000090EBB2F2B2F9B24046FFF7B5FD05B01C
:10652000BDE8F08FBCF1000F18BFBCF1010F3FF4C4
:106530000CAF03E7FD49002088627047FB49002249
:106540008A6288707047F94890F902007047F748EE
:1065500000787047F54840787047F4480021C171D1
:10656000417141728172C1727047F04920F07E40E2
:1065700008627047ED48006A7047EC48408A7047EF
:10658000EA48808A7047E948B0F916007047E74842
:10659000B0F918007047E548B0F91A007047E348B1
:1065A000007B7047E148C078002818BF0120704781
:1065B00010B54FF4E461DE4819F0EFFCDB49002030
:1065C000C87010BD2DE9F74F90B00025D94801954E
:1065D00002950395049505950695079508950995E7
:1065E000006817460C46052A08BFB0F964600AD057
:1065F000062F08BFB0F9666005D00A2F0CBF1E2613
:10660000B0F960600FD0B0F96200DFF82883B042C3
:1066100009DA13F0FEFF10F4817F1CBFD8F80000E8
:10662000B0F8626036B2324601A9109819F0DDFC6C
:10663000059800B22080BDF826106182BDF81E10BA
:106640006181BDF82010A181BDF82210E181BDF863
:1066500024102182BDF81810A180BDF81A10E18025
:10666000BDF81C1021810028B8BF25808DF8285066
:10667000B148B24900788DF82A008DF82950097880
:106680008DF82B107142ADF82E10ADF8300080B2AD
:10669000ADF82C60ADF80000DDE90A232146109822
:1066A00000F088FD052F11D0E582A5822583A08802
:1066B000002804BF4FF40040A0806089002804BF78
:1066C00047F6FF70608113B0BDE8F08FFEF776FEED
:1066D000002119F08FFC002800F0F180DDF828C0BF
:1066E000DDE90B0ACCF3072310994FEA1C62ADF8E1
:1066F0000050ADF8345099469A4269D91FFA8AF58C
:106700000CF0FF0603FB056E1FFA8EF80E9531F9AB
:106710001880BDF80060BDF834500FFA80FBD845F2
:10672000C4BF761CB6B24FEA204BD845BCBF6D1C27
:10673000ADB2ADF800600EF101081FFA88F8ADF8AF
:10674000345031F918800FFA80FBD845C4BF761C4D
:10675000B6B24FEA204BD845BCBF6D1CADB2ADF808
:106760000060DDF83880CCF3074B03FB08BEAEF1C8
:1067700002081FFA88F8ADF8345031F918800FFA82
:1067800080FBD845C4BF761CB6B24FEA204BD84533
:10679000BCBF6D1CADB2ADF80060AEF101081FFAD0
:1067A00088F8ADF8345031F918800FFA80FBD845DD
:1067B000C4BF761CB6B24FEA204BD845BCBF6D1C97
:1067C000ADB2ADF800605B1CADF834509A4295D87C
:1067D0000CF0FF03CCF3074E9E456CD91FFA8AF6E6
:1067E00009FB063C1FFA8CF8BDF800C031F918808F
:1067F0000FFA80FBADB2D845C4BF0CF1010C1FFAF3
:106800008CFC4FEA204BD845BCBF6D1CADB2ADF837
:1068100000C009F1010808FB06381FFA88F8ADF836
:10682000345031F918800FFA80FBD845C4BF0CF101
:10683000010C1FFA8CFC4FEA204BD845BCBF6D1CE5
:10684000ADB2ADF800C0A2F1020808FB06381FFA8D
:1068500088F8ADF8345031F918800FFA80FBD8452C
:10686000C4BF0CF1010C1FFA8CFC4FEA204BD84539
:10687000BCBF6D1CADB2ADF800C0A2F1010808FBB1
:106880000636B6B2ADF8345031F916600FFA80F81A
:106890004645C4BF0CF1010C1FFA8CFC4FEA20489E
:1068A0004645BCBF6D1CADB2ADF800C05B1CADF879
:1068B00034509E4592D8E582BDF80000A082DDF8F4
:1068C00030900A9E109D4FF0000C052F01D0062F2E
:1068D00047D0184801270068B0F860200020B4F9BC
:1068E0000230B4F900108B4242D1914240DDC6F330
:1068F00007210144C0EB166A8A452FD9C6F3074227
:10690000F0B2D21B3844A2F10108804523D91FFA06
:1069100089F201FB020292B235F9123005EB420214
:10692000B2F90220B3EB020B0AE000001885001058
:10693000B0A10010C88600105D8500105E850010B3
:1069400048BFA2EB030B0FFA8BF26245C8BF944617
:10695000401C8045DBD8491C8A45CFD8A4F818C014
:10696000A5E6F94802270068B0F866203846B6E781
:1069700021839CE6084318BF7047F448016A11F070
:10698000807F08BF7047F0490968C96D11F4003F66
:1069900008BF704700211170182101827047EB4831
:1069A000006B70472DE9FF5FE9480027DDF83CA048
:1069B00005780E98119E8B46B9463C4650452CD022
:1069C00006FB050E10983BF91EC006FB05093BF9B6
:1069D0001900BCEB000148BFA0EB0C0106FB05A8A9
:1069E0003BF91840B4EB000C48BFA0EB040C01EBE2
:1069F0000C0004B232F91EC032F91900BCEB0001E0
:106A000048BFA0EB0C0132F918C0BCEB000248BF34
:106A1000A0EB0C0288180FFA80F9CC48006B012813
:106A200018BF012B37D04FF0010819F0E8FAC94917
:106A3000002C0A7807DD109906FB05113BF91110AF
:106A40001431282909D80099B1F914103C2904DC23
:106A50000099B1F916103C2926DD0E9902EB0A0CBB
:106A600011448C4520D9129B139D13442A448B4218
:106A70001CBF8D1A15F1020F30F9115000EB4106C1
:106A8000B6F90260A5EB060508D01E353C2D08D9E5
:106A90004FF0000808E0A1450CDD0AE00A35142D8E
:106AA000F6D8491C8C45E2D8A14503DDB8F1000FAA
:106AB00000D0012704B03846BDE8F09F7047A348D6
:106AC000B0F90E007047A1490020C881704700212D
:106AD000018041804FF400428280C1800181521EBA
:106AE00042818181C181018241828182C18201838F
:106AF00070479648C06A7047002818BF0120934924
:106B0000C86270479148002181628021817070477E
:106B10002DE9F0418D4D04460027286B6FF07F066C
:106B200084420AD044EA012200236B2107200AF0A4
:106B300001FF002C04BFAF62AE70286B204304BF7E
:106B4000AF62AE702C63BDE8F0812DE9F0478A4654
:106B50008146002513F045FD044613F03EFD04FB7D
:106B600000F17A4E0AB22044002496F90210336BE9
:106B700027466FF07F084BB1B6F91A10643A91427C
:106B80001EDD0124BAF1000F16D107E011F1800FCC
:106B900018BF0029A8BF0225EEDB3BE0002100283A
:106BA0000AD939F91120B2F5487F01DA002407E04B
:106BB000491C8142F5D31CB1306B01282AD106E073
:106BC00011F028F901280CBF01240125F4E70CB3CA
:106BD000B06A4EF6C42188420BD200F041FD00217C
:106BE000022810D0042808BF4FF4FA71B06A084494
:106BF000B0624EF6602181420DD20325B7620024B7
:106C000086F8028007E00BF02EFF002814BF112148
:106C10000821EBE7B762306B84420BD044EA0522CF
:106C200000236B2107200AF085FE002C04BFB76209
:106C300086F80280306B204304BFB76286F802807A
:106C40003463BDE8F087002818BF01203F4948633E
:106C500070473E48406B70473C49888370473B48CB
:106C6000808B704710B507F059F841F2883188429F
:106C700094BF0120002010BD3448406A704733495A
:106C80004862F9F7D0BB3149886370472DE9F04F6E
:106C9000314987B002240A782D49A2F1020C521E14
:106CA00091F8008000210091A8F10101CDE9011CBB
:106CB00000212546A8F102090B46BCF1020F84BF52
:106CC000A9F1010CCDF80CC069D94FF0000CCDF83A
:106CD00014C0CDF810C0AC464D455BD2039F04FBF9
:106CE00008C6BC450FD230F9167000EB4606B6F95F
:106CF0000260B7EB060E48BFA6EB070EBEF1320FDF
:106D000001D9E34608E00CF1010CE145E6D8DDF8D5
:106D100014C0BCF1000F25D0A9F1010CAC4521D362
:106D200004FB08C6654519D230F9167000EB46061B
:106D300036F9026CB7EB060E48BFA6EB070EBEF1A4
:106D4000320F0BD9E24612E0C886001018850010F9
:106D50005D850010638500105E850010ACF1010CAC
:106D6000AC45DDD2DDF810C0BCF1000F12D04FF001
:106D7000010CCDF800C0DDF804C0DC4588BFCDF8BB
:106D800004B0514538BF5146A24288BF2246A342B3
:106D900038BF2346641CDDF808C0644595D3FA4823
:106DA000DDF800C0846B644518BFC0F838C0019896
:106DB00007B0BDE8F04F14F065BB2DE9FF4F8BB075
:106DC000F14DDDE918A704460020287068700BF02B
:106DD0005EFE002840F03A8100F03CFC052871D0AE
:106DE000287B0190EA49E948DDF8309091F800B03D
:106DF0000068E84990F8726009780091B0F97080F5
:106E0000B5F918003228688A05DA002804BF700630
:106E1000060E04D100E010B9287901282BD10BF01F
:106E200075FE40BB012F26D0BAF1010F02D1A88A0E
:106E3000C82820D8A88A002804BF688A00281AD049
:106E40000BF011FE012819D0B9F80000E881009973
:106E500000201BEB01030AD039F91010B5F90E2000
:106E60009142C8BFE981401C80B28342F4D8B5F991
:106E70000E0040450EDD0020A87223E0C3480068E4
:106E800090F873600198012814BF4FF03C084FF050
:106E90004108D9E7286A10F4803F13D0BB48006846
:106EA000C06D10F4803F0DD0A87A401CC0B2A8720B
:106EB000B04207D9102028820120287200204FF00C
:106EC000FF34A87210F0A6FFA8B100F0C9FB042897
:106ED00011D195F8200010F0800F0CD0AB4800685D
:106EE00090F85C0010F0800F05D007202882012068
:106EF0004FF0FF3428720BF0B6FD012871D1A34882
:106F0000BAF1000F00680A9090F874106BDC012F42
:106F100069D0286A10F4003F12D00A98C06D10F4AE
:106F2000003F0DD0687A401CC0B26872884207D911
:106F3000112028820120287200204FF0FF3468724F
:106F40000C98009092484FF0000B012F00780390AE
:106F50009048007801900A9890F87300069045D008
:106F60000198400807900398400809900020049079
:106F700082460590DDE9001001EB400002900023FD
:106F80001A461946BAF1000F0CBFDDE90076DDE9BB
:106F900002760020002E88BFA6F1010E29D937F90C
:106FA0001080B8F1640FD8BF002214DD70450DD2F7
:106FB00007EB400CBCF902C0B8EB0C0948BFACEBC6
:106FC00008090FFA89FCDC45A8BFE346491C002AE2
:106FD00004BF01225B1C401C8642E0D8012B05D86F
:106FE00007E033E0FFE700206872A9E70020E872BD
:106FF0002CE0BAF1000F0CBF049105910AF1010ACF
:10700000BAF1020FBBD3079904988842EED90999C7
:1070100005988842EAD9BBF1320FE7DCE87A401CD8
:10702000C0B2E872296A11F4801F0FD00A99C96DA5
:1070300011F4801F1CBF0699884207D914202882AA
:107040000120287200204FF0FF34E87213F0E1FABB
:1070500010F4807F28D000F0FDFA022824D14FF0F0
:10706000010818F0D1FF074613F0BBFA064613F0EB
:10707000B4FA024600210020002E08D900FB0213BA
:1070800037F913300F2B0FDB401CB042F6D3B8F1A9
:10709000000F09D0491C0129EDD9B8F1000F03D028
:1070A00001204FF0FF3428720EF0E5FF032823D1B2
:1070B000002000900190287C8DF80000BDF80000B1
:1070C000022264F30F20ADF80000E979BDF8020058
:1070D00061F30300697961F30710297A61F30820ED
:1070E000A97961F34920ADF80200E889ADF8040000
:1070F000062168460EF0C2FFB4F1FF3F26D0002CF7
:1071000007BFA87901280FB0BDE8F08FFEF7F4FCA7
:107110000024AC71012028704FF4E4611E4818F07F
:107120003CFFEC7000F09CFA04280D9836D0002843
:1071300018BFFEF771F90E98002804BF0FB0BDE824
:10714000F08F0FB0BDE8F04FFEF717B9287A01288D
:107150001CBF0FB0BDE8F08F0D98FEF7D6FC0024E1
:107160002C72012068704FF4E4610B4818F015FF91
:10717000EC700D98002818BFFEF74EF90E98002805
:10718000DFD10FB0BDE8F08F18850010C886001061
:107190006285001063850010B0A10010002818BFA0
:1071A000FEF70EF90E980028EBD00FB0BDE8F04FB7
:1071B00018F02FBF2DE9F8070023DDF820C0C2F337
:1071C0000724ADF80030160E2546D3B21FFA8CFC0A
:1071D000C2F30747A64259D904FB0C381FFA88F2BC
:1071E00030F9129000EB4202B2F902A0B9EB0A02A8
:1071F00048BFAAEB090212B2BDF900909145B8BF91
:10720000ADF8002008F1010292B230F9129000EBC3
:107210004202B2F90280B9EB080248BFA8EB0902AA
:1072200012B2BDF900809045B8BFADF8002004FB54
:107230000C78A8F1030292B230F9129000EB4202EE
:10724000B2F902A0B9EB0A0248BFAAEB090212B2D6
:10725000BDF900909145B8BFADF80020A8F1020239
:1072600092B230F9128000EB4202B2F90290B8EB10
:10727000090248BFA9EB080212B2BDF9008090458F
:10728000B8BFADF80020641CA642A5D8A7F101083C
:10729000984559D96F1CB41E761E05FB0C3292B26C
:1072A00030F9129000EB4202B2F902A0B9EB0A02E7
:1072B00048BFAAEB090212B2BDF900909145B8BFD0
:1072C000ADF8002007FB0C3292B230F9129000EBBF
:1072D0004202B2F902A0B9EB0A0248BFAAEB0902C6
:1072E00012B2BDF900909145B8BFADF8002004FB83
:1072F0000C3292B230F9129000EB4202B2F902A0C5
:10730000B9EB0A0248BFAAEB090212B2BDF900901C
:107310009145B8BFADF8002006FB0C3292B230F9AF
:10732000129000EB4202B2F902A0B9EB0A0248BF88
:10733000AAEB090212B2BDF900909145B8BFADF8B1
:1073400000205B1C9845A8D8BDF800004880BDE827
:10735000F80770472DE9FF4FDFF8C0B2044689B047
:10736000DBF800001D461646B0F866A012F0A7FD37
:10737000012804BF4FF6FF7000EA4A0A13F049F9EA
:1073800010F4817F07D0B5F9141001232046169A16
:1073900018F044FE04E0012220461699FFF712F986
:1073A0009F4F002425463C71DDF82880FEF706F843
:1073B0000094019402940394049405940694079411
:1073C0000894DBF800006946B0F86020404618F0E9
:1073D0000CFEDBF80010BDF91A00B1F9601049424B
:1073E0008842B8BF0125BDF82000B0F5E17F88BF15
:1073F00001258B48057113F00CF910F4817F0DD134
:107400001698B0F91200002808DC0BF02CFB0128BC
:1074100004D083480079012840F0CA8013F0F9F8BD
:1074200010F4817F00F0BC8047F6FF7003907D4828
:107430004FF00009179C007801907B484D46077873
:1074400013F0E7F810F4817F0EBF5046DBF8000020
:10745000B0F862000FFA80F813F0DBF810F4817FC7
:107460001DBFDBF80000B0F862004042CAF1000026
:1074700000B2029013F0CDF810F4807F19BF4FF0E6
:10748000010B4FF0220C4FF0000BBC460020009087
:107490000398804568DADDE9002000287CD9ACF14A
:1074A000010005900198401E0490ACF10200039089
:1074B0005846E34538BF13B251D202FB070A1FFA00
:1074C0008AF136F911100029B4BFC1F1000E8E46C1
:1074D000C6451ADD41450BDDB4F904E0714502DD16
:1074E000A180E080238109F101010FFA81F90CE00C
:1074F000DDF808E08E4508DDB4F90AE08E4502DDCE
:107500006181A081E381691C0DB20599884223D273
:1075100006EB4A0136F91AE0B1F902A0BEEB0A0106
:1075200048BFAAEB0E0109B2DDF800A052451CBF0E
:10753000DDF810A0524505D058451CBFDDF80CA061
:10754000504504D1B4F902A08A45B8BF6180B4F9AE
:1075500000A08A45B8BF2180401C6045ADD301988A
:10756000521C8242A4D317E0DDE90001002913D99F
:107570005B46E3450CD200FB073189B236F9112096
:1075800002998A42BCBF691C0DB25B1C6345F2D3F1
:107590000199401C8842EBD3A4F81090658204E066
:1075A000062230461799FFF70DF819990120087047
:1075B0001798B0F91000002808DC1798B0F91200ED
:1075C000002803DC16480079012814D113F021F8B3
:1075D00010F4817F07D0052347F6FF71189A0A98A7
:1075E00018F01CFD04E0052218990A98FEF7EAFF3E
:1075F0001A99012008701698418A09484182169903
:10760000098A818216994989C182169989880183DC
:107610001899098A41830DB0BDE8F08FC886001023
:10762000188500105E8500105D85001010B50BF008
:107630002BF80BF00BF9002010BD0000FE49C870BC
:107640007047FD48C0787047FB4908717047FA4899
:1076500000797047F84800787047F748807870479D
:10766000F5480078022805D005281CBF0020704787
:1076700006F04BBB0BF0DAB9EF4908707047EE49E2
:1076800048707047EC484078704770B5EA4E044641
:107690000D463078A04212D002281ED0052814BF13
:1076A000002006F032FB44EA05213278002341EA4B
:1076B000024141EA0062612107200AF03BF930787B
:1076C000844218BF7070B570072C28BF70BDDFE80A
:1076D00004F016070B13160F16000BF0A7F9E2E7DC
:1076E000284600F0C1FA0AE028460BF047FA06E007
:1076F000284606F0FFFA02E028460AF009FA34703C
:1077000070BDCE4900200968B1F89C1011F4807F4B
:1077100008BF7047FCF7CDBAC84900200968B1F826
:107720009C1011F4807F08BF7047FCF7D1BAC349A1
:1077300000200968B1F89C1011F4007F08BF704761
:1077400018F071BCBC49487900281CBF401E487124
:10775000704770B5BA480068B74C10F0130F0FD0DF
:1077600010F0100F05D0B74951F88C2F42F4805219
:107770000A60B54908606079002804BF0120607183
:107780004FF040208069AD4D10F0020F296806D1FE
:10779000AE48006810F0010F01D0607940B1B1F837
:1077A0009C10002011F4807F18BFFCF791FA07E0CD
:1077B000B1F89C10002011F4806F18BF18F038FC4D
:1077C000A349084208BF70BD2968D1F89C10090C74
:1077D000617170BD10B572B6FDF758FDBDE810407F
:1077E000FDF768B910B5012802D0022805D007E0DE
:1077F0004FF47F30FCF742FB02E097499548086060
:1078000072B6FDF743FDBDE81040FDF753B98A4954
:1078100000288A7918BF01208871C0B2824208BF4F
:1078200070470022002818BF0122002301210220F6
:107830000AF080B880488079002818BF012070477E
:1078400070B57D4C0028E57918BF0120E071C0B209
:10785000F8F7A8FDE079854214BF002870BD2078B4
:1078600002281CBF052870BD0221BDE870400CE74E
:107870007148C079002818BF012070476E48007A0F
:1078800070472DE9F0416C4D00281CBF0020287284
:1078900004D1287A002818BFBDE8F0816F4E376800
:1078A0003020FCF76DFC06213020FCF782FCF06AEA
:1078B00040F03000F0626A4C4FF07F0811E0FDF7B5
:1078C000FCFCF06A10F0100F03D0287A40F07E0024
:1078D0002872F06A10F0200F03D0287A40F00100DF
:1078E0002872201EA4F1010403DD287A38EA000082
:1078F000E5D13020FCF78AFC3760BDE8F0814E48C6
:10790000806970474C48406970474B48406900287F
:1079100018BFC07A70474849C86170474648C06977
:1079200070474549086270474348006A70474348BA
:10793000026802F5BE73118A508A02F59E72FBF747
:10794000A3BB10B506F0A7FF002818BFC07A10BD72
:1079500010B506F0A0FF00280CBF4FF0FF3090F9E3
:10796000240010BD2DE9F04FDFF8CCA099B00E46F1
:10797000CAF8180006F08FFFCAF81400002871D06A
:1079800090F800C08AF809C041788AF80A10837814
:1079900004460CF101008AF80B3000F0FE008AF872
:1079A0000C00E2788AF80D2020798AF80E006079C0
:1079B0008AF80F000AF111004FF0000B80F800B0B8
:1079C00080F801B020788AF810006046FBF719FDB6
:1079D0009AF80F109AF80E00FBF736FD694620461C
:1079E00006F077FFE089DAF81C5000281CBF6843D6
:1079F000050BB4F81280DAF82090B8F1000F08BF38
:107A00004FF48058E78A002F08BF4FF480574FF497
:107A100080501890002016F0040F18BF052016F0B3
:107A2000080F18BF40F0020016F0020F18BF40F018
:107A3000F00016F0010F16E054850010C886001003
:107A4000184800400030004014480040144C0040EA
:107A500008001300AD2007B0304C0040001000407B
:107A60008038010048E018BF40F4774016F4807F6A
:107A700018BF40F4803016F4007F18BF40F47E0039
:107A8000E16901EA000600981090059812900798A5
:107A9000CDF844B0CDE9130B01981590A07A17905A
:107AA0000398169010A93046FBF79BF816F0070FC5
:107AB00061D006F0CEFB18B101460020F9F72FFE89
:107AC00006F0DEFB6843050B06F0FAFB09FB00F04D
:107AD000000B4030C1090A20012202FA00F30B42D8
:107AE00001D1401EF9D5A0F10509207B002818BF5F
:107AF000A0F1010B11D10CE059480068B0F89C00CE
:107B000010F4807F18BFFCF7E3F8002019B0BDE83F
:107B1000F08F0020F9F7EFFF8346607B002814BF49
:107B2000401EFAF720F80BEB0901052905DDA9EB4A
:107B3000010101F10509052104E00029BCBFA9EB01
:107B4000010900218144B9F1050F05DDA9F1050006
:107B5000C5404FF0050907E0B9F1000F04DAC9F19B
:107B6000000085404FF000090020F9F7DEFF49468C
:107B70000020FAF712F816F0F00F43D0207C70B115
:107B800016F0100F03D0411E0120F9F7CEFF16F0BA
:107B9000400F04D0207C411E0220F9F7C6FF207D53
:107BA00070B116F0200F03D0411E1120F9F7BDFF70
:107BB00016F0800F04D0207D411E1220F9F7B5FF8A
:107BC000607C70B116F0100F03D0411E0120F9F750
:107BD000E4FF16F0400F04D0607C411E0220F9F74C
:107BE000DCFF607D70B116F0200F03D0411E112024
:107BF000F9F7D3FF16F0800F04D0607D411E1220EC
:107C0000F9F7CBFFE07A00281CBF0001F9F7C0FCB0
:107C1000029806F0FAFA049830B12B469AF80A2036
:107C20009AF8091018F009FA3A4641462846189B76
:107C300018F008FA0698FDF7F8FF0898FEF72EF8F6
:107C40000BF038F819B00120BDE8F08F10B5FBF744
:107C50009EF806F0E2FA034900204861012010BDB9
:107C6000C886001054850010FE4908707047FD4812
:107C700000787047FC4810B4FC4A016891421CD15E
:107C80004168B1F5987F18D8D0F808C00146BCF516
:107C9000007F12D800220B461146B2EB9C0F24BF86
:107CA00010BC704753F82140491C2244B1EB9C0F93
:107CB000F8D3002A04BF10BC7047002010BC7047E6
:107CC000E948FCF7DBB8E7490120087070472DE967
:107CD000F04117460E4605461024FFF713FE15F037
:107CE000070F18BF062403D115F0F00F18BF0824A2
:107CF0003246102C28BFBDE8F081002A08BFBDE83D
:107D0000F08120443B4690F920102046BDE8F04128
:107D100006F007BEF0B5ADF6E43D0446FFF7F2FD10
:107D2000054614F0070F0CD06F4605263846FBF7C2
:107D3000E9FB95F925104FF43E633A46304606F0CC
:107D4000F0FD14F0F00F04BF0DF6E43DF0BD072484
:107D50006E46FBF759F810F0300F0CBF02200120DF
:107D60006946FBF71FFC95F927104FF4187332464C
:107D7000204606F0D6FD0DF6E43DF0BD2DE9F34FAB
:107D800089B00020069008780390486804908868BD
:107D900005900D7B487B0190887B8A8AD1E9088B0E
:107DA000C0F5807602EA00070998B1F91090B1F9A0
:107DB00012A0896910F0010F07914FF0000044D024
:107DC00000900198002840F2D7800098012101FA24
:107DD00000F20798104018BF0120002402906109AA
:107DE00004A804F01F0250F8211001209040014225
:107DF00000F0B7803BF9020B0299A0EB0A000029C2
:107E00000CBFA9EB000509EB000538F9020BA0EB4C
:107E10000A0014BF4844A9EB0000002DB4BF69421A
:107E200029460028B8BF4042884278D922460099A6
:107E30000398FAF753FC0246C0F30420D1B212F4BF
:107E4000803F6FD0002D6FDB70E0F9F7B0FF00903E
:107E500001980321684301EB400020F003024146F2
:107E6000584618F0A4F80098F9F7A1FF01984FF0D0
:107E7000000B002852D90121079801FA0BF210409B
:107E800018BF012000250290690904A805F01F020F
:107E900050F8211001209040014237D038F9020BF0
:107EA0000299A0EB0A0000290CBFA9EB000409EB22
:107EB00000042A4659460398FAF710FCC0F304213F
:107EC000C2B210F4803F02D0002C02DB03E0002C91
:107ED00001DD941B00E09419BC4205DD1F293ABF67
:107EE0000024491C3C4606E0002C04DA0029C6BFE9
:107EF0003C46491E002400F4783040EA012040EA64
:107F000004032A4659460398FAF73BFC6D1C262DBC
:107F1000BAD301980BF1010B8345ACD32CE020E0E0
:107F200000E001E0002D01DD8D1900E08D1BBD4258
:107F300005DD1F283ABF0025401C3D4606E0002D08
:107F400004DA0028C6BF3D46401E002502F4783101
:107F500041EA002040EA0503224600990398FAF717
:107F600010FC641C262CFFF43AAF00980199401CC9
:107F700000908842FFF429AF0998032826BF01200A
:107F8000069006980BB0BDE8F08F2DE9F04F8BB04E
:107F9000002205920A7800924A6802928A68039247
:107FA0004D7B8A7B0492B1F91080B1F912200792BF
:107FB0000C6A8A690892898A049AC0F1080A01EA5F
:107FC000020600283BD0BAF1000F7DDB4FF0000B1A
:107FD000002D7AD9012000FA0AF00690AAF10100DA
:107FE000012101FA00F009900121089801FA0BF231
:107FF000104018BF012000270190790902A807F05E
:108000001F0250F821100120904001427DD034F928
:10801000021B0798081A019900290CBFA8EB000958
:1080200008EB00093A4659460098FAF757FB034611
:1080300010F4803F7BD0B9F1000F7DDA7AE04FF089
:10804000000B002D41D90121089801FA0BF21040D4
:1080500018BF012000270190790902A850F82110CB
:1080600006E000007885001000EE030054435246FD
:1080700007F01F0201209040014250D034F9021B4A
:108080000798081A019900290CBFA8EB000908EB12
:1080900000093A4659460098FAF720FBFE4901408C
:1080A00011F4803F18D0B9F1000F2ADA11F4F85119
:1080B0001CBFA1F5807141F4803122D110F4604FD2
:1080C0001FD04FF4D05101E050E048E0A0F500503F
:1080D00010F4003F15D012E0B9F1000F11DD11F4DA
:1080E000F85118BFA1F580710BD110F4604F08D082
:1080F000A0F500504FF4D05110F4003F01D04FF4E0
:108100008D3100F43830084302E01FE00FE013E047
:1081100040F080033A4659460098FAF732FB7F1C3C
:10812000262F99D30BF1010BAB458CD317E0B9F196
:10813000000F01DD06988343BAF1000FC4BF099810
:1081400003433A4659460098FAF71BFB7F1C262F3B
:10815000FFF453AF0BF1010BAB45FFF445AFBAF1A0
:10816000000FC2BF05980BB0BDE8F08F0027002DAF
:108170002ED904980DF1080A4FF0010BC0F5807953
:1081800040F480780024600904F01F015AF82000B0
:108190000BFA01F1084215D0224639460098FAF749
:1081A0009DFAC1B201EB590101EA0801B14288BF51
:1081B000314620F0FF0040EA01032246394600988C
:1081C000FAF7DFFA641C262CDDD37F1CAF42D9D32B
:1081D000012005900BB0BDE8F08F2DE9F04F89B07C
:1081E000002204920A7800924A6802928A680392F6
:1081F0004A7B0192B1F91060B1F912B00C6A896939
:10820000C0F105080591002837D0B8F1000F70DBE8
:108210004FF00009002A6BD908F10800012101FA8A
:1082200000FA401E01FA00F006900121059801FABB
:1082300009F2104018BF012000250790690902A823
:1082400005F01F0250F821100120904001425FD03C
:1082500034F9020B0799A0EB0B0000290CBF371A69
:1082600037182A4649460098FAF738FA034610F4B8
:10827000803F3FD0002F41DA3EE00027002A4FD94F
:108280000120059900FA07F20A4214BF4FF0010AD3
:108290004FF0000A0025690902A805F01F0250F8F6
:1082A00021100120904001421BD034F9020BBAF199
:1082B000000FA0EB0B000CBFA6EB000906EB0009BA
:1082C0002A4639460098FAF709FAB9F1000FC8BFF3
:1082D00040F4803040F480532A4639460098FAF73B
:1082E00050FA6D1C262DD6D301987F1C8742C7D328
:1082F00016E01AE0002F01DD23EA0A03B8F1000FAF
:10830000C4BF069803432A4649460098FAF739FA4B
:108310006D1C262D92D3019809F10109814584D362
:10832000B8F1000F04BF01200490049809B0BDE823
:10833000F08F2DE9F04F89B0002204920A78009264
:108340004A6802928A6803924A7B0192B1F91060EE
:10835000B1F912B00C6A896905915049C968421A8D
:10836000C2F10308814277D83DD101984FF0000750
:10837000002871D90120059900FA07F20A4214BFBA
:108380004FF0010A4FF0000A0025690902A805F024
:108390001F0250F821100120904001421BD034F9F7
:1083A000020BBAF1000FA0EB0B000CBFA6EB00090B
:1083B00006EB00092A4639460098FAF78FF9B9F119
:1083C000000FC8BF40F4003040F400432A4639464D
:1083D0000098FAF7D6F96D1C262DD6D301987F1C8C
:1083E0008742C7D34FE0B8F1000F51DB01984FF03F
:1083F0000009002847D908F10D00012101FA00FA0F
:10840000401E01FA00F006900121059801FA09F2D8
:10841000104018BF012000250790690902A805F047
:108420001F0250F8211001209040014223D034F95E
:10843000020B0799A0EB0B0000290CBF371A371865
:108440002A4649460098FAF749F9034610F4003FD6
:1084500003D0002F05DA02E015E0002F01DD23EA4A
:108460000A03B8F1000FC4BF069803432A464946E1
:108470000098FAF786F96D1C262DCED3019809F1E4
:1084800001098145C0D3B8F1000F04BF0120049059
:10849000049809B0BDE8F08F001F01007885001036
:1084A0002DE9F14FADF54E7D0020C090BF9072B622
:1084B000FAF7AAFC0746FCF7A7FB48B1FCF74CFC0F
:1084C000C090FCF733FCFCF74CFCBF90FCF739FC88
:1084D000FAF77BFBFAF780FAC590FAF7BDFCC49077
:1084E000FAF77CFAFAF742FDBC900020FAF735FD66
:1084F0000120F9F7F8FBC8901120F9F7F4FBC990B7
:108500000220F9F7F0FBCA901220F9F7ECFBCB90B0
:10851000FCF7C3F9C390FCF7A8F94FF49350FCF7AC
:1085200016F962B60020F9F7AFFBC29001210020D6
:10853000F9F79DFB0020F9F7BCFB0021C19008462C
:10854000F9F7AAFB0120F9F732FCCC900020FAF7EA
:108550008EFAC7900020FAF77DFAC690F8F7D3FF9D
:10856000CD900020F8F7D4FF002006469EAD45F8D8
:108570002060401C0C28FAD317F0070F4FF00104BD
:108580000AD040F68C61FE489E9417F006FD40F636
:108590008C61FC4817F001FD17F0F00F47D0012067
:1085A000F8F7A7FA38B19821F74817F0F6FC9821A8
:1085B000F64817F0F2FC1120F8F79BFA38B1982131
:1085C000F34817F0EAFC9821F24817F0E6FC022085
:1085D000F8F78FFA38B19821EF4817F0DEFC9821B0
:1085E000EE4817F0DAFC1220F8F783FA38B1982138
:1085F000EB4817F0D2FC9821EA4817F0CEFC012096
:10860000F8F777FA002818BFA0941120F8F771FA4C
:10861000002818BFA1940220F8F76BFA002818BFB1
:10862000A2941220F8F765FA002818BFA3944FF01F
:10863000405ADFF874B3DFF874939E984FF0FF0848
:1086400058B330468DF8006001A9F9F7B1F99DF8EB
:108650000000F9F7CDF98DF80C009DF80000F8F74F
:1086600017FA8DF80D009DF80000F9F786FB002839
:108670000CBF4FF0FF31002106918DF80E80B9F844
:108680000200ADF81000ADF812609DF80000F9F797
:108690002FF9ADF81400CDE908AB9F986F4640B3B1
:1086A0008DF8286007F12C013046F9F781F99DF823
:1086B0002800F9F79DF98DF834008DF835401096B3
:1086C0008DF83680B9F80200ADF83800ADF83A60A0
:1086D0009DF82800F9F70CF9ADF83C009DF80C0066
:1086E0009DF80D1048430AEB40010BEB4000CDE92B
:1086F0001210A0984FF4806A02264FF0AA3BE0B314
:108700008DF8504007F154012046F9F751F99DF8D2
:108710005000F9F76DF98DF85C009DF85000F9F7FD
:10872000EAF904FA00F08DF85D009DF85000F9F7C1
:10873000DAFA1A908DF85E80B9F80400ADF860009E
:10874000ADF862A09DF85000F9F7D2F8ADF86400DA
:1087500097481C9097481D909DF85D00022809D904
:108760009DF85C10801E48431C9901EB40001C9052
:108770008DF85D601A9800B100E007E09DF85000A8
:108780004FF0AA31F9F79DFACDF868B0A198E0B39F
:10879000112007F17C018DF87800F9F709F99DF8AF
:1087A0007800F9F725F98DF884009DF87800F9F73D
:1087B000A2F904FA00F08DF885009DF87800F9F729
:1087C00092FA24908DF88680B9F80400ADF88800FC
:1087D000ADF88AA09DF87800F9F78AF8ADF88C001A
:1087E00075482690754827909DF88500022809D97C
:1087F0009DF88410801E4843269901EB4000269086
:108800008DF88560249800B100E007E09DF87800BD
:108810004FF0AA31F9F755FACDF890B0A298E0B32D
:1088200007F1A40130468DF8A060F9F7C1F89DF872
:10883000A000F9F7DDF88DF8AC009DF8A000F9F77D
:108840005AF904FA00F08DF8AD009DF8A000F9F790
:108850004AFA2E908DF8AE80B9F80400ADF8B00059
:10886000ADF8B2A09DF8A000F9F742F8ADF8B40059
:1088700053483090534831909DF8AD00022809D9F3
:108880009DF8AC10801E4843309901EB40003090B9
:108890008DF8AD602E9800B100E007E09DF8A000D3
:1088A0004FF0AA31F9F70DFACDF8B8B0A398E0B3BC
:1088B000122007F1CC018DF8C800F9F779F89DF87E
:1088C000C800F9F795F88DF8D4009DF8C800F9F7BD
:1088D00012F904FA00F08DF8D5009DF8C800F9F7F8
:1088E00002FA38908DF8D680B9F80400ADF8D800B7
:1088F000ADF8DAA09DF8C800F8F7FAFFADF8DC0093
:1089000031483A9031483B909DF8D500022809D96A
:108910009DF8D410801E48433A9901EB40003A90EC
:108920008DF8D560389800B100E007E09DF8C800E8
:108930004FF0AA31F9F7C5F9CDF8E0B0F8F732FBFE
:1089400010F0010F0BD0FEF7E0FF3C2807D1FCF739
:108950006DFB20B10420FCF718FBFCF7EFFBFAF7E6
:10896000BAFA4FF00008C346C2464646C14603F075
:108970007DFF01287DD0BBF1800F7AD8AAA827E01F
:1089800000000130004001308C0E01308C4E01306F
:10899000240F0130244F0130BC0F0130BC4F013097
:1089A00054100130545001300040003078850010E0
:1089B000CC090030CC490030CC0E0030CC4E003019
:1089C0004C1800304C5800304C1D00304C5D0030CD
:1089D000FAF74BFD00286ED0AAA804F052FEBC980E
:1089E000002818BF00273BD09EA850F82700A0B34E
:1089F00007EB8701684600EBC104207810F00F0FE9
:108A00002BD0F9F770F910F0010F26D0216A257BE1
:108A100001F0030000EB8502D21C22F0030221F0DA
:108A20000301CDE9BD1278A90C1878A8BD9917F0FB
:108A3000BEFA0020002D0BD9411934F8102034F86B
:108A4000113024F81030401C24F811208542F3D84E
:108A500078A9BE9ABD9817F0AAFA7F1C0C2FC3D331
:108A60001AF1010A7DD04FF0000A5046B0AD01273F
:108A700000E077E00BF1010B45F82070401C0C285A
:108A8000FAD3052E6ED2DFE806F003172A3D500018
:108A900000249EA850F8240048B104EB84016846E5
:108AA00000EBC1014846FFF744FC45F82400641C74
:108AB0000C2CEED33BE068E000249EA850F8240084
:108AC00048B104EB8401684600EBC1014846FFF75A
:108AD00084FB45F82400641C0C2CEED327E0002412
:108AE0009EA850F8240048B104EB8401684600EBCE
:108AF000C1014846FFF749FA45F82400641C0C2CD4
:108B0000EED314E000249EA850F8240048B104EBF2
:108B10008401684600EBC1014846FFF72FF945F88C
:108B20002400641C0C2CEED301E04FF0010801215D
:108B3000002055F82020CAB1401C0C28F9D3A9B157
:108B40001F2E0DD2761CCE9807FA06F1014207D1EE
:108B5000761C042E04D8CE9807FA06F10142F7D00D
:108B600001E005E017E04FF0000901E009F101091B
:108B7000FAF7C3FCB8F1000F0DD1BC98002818BF5C
:108B8000F9F7C3F8FAF7A7F9F1E6FEF7C5FDB8F172
:108B9000000F3FF4ECAEFAF7B0FCF9F71FFF052029
:108BA000FCF7F3F90120C899F9F78BF81120C9995E
:108BB000F9F787F80220CA99F9F783F81220CB99C0
:108BC000F9F77FF8BC98FAF7C8F90020C199F9F7CE
:108BD00063F80020C299F9F74AF8CC98F9F7E7F85A
:108BE000C798F9F744FFC698F9F734FFCD98F8F71E
:108BF0008FFCC59830B1C49810B1FAF76CF901E058
:108C0000FAF730F9FCF700F848B1C098002818BF0F
:108C1000FCF700F8BF98002818BFFCF734F8C39899
:108C2000002818BFFBF7CAFDB8F1000F0CBF0120E8
:108C300000200DF54F7DBDE8F08F70B5FD4D164657
:108C4000D5F844231205120D1DD000281CBFC1F316
:108C50000800FAF7D3FFD5F8480340F00100C5F843
:108C60004803D5F8480320F00100C5F84803002266
:108C7000341E23DDD5F8481340F21F2011F0010FF8
:108C800008D1401E01D2002070BDD5F8481311F064
:108C9000010FF6D0D5F84403C0F30B000244D5F819
:108CA000480340F00100C5F84803D5F8480320F018
:108CB0000100C5F84803641E002CDBDC1001B0FB8A
:108CC000F6F080B270BD2DE9F84F040016D0DA48F6
:108CD000006CC0F30829FAF7A3FF49EA0042002319
:108CE0007621072008F026FED248D0F8401341F440
:108CF0008031C0F84013322000900AE0FAF78BFF71
:108D00000120BDE8F88F00BF00BF00BF00BF00BF5B
:108D10000846411E0091F6D24FF0000840F2FF17BE
:108D2000C246464608EB070000EBD0704510A9B2DA
:108D300064220120FFF781FFF0B1A04288BF6F1EBF
:108D400038BF05F101081ED1AA461FFA8AF14FF07B
:108D500064024FF00100FFF770FF04460023524603
:108D60007721072008F0E6FDA4F58050AF38A02851
:108D70009CBF0120BDE8F88FB9F1000F10D0484624
:108D8000FAF73CFF0EE0011B48BF211A321B48BF17
:108D9000A21B9142BCBFAA460646B845C2DDD4E735
:108DA000FAF739FF49F4803200237721072008F0D1
:108DB000C1FD0020BDE8F88F2DE9F04F9F4CADF6C6
:108DC000244D01262778FEF745FC012840F0AF81AD
:108DD00004F067FE9A480068B0F91E10B0F91C0054
:108DE00017F035F917F0020F00F0988101ADFEF78A
:108DF00041FF4FF00009A8B1B0E80E1001AC84E8C3
:108E00000E10B0E80E1005AC84E80E10B0E80E109D
:108E100009AC84E80E1070E80C12806B0D91CDE95E
:108E20000E2022E0FF223C21284617F0D4F8854886
:108E300001904FF4987002903C20CDE90309502036
:108E4000CDE905094FF0FF30CDE908900A90ADF863
:108E50003C900C908DF83E900B90CDF81C90CDF886
:108E60003490CDF838908DF83F907748FBF706F8AE
:108E70000698401C0690F9F7A8FE41F2FF00FFF7A4
:108E800022FF6E498860F9F768FF40F23338002509
:108E9000CDF800909AE0284605F0FDFC00287DD032
:108EA000008900EA080434F0CC0077D040F20F319A
:108EB0002846FEF757FD002870D0F9F7A5FF009966
:108EC00000296CD1F9F757FE1F20FFF7E9FA00904F
:108ED000F9F784FD0098002875D1A6B314F0010FAE
:108EE00013D0FEF70FFD824605200DF1400BCDF8A3
:108EF000200C5846FAF706FB9AF925104FF43E630A
:108F00005A46DDF8200C05F00CFD14F0100F18D0B7
:108F1000FEF7F8FC824607200DF1400BA890F9F708
:108F200073FF10F0300F0CBF0220012010A9FAF7D8
:108F300039FB9AF927104FF418735A46A89805F090
:108F4000F0FC009858BB14F0220F06D0FCF7C8FEC6
:108F50000090F9F743FD009808BB06B314F0020F28
:108F600016D0FCF791FA83463848017838480078E3
:108F700048434FEA400AFEF7C5FC4FF0060C5FEA93
:108F80000B0205D090F926105346604605F0C9FC47
:108F900014F0200F17D0FCF70EFA01E015E012E0F4
:108FA00004462C4801782C48007808444FEA400ACF
:108FB000FEF7A8FC01460820220004D091F92810F1
:108FC000534605F0AEFCFEF741FE6D1C05F05FFC5C
:108FD000A842009803D900283FF45DAF03E00028C1
:108FE00008BF012000D0002018B1FCF759FF01286C
:108FF00034D008980023401C0890502005901A4651
:109000002121072008F096FC00231A461946FE206D
:10901000CDF80090FDF738F801AC05F010FC90B3E6
:1090200081690991C1690A9141690B91C0680C90ED
:109030003DE00000005000400060004078850010D6
:10904000C88600105443524600EE030060850010AD
:1090500061850010628500106385001017F0080F0D
:1090600014BFA220A120B3490590886860B1B2481E
:10907000006CC0F30820ADF83C009DF83E00401C99
:109080008DF83E0007E00CE0ADF83C909DF83F0005
:10909000401C8DF83F00C1F808900798401C0790CD
:1090A000BAE74FF0FF300C900B900A900990A3485C
:1090B00001904FF4987002903C20CDE90309002103
:1090C000A3682246084652F820C0401C6144B0EB19
:1090D000930FF8D34D42FF224FF4007110A8E560C2
:1090E00016F079FFA268F4E8040110AB83E82700CA
:1090F0000FCC14AD85E80F000FCC18AD85E80F003C
:10910000D4E90001A2688E4CCDE91C011E922046D4
:10911000FAF7B4FE10A92046FAF752FF0020FCF738
:10912000CCFC00233A464021072008F003FC0DF652
:10913000244DBDE8F04F03F0E5BA7E4A022804BF93
:1091400091807047042808BF518070470146002075
:109150000229784A04BFB2F904007047042908BF05
:10916000B2F90200704770B50126FEF783FD20B109
:109170000069A12818BFA22801D0002070BD0024DA
:1091800005F085FB002834D9204605F084FB002833
:109190001EBF058925F0CC0030F47C4024D040F27D
:1091A0000F312046FEF7DEFBF0B115F0010F0AD0BB
:1091B000FAF7BDF938B944F4807200232021072062
:1091C00008F0B8FB002615F0100F0BD00120FAF7BD
:1091D00005FA38B944F4805200232021072008F012
:1091E000A9FB0026FEF732FD641C05F050FBA042EF
:1091F000CAD8304670BD00207047002070474D48E7
:10920000407870474B4900204870704770B5002186
:1092100005220846FFF711FD0023464A00282BD0FF
:109220005178002908BF1361A0F5805CACF1F80CFF
:10923000BCF10E0F20D9491CC9B25170D2F810C030
:109240000A296044106121D93B495370096CC1F36C
:1092500008249CB14BF6F521884294BF651C651E1D
:109260002846FAF7CBFC44EA054200237521072083
:1092700008F060FB012070BD537007E041F2FF0071
:10928000FFF721FD00281CBF012070BD002070BD2C
:1092900010B5FEF7EFFC38B3284A0168914223D19C
:1092A0004168B1F5987F1FD8D0F808C00146BCF5D9
:1092B000007F19D800220B461146B2EB9C0F07D253
:1092C00053F82140491C2244B1EB9C0FF8D35AB902
:1092D000188F00281CBFA0F57F41B1F1FF0103D01A
:1092E000FAF78CFC012010BD002010BD10B5FEF770
:1092F000C1FCD8B1114A0168914217D14168B1F55A
:10930000987F13D8D0F808C00146BCF5007F0DD86F
:1093100000220B461146B2EB9C0F09D253F82140B4
:10932000491C2244B1EB9C0FF8D30AB1002010BDB8
:10933000188F10BD788500100060004054435246DD
:1093400000EE030070470020704710B503F00700DF
:10935000042808BFFEF73EFA002010BD10B403F049
:1093600007020024FE4BDFF8FCC3012A02D0022AC8
:1093700017D013E005208CF80000FB48CCF80C4017
:1093800000681A68532111701A68452151701A68D3
:10939000010A91701968C8701868047110BC002027
:1093A00070479CF80020052A14D1DCF80C20052A0F
:1093B00028BF104605D21B689B5C0370501CCCF87C
:1093C0000C00052806D10120CCF80C4008700320C1
:1093D0008CF8000010BC0120704770B503F0070244
:1093E0000125DF4CDF4B4FF0000C012A02D0022A8E
:1093F00025D022E005201870DB48C3F80CC00068B7
:109400002268AC2111702268010A517021688870AD
:109410002068C570206880F804C005F0B1F948B133
:10942000D24D286805F0B4FA20B128682168007E82
:10943000487102E02168FF204871002070BD1A7851
:10944000052A10D1DA68062A28BF104604D22468FB
:10945000A45C0470501CD860062804D1C3F80CC06A
:109460000D7003201870012070BD03F00702022A5E
:109470001CBF002070472022027001200870704736
:109480002DE9F041B74F0D46064613F0070F04D003
:1094900003F00700022808D004E012F0040F1CBFFC
:1094A0000020B8700020BDE8F08103F025F9002805
:1094B00014BF0124002403F022F9002814BF022263
:1094C000002242EA0403B878002814BF04220022D4
:1094D00042EA0300307001202870BDE8F08170B5C9
:1094E00003F0070C00269F4C9D4DBCF1010F0AD0E4
:1094F000204613F0070F00780DD0BCF1040F08BF11
:10950000062818D029E0E6602868067028684670AA
:109510000520207021E005281FD1E068022803D231
:109520002B681A54401CE060022816D10120E66026
:109530000870062010E02868007855280BD12868AC
:109540004078AC2818BFBC2805D128680122411CEE
:10955000062003F0B7F803202070002070BD70B51E
:1095600003F0070200257E4C7E4B012A02D0022A1E
:1095700024D021E005201870DD6003F071F841F679
:10958000E8710144B0F5783F10D8CA78086862F3F2
:109590001F60774A904208BF002007D10A1823684D
:1095A00012791A54401C1428F8D305E000202168D1
:1095B0000D54401C1428FAD3002070BD1A78052AD7
:1095C00013D1DA68142A28BF104607D2D4F800C095
:1095D0001CF802C080F800C0501CD860142804D1C8
:1095E0000120DD60087003201870012070BD70B587
:1095F00003F0070200255A4C5A4B012A02D0022AD6
:109600003FD03CE005201870DD6003F029F841F6FA
:10961000E8710144B0F5783F2BD8CA78086862F346
:109620001F60534A904224D12268087C107022683F
:10963000487C50702268887C90702068CA7CC27018
:1096400020680A7A02712268487A50712268887A02
:1096500090712268C87AD0712268087D10722268E1
:10966000487D50722268887D9072C87D2168C872DA
:1096700005E0002021680D54401C0C28FAD300207E
:1096800070BD1A78052A13D1DA680C2A28BF104653
:1096900007D2D4F800C01CF802C080F800C0501CEB
:1096A000D8600C2804D10120DD60087003201870F8
:1096B000012070BD70B503F007020025284C294E2B
:1096C000012A02D0022A36D033E005F0B8F840B3C0
:1096D000D0E906212368C0681A70D4F800C0130AC4
:1096E0008CF80130D4F800C0130C120E8CF8023044
:1096F0002368DA702268117123680A0A5A71236894
:109700000A0C090E9A712268D171216808722268C8
:10971000010A51722268010C9172010E2068C17217
:1097200004E021680D54401C0C28FAD30520307049
:10973000F560002070BD3278052A10D1F2680C2A3D
:1097400028BF104604D223689B5C0370501CF06055
:109750000C2804D10120F56008700320307009E066
:10976000EC55020094850010044C0040C88600109F
:1097700034CD12AB012070BD70B503F00702002498
:10978000F54DF64B012A02D0022A3ED03BE00520DF
:1097900018700026DC6002F063FF00F50051B0F5A0
:1097A000783F98BF11F0030F27D1ED4A0868904227
:1097B00004BF0022104620D151F82030401C1A442A
:1097C0000728F9D302B1C6B128680A7C02702A685A
:1097D000487C50702A68887C90702A68C87CD07059
:1097E0002A68087D10712A68487D50712A68887D32
:1097F0009071C87D2968C87105E0002029680C5463
:10980000401C0828FAD3002070BD1A78052A13D10D
:10981000DA68082A28BF104607D2D5F800C01CF81D
:1098200002C080F800C0501CD860082804D1012074
:10983000DC60087003201870012070BD2DE9F04134
:1098400003F0070C0027C54E4FF00508BCF1010FCF
:109850000DD013F0070F0FD03246BCF1020F127873
:1098600010D0BCF1040F08BF062A26D058E086F8B5
:1098700000807770F76053E07270BA48F06206209B
:1098800030704DE0052A15D1F268042A28BF104631
:1098900009D2C2F10303D6F82CC0DB002CFA03F383
:1098A0000370501CF060042804D10120F760087098
:1098B000032030700120BDE8F0817078012500247C
:1098C00010F0010F11D002F0CBFEB0F5783F23D895
:1098D0006A030021B1EB900F07D252F8043B491CF8
:1098E0001C44B1EB900FF8D3B5B1707810F0020FB3
:1098F0000ED004F0A4FF78B182680021B1EB920F82
:1099000006D250F8043B491C1C44B1EB920FF8D32B
:10991000002D18BFF46200D1F762777086F80080DE
:109920000020BDE8F081F0B503F0070C00268A4D59
:109930008A4C83B0BCF1010F0ED013F0070F1DD07D
:10994000224603271278BCF1020F26D0BCF1040F87
:1099500008BF062A36D03CE002AA01A9684603F0F7
:1099600076FA052020702968019808702968009807
:109970004870296802988870E6602AE0E068032849
:1099800003D229680A54401CE060022821D3062132
:109990002170032808BFE6601BE0052A0FD1E268AA
:1099A000032A28BF104604D22B689B5C0370501C0E
:1099B000E060032803D10120E6600870277003B03F
:1099C0000120F0BD286882780178407803F032FAEF
:1099D000277003B00020F0BD08B503F00700012890
:1099E0000AD104F0CDFE38B101208DF80000024606
:1099F00069460D2002F066FE002008BD08B503F0A0
:109A0000070001280AD104F0BBFE38B100208DF810
:109A10000000012269460D2002F054FE002008BD1E
:109A200008B503F00700012809D104F0A9FE30B100
:109A300003208DF800000122694602F043FE002059
:109A400008BD0020704708B503F0070001280AD1BF
:109A500004F096FE38B10B208DF800000122694613
:109A6000032002F02FFE002008BD1FB513F0070FE2
:109A70000ED104F085FE58B19DF80800F0280AD0F8
:109A800004F07EFE20B1012202A9092002F01AFE94
:109A900004B0002010BDFEF713F9F9E7002070476D
:109AA00070B503F007002C4C2C4D012808D013F0A2
:109AB000070F12D0042804BF2878062816D01FE00C
:109AC0000020E8602168087021684870216888706B
:109AD0002168C8700520287012E0E86804280FD2B9
:109AE00021680A54401CE860062008E004F048FEA3
:109AF00030B104221046216802F0E4FD03202870F2
:109B0000002070BD10B503F00700012804D103F058
:109B1000C8FF124900200871002010BD7FB51C4607
:109B20000E46054613F0070F08D104F029FE28B1B0
:109B3000012202A91B2002F0C5FD03E004F007008A
:109B4000022802D004B0002070BD0AF04CF8287042
:109B50000120307004B070BDEC55020094850010F7
:109B600054464953EFBEADDE10B503F0070CFE4C72
:109B7000BCF1010F06D013F0070F09D0BCF1020FA2
:109B800018D015E00020E06007F0CBFEE0610FE0A8
:109B9000E068002804BF1002E06106D0012804D16B
:109BA000E0691043E06107F0BBFEE068401CE06044
:109BB000002010BDE26812B1012A04D007E0A18B99
:109BC000090A017003E0237F037001200870501C14
:109BD000E060012010BD10B503F0070CE24CBCF1B1
:109BE000010F06D013F0070F09D0BCF1020F18D0F7
:109BF00015E00020E06007F097FEE0610FE0E0680C
:109C0000002804BF1002E06106D0012804D1E069F9
:109C10001043E06107F08BFEE068401CE06000202C
:109C200010BDE26812B1012A04D007E0A18B090A35
:109C3000017003E0237F037001200870501CE06076
:109C4000012010BD70B503F0070CC74D0E46044649
:109C5000BCF1010F06D013F0070F07D0BCF1020FC3
:109C600018D015E00020E860286111E0E8680028BD
:109C700004BF1002E86108D0012806D1E86910434A
:109C800081B2E861E88810F0D9FCE868401CE8601F
:109C9000002070BD286902280ED2E88810F0D2FC9E
:109CA0002B6982B2002B04BF100A207004D0012B54
:109CB00002D12270012030702869401C28610120E7
:109CC00070BD10B403F0070CA74CBCF1010F08BF26
:109CD00000200BD013F0070F03D0BCF1020F09D006
:109CE00005E0E068002808BFE280401CE06010BC8E
:109CF00000207047E2681AB9A37903700120087048
:109D0000501CE06010BC012070472DE9F04706466A
:109D100003F00700944F8946012808BF002037D080
:109D2000DFF84882924D13F0070F02D0022833D09B
:109D30002FE0F868002808BF7A7027D0012804BFF8
:109D40001002F86122D0022820D1F8691043F8618E
:109D50007E7884B204F014FDC0B1062E16D2DFE87E
:109D600006F00306090C1013A8F80E400EE0A8F840
:109D70000C400BE02868848308E02868A0F80041C4
:109D800004E02868848501E02868C485F868401CE0
:109D9000F8600020BDE8F087386902282AD297F8D9
:109DA00001A0002404F0ECFCC8B1BAF1060F16D2F1
:109DB000DFE80AF00306090C1013B8F80E400EE0B5
:109DC000B8F80C400BE02868848B08E02868B0F8ED
:109DD000004104E02868848D01E02868C48D38695A
:109DE000002804BF200A307004D0012802D134704A
:109DF00089F800003869401C38610120BDE8F0870F
:109E00002DE9F0411C4617460E46054604F0B8FC05
:109E100068B114F0070F04D004F00700022809D03D
:109E200005E0002F14BF012000200CF0C5FB00202E
:109E3000BDE8F0814D4890F86C00C0082870012002
:109E40003070BDE8F0812DE9F0411C4615460F4603
:109E5000064613F0070F08D104F092FC28B1022D3A
:109E60003CBF284609F0CFFE03E004F007000228BB
:109E700002D00020BDE8F08109F0BEFE3070012064
:109E80003870BDE8F08170B503F007020026394C48
:109E9000354D012A02D0022A15D012E008F08EFEBC
:109EA00021680870FDF7D6FB2168487004F0CEF9F0
:109EB00021688870FDF7D4FB2168C87005202870E0
:109EC000EE60002070BD2A78052A10D1EA68042AC5
:109ED00028BF104604D223689B5C0370501CE860C6
:109EE000042804D10120EE600870032028700120AE
:109EF00070BD70B503F007021E4C00251A4E012AF2
:109F000002D0022A5ED05BE0FDF7B4FE002840D00C
:109F10004169FF292CBFFF21C9B2226811708169F4
:109F2000FF2934BFC9B2FF2122685170C169FF29DE
:109F300034BFC9B2FF21226891702268017CD170C0
:109F4000226890F820101171018C2268090A517161
:109F5000016A2268090C9171016A2268090ED171A7
:109F6000016BFF2908E000009485001044330110C4
:109F7000C8860010EC55020034BFC9B2FF21226828
:109F80001172406BFF2834BFC0B2FF2021684872B5
:109F900015E020680570206845702068857021688C
:109FA0005020C8702168FF2008712168487121681D
:109FB00088712168C8712068057220684572F56053
:109FC000002070BDF2680A2A28BF104604D2236818
:109FD0009B5C0370501CF0600A2802D10120F560E0
:109FE0000870012070BD03F00702FC4B4FF0000C1D
:109FF000012A08BFC3F80CC001D0022A01D00020FA
:10A000007047DA68022A3DBF80F800C0501CD86053
:10A010001046022803D10120C3F80CC008700120AB
:10A0200070472DE9F047064603F00700EB4F8A46DC
:10A030004FF00008012808BFC7F80C8001D00228A3
:10A0400002D00020BDE8F087F868A0BB00242546B8
:10A0500002F006FB014600F5005018384FF400529C
:10A060004FF04009B1F5783F20D890F803C003685D
:10A070006CF31F63DFF868C3634517D1091FB4EBA6
:10A08000910F06D252F8043B641C5D40B4EB910F73
:10A09000F8D3C17D406961F31F60A84206D104F086
:10A0A0006FFB012804BF8020307001D086F800903B
:10A0B000F868401CF860012803D1C7F80C808AF8C2
:10A0C00000000120BDE8F0872DE9F04103F0070210
:10A0D0000026C44CC14D012A02D0022A56D052E0BB
:10A0E000C14800680520287004F04AFB002849D0C8
:10A0F000BE4F386804F04CFC002843D010F081FAC1
:10A10000804610F082FA39680A7E12F0040F11D0EE
:10A11000C98A2268090A117039682268897D5170DC
:10A1200039682268898A090A917039682268097D2C
:10A13000D17010E0898A2268090A11703968226892
:10A14000097D517039682268C98A090A9170396895
:10A150002268897DD17022684FEA18211171216827
:10A1600081F805802268010A91712168C8713868F8
:10A170002268817C11722268017C5172008B2168F7
:10A18000000A8872EE600020BDE8F0812A78052A76
:10A1900010D1EA680B2A28BF104604D223689B5CC2
:10A1A0000370501CE8600B2804D10120EE60087099
:10A1B000032028700120BDE8F0812DE9F04703F06D
:10A1C00007020026874D854B012A02D0022A5DD066
:10A1D00059E0052018700024DE6002F041FA00F515
:10A1E0000053B0F5783F98BF13F0030F45D1804A74
:10A1F0001968914204BF0022114608D153F821C0CA
:10A20000491C62440729F9D3002A08BF01249F7C16
:10A2100093F8138084B341F6E8710144B0F5783FB8
:10A2200007D8CA78086862F31F606D4A904208BF79
:10A23000012491F8129091F813A0002C08BF00207F
:10A2400014D004F0FCFA2968806981F8009029682C
:10A2500081F801A02A68010C000E91702968C8706D
:10A2600028680771286880F805800CE029680E547A
:10A27000401C0628FAD306E0FFE7002029680E54A8
:10A28000401C0628FAD30020BDE8F0871A78052A7A
:10A2900013D1DA68072A28BF104607D2D5F800C0C4
:10A2A0001CF802C080F800C0501CD860072804D1F8
:10A2B0000120DE600870032018700120BDE8F087DF
:10A2C00070B5054603F007000C46022829D104F0BA
:10A2D00057FA30B3454800220068037EC3F380007C
:10A2E0008000C3F3400100EB410003F0010108448A
:10A2F000082812D2DFE800F00406080A0C0E11103C
:10A3000004220AE0052208E0062206E0072204E013
:10A31000022202E0032200E001222A7001202070C4
:10A3200070BD002070BD10B503F0070C2B4CBCF1C4
:10A33000010F06D013F0070F0AD0BCF1020F1AD09C
:10A3400017E00020E060206110F0DBF9E06110E030
:10A35000E068002804BF1002E06107D0012805D1A1
:10A36000E0691043E06180B210F0C8F9E068401C79
:10A37000E060002010BD2269022A0BD212B1012A2E
:10A3800004D007E0A18B090A017003E0237F03706A
:10A3900001200870501C2061012010BD70B503F031
:10A3A000070100260D4D0446012908BF2E6301D088
:10A3B000022901D0002070BD286B002804BF0D4881
:10A3C00015F04AFE296B082928BF267002D20948D9
:10A3D000405C2070481C2863012070BD94850010EB
:10A3E00034CD12ABEC550200044C0040C88600107E
:10A3F00054464953CC8500102DE9F04103F0070184
:10A400000026FA4D0746012908BF2E6301D0022914
:10A4100002D00020BDE8F08195F8300000F007047C
:10A420002879204304D1F24815F016FE0120287146
:10A43000052C28BF2E71EE48005D3870286B401C3B
:10A4400028630120BDE8F08170B5044603F00700E1
:10A450000D4602281CBF002070BD15F002FE2070C2
:10A460000120287070BD2DE9F04103F0070200269D
:10A47000E04DDE4C012A02D0022A1AD016E0052057
:10A480002070002211461046E66002F0E0FC4FF614
:10A49000FF7101EA40006061FDF7DCF8032803BFAB
:10A4A00028782028D44802F0E5FCA0620020BDE80E
:10A4B000F0812278052A1DD1D4F814C0E2686245E3
:10A4C00028BF104607D212F0010F1CBF637803703B
:10A4D00013D0501CE06060450CD10120E66008708C
:10A4E00003202070FDF7B6F8032806BF287820283F
:10A4F00002F0CDFC0120BDE8F081A76A22F0010343
:10A50000FB5A1F0A07706370E3E770B503F0070298
:10A510000025B64C012A02D0022A11D00EE0B7481D
:10A5200005220068B0F91210B0F91000227008443A
:10A530004000E560606102F02EFFA062002070BD67
:10A540002278052A17D1D4F814C0E268624528BFE2
:10A55000104607D212F0010F1CBF637803700CD0B5
:10A56000501CE060604506D10120E56008700320C2
:10A57000207002F01EFF012070BDA66A22F00103C8
:10A58000F35A1E0A06706370EAE7002070472DE94F
:10A59000F0419A4A03F00703944E12684FF0000806
:10A5A000012B02D0022B10D00CE005203070C6F831
:10A5B0000C80108A518A400848434000706102F0C4
:10A5C00059FCB0620020BDE8F0813378052B17D12B
:10A5D0007469F368A34228BF184607D213F0010F2D
:10A5E0001CBF727802700ED0581CF060A04207D1D8
:10A5F0000120C6F80C8008700320307002F047FC80
:10A600000120BDE8F081B2F812C05F08B7FBFCF58D
:10A610000CFB1577128AACEB070C0CFB02F2D6F898
:10A6200028C0521B0CEB420232F8022C4FEA122CCB
:10A6300080F800C07270D7E72DE9F0416F4A03F04F
:10A6400007036A4E12684FF00008012B02D0022B5C
:10A6500010D00CE005203070C6F80C80108A518AAA
:10A66000400848434000706102F004FCB0620020E2
:10A67000BDE8F0813378052B17D17469F368A342E4
:10A6800028BF184607D213F0010F1CBF7278027062
:10A690000ED0581CF060A04207D10120C6F80C80F3
:10A6A00008700320307002F0F2FB0120BDE8F08159
:10A6B000504D9C462D78282D03D1558A178A05FBCD
:10A6C00007CC4FEA5C07B2F812C0128AB7FBFCF560
:10A6D0000CFB1577ACEB070C0CFB02F2D6F828C08C
:10A6E000521B0CEB420232F8022C4FEA122C80F87B
:10A6F00000C07270CDE770B503F0070200253B4C37
:10A70000012A02D0022A14D011E03C480522006838
:10A71000B0F91210B0F91000227008444000E56052
:10A72000606102F038FE3649A06203F069F800204B
:10A7300070BD2278052A17D1D4F814C0E2686245AA
:10A7400028BF104607D212F0010F1CBF63780370B8
:10A750000CD0501CE060604506D10120E560087017
:10A760000320207002F025FE012070BD244E22F04F
:10A770000103F35A1E0A06706370EAE770B50D46CE
:10A78000044613F0070F04D003F00700022805D099
:10A7900002E01046FCF758FF002070BDFCF757FFA1
:10A7A00020700120287070BD70B503F007020325EA
:10A7B0000E4C012A02D0022A24D014E004F011F930
:10A7C0000646FCF744FF0146304604F08EFB20624B
:10A7D00000281ABF052020702570304604F06CFB5D
:10A7E00060620020E060002070BD000094850010D1
:10A7F000CC850010E5850010642B0110C886001080
:10A80000D0AA00102278052A0BD1236AE2689B5C4B
:10A810000370501CE060626A904202D3012008700D
:10A8200025700120E0E700207047002070477FB5C9
:10A830001C460E46054613F0070F08D103F0A0FF93
:10A8400028B1012202A9262001F03CFF03E004F018
:10A850000700022802D004B0002070BD02F0D3FB34
:10A8600028700120307004B070BD2DE9F04103F074
:10A8700007020027FE4E88460546012A02D0022A1A
:10A880000BD007E0052030700A20F760706102F0FD
:10A89000F1FAB0620020BDE8F0813078052819D1C6
:10A8A000F2687069824228BF104608D212F0010F88
:10A8B0001CBF7078287010D0F068401CF06071697F
:10A8C000884207D10120F76088F80000032030702B
:10A8D00002F0DDFA0120BDE8F081002402F093FBD4
:10A8E000012804D1F068B16A20F001000C5A200A56
:10A8F00028707470E0E770B50D46044613F0070F3A
:10A9000004D003F00700022805D002E0104604F04E
:10A9100065F8002070BD04F064F8207001202870F4
:10A9200070BD7FB51C460E46054613F0070F08D1D3
:10A9300003F026FF28B1012202A9202001F0C2FE67
:10A9400003E004F00700022802D004B0002070BD2C
:10A9500008F076FA28700120307004B070BD7FB521
:10A960001C460E46054613F0070F08D103F008FFFA
:10A9700028B1012202A9212001F0A4FE03E004F085
:10A980000700022802D004B0002070BD08F05EFA73
:10A9900028700120307004B070BD7FB51C460E4693
:10A9A000054613F0070F08D103F0EAFE28B1012293
:10A9B00002A91C2001F086FE03E004F00700022833
:10A9C00002D004B0002070BDFCF752FF28700120B7
:10A9D000307004B070BD7FB51C460E46054613F0BE
:10A9E000070F08D103F0CCFE28B1012202A90C20E8
:10A9F00001F068FE03E004F00700022802D004B072
:10AA0000002070BD08F0DAF828700120307004B022
:10AA100070BD7FB51C460E46054613F0070F08D1E2
:10AA200003F0AEFE28B1012202A90F2001F04AFE78
:10AA300003E004F00700022802D004B0002070BD3B
:10AA40000FF03DFA00F00F0040F0100028700120D8
:10AA5000307004B070BD2DE9F04103F0070C844D57
:10AA60000E460746BCF1010F07D0824C13F0070FCA
:10AA700007D0BCF1020F1BD017E00020E86028616E
:10AA800013E0E86804283CBF21680A54032809D170
:10AA9000206821680068C97800BA20F0FF000843E8
:10AAA000FBF763FDE868401CE8600020BDE8F0812A
:10AAB000286970B9FBF75EFD216820F07E42100E18
:10AAC00008702168100C48702168100A887020688E
:10AAD000C2702A69042A06D22068032A805C387072
:10AAE00004BF01203070501C28610120BDE8F081B6
:10AAF0007FB51C460D46064613F0070F08D103F03C
:10AB00003FFE28B1012202A9102001F0DBFD03E085
:10AB100004F00700022802D004B0002070BD0FF03E
:10AB2000D2F900F00F040FF0CAF964F31F1030706F
:10AB30000120287004B070BD70B54D4D144613F05F
:10AB4000070F04D003F00702022A06D003E01046E4
:10AB5000F5F732FC6C63002070BD95F8342002706C
:10AB60000120087070BD70B514460E46054613F0FE
:10AB7000070F04D003F00700022808D005E01046B4
:10AB8000FBF7DCFC60B215F071FA002070BDFBF73A
:10AB9000DAFC28700120307070BD2DE9F04103F01F
:10ABA000070C344D324C4FF00008BCF1010F0DD0B2
:10ABB00013F0070F1AD022462F4E03271278BCF14C
:10ABC000040F1DD0BCF1020F3DD02FE0C4F80C8063
:10ABD000286880F80080286880F80180286880F85C
:10ABE0000280286880F80380052007E0E0680428D8
:10ABF0001CD229680A54401CE0600620207015E031
:10AC0000062A13D103F0BCFD80B12868007810B18A
:10AC100001280ED009E0286840780028706814BF29
:10AC200040F0800020F08000706027700020BDE8B8
:10AC3000F081286840780028706814BF40F40070E4
:10AC400020F40070F0E7052A0FD172687368C2F330
:10AC5000C01203F4007342EA53122B681A70027098
:10AC60000120C4F80C80087027700120BDE8F08135
:10AC700094850010EC5502000010004010B503F060
:10AC80000702F74C012A02D0022A0DD00AE004F094
:10AC900082F90021206200281ABF4FF4056060622B
:10ACA0006162E160002010BD636AE2689A4228BFD9
:10ACB000104607D2D4F820C01CF802C080F800C0AB
:10ACC000501CE060984204BF01200870012010BDB4
:10ACD00010B4DFF890C313F0070F04D003F007029D
:10ACE000022A13D00FE0012A04BFDCF8000040F074
:10ACF000010006D0002A04BFDCF8000020F00100AB
:10AD000001D1CCF8000010BC00207047DCF8003006
:10AD1000002213F0010F18BF0122D34BD3F804C057
:10AD2000D24B1B68B3F8DC30C3F30334012303FABE
:10AD300004F41CEA040F18BF42F0020202700B7008
:10AD400010BC0120704770B514460E46054613F03E
:10AD5000070F04D003F0070002280ED00BE0002CF0
:10AD600014BF0120002002F07BFE24B1BE48016820
:10AD700021F440510160002070BD02F078FE0028EF
:10AD800014BF012200222A700120307070BD2DE90D
:10AD9000F04103F0070CB24C0F468046BCF1010FA6
:10ADA00012D0B14E13F0070F4FF0030510D020461C
:10ADB000BCF1020F027826D0BCF1040F02BFE0689C
:10ADC0000128062A33D036E005202070002018E044
:10ADD000E06810B1012804D011E0627006202070F4
:10ADE0000DE07168607800EA0203194371607168D0
:10ADF00020EA020291437160F9F7ACF92570E0682E
:10AE0000401CE06017E0E068012808BF062A03D173
:10AE10006078F9F7B5F92570706888F800000120AE
:10AE20003870E068401CE0600120BDE8F081607887
:10AE3000F9F7A6F925700020BDE8F08170B5044649
:10AE400003F007000D4602281CBF002070BDFCF770
:10AE5000F1FC002814BF012200222270012028707A
:10AE600070BD70B50D46044613F0070F04D003F013
:10AE70000700022805D002E0104607F0C9FD0020B7
:10AE800070BD07F0C8FD20700120287070BD70B53E
:10AE90000D46044613F0070F04D003F00700022804
:10AEA00005D002E01046F6F780F8002070BDF6F7F6
:10AEB0007FF820700120287070BD70B503F0070284
:10AEC000DFF89CC10C460546012A08BF05200DD0BD
:10AED00013F0070F08BF062008D0022A09D0042A61
:10AEE00004BF9CF80000062809D00EE08CF8000092
:10AEF0000BE0FCF7C3FC28700120207070BD03201C
:10AF00008CF800000120FCF7BCFC002070BD70B57F
:10AF100003F00702524D0E460446012A04BF0020EA
:10AF2000E86001D0022A01D0002070BD10F0FEFAC6
:10AF3000EA68002A04BF000A207004D0012A02D166
:10AF4000207001203070501CE860012070BD03F0BB
:10AF5000070210B4424B012A04BF0020D86001D080
:10AF6000022A02D010BC00207047DA68022A0CD2F4
:10AF70004FF0010C002A08BF80F800C005D0012A5C
:10AF800003D14024047081F800C0501CD86010BC6C
:10AF90000120704770B5044603F007000D460228F3
:10AFA00007D013F0070F04BF1046FCF747FB002043
:10AFB00070BDFCF746FB20700120287070BD70B595
:10AFC000044603F00700264D0E46012804BF00206A
:10AFD000E86014D013F0070F02D0022811D00EE061
:10AFE000E868234904283CBF0B681A54401CE860F9
:10AFF000042804D104220968132001F063FB002017
:10B0000070BD0DF063FCEA68002A04BF000E2070DA
:10B010000FD0012A08BF000C06D0022A08BF000A80
:10B0200002D0032A02D004E0207002E02070012048
:10B030003070501CE860012070BD70B503F0070C43
:10B04000074D0E460446BCF1010F04BF0020E86026
:10B050001FD013F0070F0DD0BCF1020F1BD018E06A
:10B0600094850010144C004000100040C886001069
:10B07000EC550200E868F94902283CBF0B681A54F5
:10B08000401CE860022804D102220968142001F063
:10B0900019FB002070BD0DF0E5FBEA68002A04BF33
:10B0A000000A207004D0012A02D1207001203070E3
:10B0B000501CE860012070BD70B5044603F0070025
:10B0C000E74D0E46012804BF0020E86014D013F0BD
:10B0D000070F02D0022811D00EE0E868DF490428EB
:10B0E0003CBF0B681A54401CE860042804D10422B9
:10B0F0000968152001F0E6FA002070BD0DF021FC72
:10B10000EA68002A04BF000E20700FD0012A08BF91
:10B11000000C06D0022A08BF000A02D0032A02D07F
:10B1200004E0207002E0207001203070501CE860C4
:10B13000012070BD2DE9F041044603F00700002511
:10B14000C74E0F46012808BFF5603BD013F0070F2C
:10B1500002D0022839D035E0F068C04C002804BF86
:10B1600021680A7021680978012901D039B11FE0EE
:10B17000002818BF06283CBF21680A5418E00DF0CB
:10B18000FBFB2168000948700DF0EAFBC0F30327C0
:10B190000DF0F2FB216847EA001088700DF0E0FB2B
:10B1A0002168C87020680571206845710520F0602D
:10B1B000F068401CF060062804D1062216202168A1
:10B1C00001F080FA0020BDE8F0810DF0EDFB0546AE
:10B1D0000DF0DEFB80460DF0E1FBF268002A04BFB3
:10B1E000280E207018D0012A08BF280C0FD0022A80
:10B1F00008BF280A0BD0032A08BF25700CD0042AE8
:10B2000008BF84F8008007D0052A02D004E020702F
:10B2100002E0207001203870501CF0600120BDE871
:10B22000F08110B503F007028D4C012A02D0022AEA
:10B2300027D024E003F0AFFE0023002804BF2362E0
:10B2400063621BD000F1500121624168B1F5887F33
:10B2500090F820100CD390F8212001EB020C01FB98
:10B2600002C190F8222090F823001044084404E022
:10B2700090F822000A1801FB00206062E3600020C1
:10B2800010BD636AE2689A4228BF104607D2D4F81C
:10B2900020C01CF802C080F800C0501CE06098423A
:10B2A00004BF01200870012010BD03F00702012A2D
:10B2B00002D0022A05D002E069490020C8600020BF
:10B2C0007047012202700A701046704710B513F0E3
:10B2D000070F04D003F00702022A05D002E010464F
:10B2E00001F0E2FD002010BD5E4A127802700120DC
:10B2F000087010BD10B513F0070F04D003F007025B
:10B30000022A05D002E0104602F060F8002010BDCD
:10B31000554A127802700120087010BD0020704755
:10B3200003F007024E4B4FF0000C012A08BFC3F890
:10B330000CC001D0022A01D000207047DA68002A30
:10B3400008BF80F800C0501CD860012804BF01204D
:10B350000870012070471FB513F0070F07D103F0E5
:10B360000FFA20B1012202A90B2001F0ABF904B0C1
:10B37000002010BD70B503F00700394C15460128B8
:10B3800004BF0020E06024D013F0070F21D103F0A8
:10B39000F7F9F0B1E068314E03283CBF31680D5435
:10B3A000401CE060032814D1F7F70FFC3068B0F8B8
:10B3B000010045BAF7F710FB040018BFF7F7A7FD27
:10B3C000306829460078F6F7AAF9002C18BFF7F77D
:10B3D000A1FD002070BD70B503F00700204D14469C
:10B3E000012804BF0020E86020D013F0070F1DD112
:10B3F00003F0C6F9D0B1E868184E02283CBF3168A6
:10B400000C54401CE860022810D1F7F7DEFBF7F778
:10B41000E3FA040018BFF7F77AFD30684178007846
:10B42000F6F729FA002C18BFF7F774FD002070BD5D
:10B4300070B50D46044613F0070F04D003F0070063
:10B44000022805D002E01046F7F781FD002070BD0C
:10B45000F7F780FD20700120287070BDEC550200C8
:10B4600094850010E5850010EB8500107FB51C4623
:10B470000E46054613F0070F08D103F081F928B1F5
:10B48000012202A9172001F01DF903E004F00700D2
:10B49000022802D004B0002070BD07F06AFB00282B
:10B4A00014BF012200222A700120307004B070BD48
:10B4B0007FB51C460E46054613F0070F08D103F072
:10B4C0005FF928B1012202A9182001F0FBF803E07E
:10B4D00004F00700022802D004B0002070BD07F07D
:10B4E00035FB28700120307004B070BD2DE9F041AB
:10B4F00003F0070CFE4C0E460746BCF1010F07D0C7
:10B50000FC4D13F0070F07D0BCF1020F19D015E066
:10B510000020E060206111E0E06803283CBF29685A
:10B520000A54401CE060032808D12868B0F80100E4
:10B5300040BA01B228680078FDF7FFFD0020BDE8A1
:10B54000F0812269022A12D242B928680078FDF7F8
:10B55000FDFD2A68010A51702968887028682269EF
:10B560001044012A4078387004BF012030702069EF
:10B57000401C20610120BDE8F08110B503F00700F8
:10B58000DB49012808BF00200CD013F0070FD94B6E
:10B5900002D0042808D018E0C86804283CBF1B6803
:10B5A0001A54401CC86010E0C86804280DD31868FD
:10B5B000196840788978000440EA01201968C97840
:10B5C000014318680078F8F721F9002010BD10B584
:10B5D00003F00702C64C012A02D0022A07D004E079
:10B5E0000020E060F9F799F9E061002010BDE26801
:10B5F000042A07D2C2F10303D4F81CC0DB002CFAE2
:10B6000003F30370501CE060042804BF012008709D
:10B61000012010BD10B503F00700012807D103F089
:10B62000AFF820B1002211461D2001F04BF8002098
:10B6300010BD2DE9F04103F00705AD4E17468846D1
:10B640000446012D04BF0020F0601BD013F0070F4B
:10B6500016D103F095F898B1F068A64B03283CBFCB
:10B6600019680F54401CF06003280BD1186890F93A
:10B67000022090F9011090F90000FAF7A1FD01E015
:10B68000022D02D00020BDE8F081F06830B1012821
:10B6900009D002280CD003280FD015E01420FAF7A7
:10B6A00038FC207010E01520FAF733FC20700BE016
:10B6B0001620FAF72EFC207006E01720FAF729FC76
:10B6C0002070012088F80000F068401CF060012024
:10B6D000BDE8F08170B50D46044603F00700002177
:10B6E000834E012814BF13F0070FF16001D0022828
:10B6F00001D0002070BDF06840B101280BD00228B5
:10B700000ED0032811D0042814D019E00120FAF734
:10B7100000FC207014E00220FAF7FBFB20700FE021
:10B720000320FAF7F6FB20700AE00420FAF7F1FB99
:10B73000207005E00520FAF7ECFB2070012028704E
:10B74000F068401CF060012070BD70B503F0070C7C
:10B750000026684C664DBCF1010F06D013F0070FB0
:10B760000CD0BCF1020F1FD01CE007F035FBEE60DF
:10B77000216808702168000A487013E0E868022810
:10B7800003D221680A54401CE86002280AD1EE6006
:10B790002068007810F0010F04D0022219202168DF
:10B7A00000F090FF002070BDEA68022A28BF104612
:10B7B00004D223689B5C0370501CE860022804D10B
:10B7C0000120EE60087003202870012070BD7FB555
:10B7D0001C460E46054613F0070F08D102F0D0FFB5
:10B7E00028B1012202A9242000F06CFF03E004F03C
:10B7F0000700022802D004B0002070BD0EF070FFD8
:10B8000028700120307004B070BD7FB51C460E4614
:10B81000054613F0070F08D102F0B2FF28B101224C
:10B8200002A91F2000F04EFF03E004F007000228E9
:10B8300002D004B0002070BD0EF05DFF2870012022
:10B84000307004B070BD7FB51C460E46054613F03F
:10B85000070F08D102F094FF28B1012202A923208A
:10B8600000F030FF03E004F00700022802D004B02B
:10B87000002070BD11F0B0FF28700120307004B0BE
:10B8800070BD7FB51C460E46054613F0070F11D15B
:10B8900002F076FF70B10EF03AFF01469DF8080005
:10B8A00081420BD00EF030FF012202A91E2000F0D1
:10B8B00009FF03E004F00700022802D004B00020D2
:10B8C00070BD0EF024FF28700120307004B070BDF0
:10B8D0002DE9FF41064E1C460F46054613F0070FA3
:10B8E00021D102F04DFFF0B19DF80800002803E0DF
:10B8F00094850010EC55020018BF012802D00228E0
:10B9000007D014E0F070012202A9082000F0DAFE4E
:10B910000DE0F07004208DF80800012202A9082033
:10B9200000F0D0FE03E004F00700022803D004B0CA
:10B930000020BDE8F081F07828700120387004B054
:10B94000BDE8F0817FB51C460D46064613F0070F93
:10B9500008D102F015FF28B1012202A9082000F049
:10B96000B1FE03E004F00700022802D004B000207A
:10B9700070BDFBF76FFE801E052813D2DFE800F0D4
:10B9800003070E05100000240DE001240BE0022443
:10B9900006F0C1F8042808BF052404E0032402E0EF
:10B9A000042400E0FF2434700120287004B070BD2E
:10B9B0002DE9F0411C4617460E46054613F0070FC9
:10B9C0000BD102F0DDFE40B1384607F01BF8002233
:10B9D0001146012000F076FE03E004F00700022883
:10B9E00002D00020BDE8F08107F00FF82870012098
:10B9F0003070BDE8F08110B5104613F0070F08BF96
:10BA000007F0CAF8002010BD10B5104613F0070F5C
:10BA100008BF07F0C8F8002010BD70B5044603F059
:10BA200007000D4602281CBF002070BD07F0C3F8B8
:10BA300020700120287070BD03F0070230B4FD4B68
:10BA40004FF0000C012A05D0022A04BF1A78022AFE
:10BA50000BD01EE002201870F748C3F80CC06FF03E
:10BA60007F410068081AD86113E0DA68042A28BF09
:10BA7000104606D2DD69D40025FA04F40470501C87
:10BA8000D860042805D10120C3F80CC00870032039
:10BA9000187030BC0120704713F0070F04BFE7484F
:10BAA00002700020704710B503F00700E14901283B
:10BAB00004BF0020C86013D013F0070F10D1C8686E
:10BAC000DF4B04283CBFD3F800C00CF80020401C1A
:10BAD000C860042804D104221220196800F0F2FD85
:10BAE000002010BD2DE9F047164603F007020024A0
:10BAF000D04F012A04BFFC603C6164D0DFF844836E
:10BB000013F0070F07D0022A33D0042A04BF387875
:10BB100006284FD058E0FD68002D08BF3E6225D0B2
:10BB2000012D06D0D7F81490AC1E4C4516D284B91E
:10BB300008E0701C7861396A0844B0F5007F88BF5E
:10BB40007C6113E04FF400724FF47A31BE4814F078
:10BB50001FFABB49386A096820440E54601C4845E6
:10BB600004D1B948C0F8FC8106203870681CF86020
:10BB70002AE0FF2202707B69CBB1D7F820C03A6976
:10BB80009444BCF5007F10D2B04D2D68454518BFD8
:10BB9000047005D10CF5783C9CF800C880F800C012
:10BBA000501C984204BF01200870501C38610120CD
:10BBB000BDE8F0874FF47A30F8F760F9A2494FF406
:10BBC0007A30F8F7FDF93C700020BDE8F0872DE9E8
:10BBD000F0478C4603F007010024964F16460129D2
:10BBE00004BFFC603C6162D013F0070F984BDFF894
:10BBF000648207D0022932D0042904BF387806288D
:10BC00004DD055E0FD68002D08BF3E6224D0012DC7
:10BC100006D0D7F81490AC1E4C4515D27CB908E07C
:10BC2000701C7861396A0844B0F5007F88BF7C6178
:10BC300012E04FF400721946834814F0A9F98049C4
:10BC4000386A096820440E54601C484504D17E4877
:10BC5000C0F8FC8106203870681CF86028E0FF21DD
:10BC600001707B69C3B13A6A39690A44B2F5007F51
:10BC700010D2794D2D68454518BF047004D102F5E6
:10BC8000783292F800260270481C984204BF0120C6
:10BC90008CF80000481C38610120BDE8F0871D4683
:10BCA0001846F8F7EBF868492846F8F789F93C7028
:10BCB0000020BDE8F08770B503F007005D4C154625
:10BCC000012804BF0020E06014D013F0070F11D149
:10BCD00002F056FD70B1E068594902283CBF0A687D
:10BCE0001554401CE060022804D102220968052096
:10BCF00000F0E8FC002070BD2DE9F041054603F09E
:10BD000007004F4C4B4E0F4601280AD013F0070F87
:10BD100014D002281BD0042804BF3078062834D061
:10BD20003FE00020F06021680870216848702168B9
:10BD300088702168C8700520307032E0F0680428EF
:10BD40002FD221680A54401CF060062028E0F068D9
:10BD500060B906F069FC216808702268010A517018
:10BD60002268010C000E91702168C870F0680428E8
:10BD70003ABF2168095CFF21297024BF0121397075
:10BD8000401CF0600120BDE8F08102F0F9FC40B1F8
:10BD90002068C178006861F31F6006F040FC032052
:10BDA00030700020BDE8F081002070477FB51C4650
:10BDB0000E46054613F0070F08D102F0E1FC28B14A
:10BDC000012202A9272000F07DFC03E004F0070017
:10BDD000022802D004B0002070BD06F012FF2870C7
:10BDE0000120307004B070BD03F007001149012834
:10BDF00008BF002009D013F0070F07D1C86818B991
:10BE0000164B1B681A448A61401CC86000207047AA
:10BE10002DE9F04103F00701064C164605460129BD
:10BE20001ED00E4F13F0070F38681DD0022930D0F6
:10BE30002CE0000094850010B484001036840010BB
:10BE4000EC550200554E564DD0A80010FCE90300F9
:10BE500000E60300324E564DFCE70300E886001072
:10BE60000020E060206111E0A56905F063FE012873
:10BE70000CD1A0693968884224BFD431814205D9E8
:10BE8000E068042838BF2E54401CE0600020BDE864
:10BE9000F081A66905F04EFE50B1A26939688A4268
:10BEA00024BF01F1D400904284BF2069305C00D8E7
:10BEB000FF2028702069401C20610120BDE8F0812E
:10BEC0007FB51C460E46054613F0070F08D102F059
:10BED00057FC28B1012202A9112000F0F3FB03E076
:10BEE00004F00700022802D004B0002070BD11F059
:10BEF000E6FA28700120307004B070BD0020704751
:10BF00000020704770B50D46044613F0070F04D0AB
:10BF100003F00700022805D002E010460AF09FF85F
:10BF2000002070BD0AF0A7F820700120287070BDB5
:10BF300010B503F00702FF4CFF4B4FF0000C012A35
:10BF400002D0022A30D02DE0C3F80CC002F018FC59
:10BF5000002827D0F94802F02AFD18B3F8480068F5
:10BF6000007E10F0040FF5480ED0C18A2268090A3D
:10BF700011702268817D5170818A2268090A91704E
:10BF80002168007DC8700DE0818A2268090A11705D
:10BF90002268017D5170C18A2268090A9170216866
:10BFA000807DC870002010BDDA68042A28BF1046C2
:10BFB00004D22468A45C0470501CD860042803D107
:10BFC0000120C3F80CC00870012010BD70B503F04B
:10BFD0000701D84DD84C012902D0022914D011E014
:10BFE000012001F04DFC0020E06001F05EFC2081AA
:10BFF000296808702A68010A0028517004BF0020CF
:10C0000001F03EFC002070BDE168022902D22A68DE
:10C01000525C0270481CE060012070BD2DE9F041C7
:10C0200003F007020026C44D0F460446012A02D041
:10C03000022A09D005E005202870EE60288940001A
:10C0400068610020BDE8F0812878052817D1EA68EA
:10C050006869824205D212F0010F1CBF6878207017
:10C0600010D0E868401CE8606969884207D1012067
:10C07000EE60387003202870002001F001FC0120E0
:10C08000BDE8F08101F02AFC010A21706870E8E740
:10C090001FB513F0070F04D1012202A91A2000F0E6
:10C0A00011FB04B0002010BD002070470020704735
:10C0B00003F00700A049012806D013F0070F04BFC2
:10C0C0000878012806D014E0012008700020C8601C
:10C0D00088610DE0C868042805D28B69401C42EADB
:10C0E00003228A61C860042803D10320087088698C
:10C0F00008620020704703F00700DFF83CC2012807
:10C1000007D013F0070F04BF9CF80000022809D0E5
:10C110001EE002208CF800000020CCF80C00CCF8C7
:10C120001C0015E0DCF80C00022808D2DCF81C101A
:10C13000401C42EA0121CCF81C10CCF80C0002286B
:10C1400006D1DCF81C00CCF8240003208CF8000099
:10C150000020704770B403F007020025764C012AD6
:10C1600002D0022A06D002E002202070E56070BCF6
:10C17000002070472278022A1CD1D4F824C0E2683B
:10C18000624528BF10460ED212F0030F04D1236A75
:10C1900053F8046BC4E90763237F0370E069000A66
:10C1A000E061501CE060604504D10120E56008704A
:10C1B0000320207070BC0120704770B503F00700A9
:10C1C00000255D4C0E46012806D013F0070F04BF72
:10C1D0002078022805D02BE002202070E560E56180
:10C1E00026E0616AE068884219D2E169090A41EAF9
:10C1F0000262401CE26110F0030FE0600FD1206A80
:10C20000B0F5802F28BF026006D2B0F5005F03D3DF
:10C2100004224C49F7F728FF206A001D2062616A5A
:10C22000E068884204D10120E5603070032020706E
:10C23000002070BD70B503F0070C00253E4CBCF12A
:10C24000010F08BFE5603AD013F0070F03D0BCF12F
:10C25000020F36D033E0052A08BF4FF47A302DD0D4
:10C2600005DC16D2DFE802F0171A1D202200344840
:10C27000202A006808BFE43020D006DC102A1DD038
:10C28000112A08BF2D4819D003E0302A11D0312AD5
:10C2900012D0A56113E04FF400500FE04FF47F304F
:10C2A0000CE04FF4503009E0274807E04FF47C30B1
:10C2B00004E001F05BFC01E010F097FCA0610020BD
:10C2C00070BDE268042A07D2C2F10303D4F818C093
:10C2D000DB002CFA03F30370501CE060042824BF39
:10C2E00001200870012070BD70B403F0070C124DDE
:10C2F000BCF1010F07D00F4C13F0070F07D0BCF1B2
:10C30000020F2ED02AE00020E860286126E0E868CD
:10C3100005283CBF21680A5404281DD123682268DF
:10C32000A969D3F8013012781BBA23F0FF03D4F8BF
:10C3300000C00BE0EC55020094850010443301105E
:10C34000C8860010B085001000EE03009CF804C001
:10C3500043EA0C0341F82230401CE86070BC002026
:10C3600070472B6973B1042B07D22268032B1A4440
:10C370005278027004BF01200870581C286170BCFC
:10C38000012070472268D5F818C012785CF8222086
:10C3900026684FEA126C86F801C026684FEA124CF4
:10C3A00086F802C026684FEA122C86F803C0D4F83B
:10C3B00000C08CF80420D8E710B503F0070001286E
:10C3C00004D1002211460E2000F07CF9002010BD9F
:10C3D0002DE9F04103F00704A94E174688460546AB
:10C3E000012C04BF0020F06017D013F0070F12D10A
:10C3F00002F0C6F978B1F068A24902283CBF0A6889
:10C400001754401CF060022807D102220968072057
:10C4100000F058F901E0022C02D00020BDE8F081C4
:10C42000F26812B1012A04D009E0FBF713F9287071
:10C4300005E0FBF715F92870012088F80000F06886
:10C44000401CF0600120BDE8F08170B503F00700EA
:10C4500000258B4C012808D013F0070F0BD00428BF
:10C4600004BF2078062825D02DE0A561E561657020
:10C47000E560257027E0E068022807D2A16942EA5A
:10C480000121A16161781144617010E0042807D294
:10C49000E16942EA0121E16161781144617006E0DD
:10C4A000052804D261788A4204BF06212170401C0D
:10C4B000E06008E0D4E9060101F0CAFB002804BFEF
:10C4C0000120A0702570002070BD10B56C4C13F0D9
:10C4D000070F07D003F00700042804BF20780628C0
:10C4E00022D02BE0E068022807D2A16942EA0121AC
:10C4F000A16161781144617013E06349091808D2A1
:10C5000060490968014401F8022C617811446170A6
:10C5100007E05E49091804D261788A4204BF062107
:10C520002170401CE06009E05949A06901F0B2FBAC
:10C53000002804BF0120A07000202070002010BD42
:10C5400003F0070CBCF1010F00D0BEE74C490020FE
:10C5500088614870C8600870704730B403F0070500
:10C560000024DFF81CC1012D07D013F0070F0DD0F8
:10C57000022D3CD0042D54D06FE0CCF81840CCF8FC
:10C580001C40CCF80C408CF8004066E0DCF80C0055
:10C5900002280BD2DCF8181042EA0121CCF818105E
:10C5A0009CF8011011448CF8011019E0042817D2EE
:10C5B000DCF81C10032842EA0121CCF81C109CF87E
:10C5C00001301A448CF801200AD106228CF8002090
:10C5D000DCF81820114304BF4FF40071CCF81C1094
:10C5E0002C49401CCCF82C10CCF80C0035E0DCF8C1
:10C5F0000C20042A28BF10460AD2C2F10303DCF83B
:10C600002C50DB0025FA03F30370501CCCF80C000F
:10C61000042803D10120CCF80C40087030BC012064
:10C6200070479CF80000062815D1DCF8180000229D
:10C630004102DCF81C0043021046B2EB930F06D215
:10C6400051F8045B401C2A44B0EB930FF8D3CCF8AC
:10C650002C208CF80040CCF80C4030BC00207047F7
:10C660004FF47F300168880A424211EB822218BFE2
:10C67000401C404201EB8000C01C20F003007047CA
:10C6800094850010EC550200FEFDFFFFFDFDFFFF4D
:10C69000D0A80010EFBEADDEF94800220270427053
:10C6A000827002714271C270DFF8D8C31146002057
:10C6B0000CEBC1031A54401C0828FBD3491C202949
:10C6C000F5D3704713F0D7BC2DE9F04115460E465F
:10C6D0000746F8F737F800F008040820F8F72DF8B7
:10C6E0002A463146384613F0C6FC05462046F8F780
:10C6F0001FF82846BDE8F081E14880787047E0489F
:10C7000040787047DE49002048707047DC49CA68AD
:10C710001043C860704710B568B1F8F749FC78203D
:10C72000F4F757FCD848F8F765FDF8F748FDBDE881
:10C730001040F8F7CBBCF8F7D2FCF8F74DFD00201D
:10C74000F8F758FDBDE81040F8F714BCCC4910B517
:10C7500008208871FAF77EFFAFF24500BDE810406F
:10C76000F6F74DBB2DE9F0474FF00008F6F74FFB09
:10C77000DFF80CA30446DAF80C00C14640B1DAF841
:10C780000C0010F0400F18BF44F00404CAF80C90DD
:10C7900014F00F0664D00127FAF75CFF0546304617
:10C7A000F6F752FB012E1DD0FAF75AFF44EA006457
:10C7B000002322460321072005F0BCF814F0050FE2
:10C7C00014BF00200120F3F7D7FD14F0060F47D067
:10C7D0004FF0010806F02AF90646022D2CD0052D4F
:10C7E0000AD03DE09AF80600854208BF00278AF883
:10C7F0000650002FD8D1E8E714F0020F13D0F4F759
:10C8000036F8F8B1F4F742F8040AF4F73FF8C0B28A
:10C8100044EA002200236C21022005F08BF800205E
:10C82000F4F71FF80EE0994C206858B10120F9F791
:10C8300044F9C4F8009005E014F0020F1CBF012079
:10C84000F9F73BF901F076FA002818BF01F079FA00
:10C85000022E05D0022D4FF0020004D001F04AFA5A
:10C860004046BDE8F08706F089F9F9E72DE9F04F79
:10C8700083B00027F8F721FDFAF7ECFE022804D177
:10C8800001F03AFF002818BF0127FFF76BFF0028CF
:10C8900018BF0127DFF8E89199F80200002800F09E
:10C8A0008A82D9F808006D464FF0FF34002640B167
:10C8B000D9F8082000230121084605F03BF8C9F803
:10C8C0000860F7F73FFF00F0080A0820F7F735FF88
:10C8D00099F80300DFF8ACB1F0B199F805000BEB63
:10C8E000C001401CC0B289F80500202828BF89F883
:10C8F000056099F80300401E89F803004C7891F810
:10C9000000800020002C05DD0A1892782A54401C73
:10C910008442F9DC0E704E705046F7F709FF002C88
:10C92000C0F2398208F0FF000024282880F0ED8151
:10C93000DFE800F0B93A14212C3D184AEE4FB98BCC
:10C9400091CCED96A0B4ECEBEAE9E8F4E6E5E4E39B
:10C95000E2E1B9E0DFDEB9DDDCB9DBAE0020F9F7FA
:10C96000ACF821E09DF80000AC280CBF01200220AB
:10C97000FAF738FF18E09DF800100120FAF785FE5D
:10C98000012089F80100044600F0BFB99DF80310AA
:10C99000009861F31F6002F01BF801210320FAF7F1
:10C9A00074FE012089F80100012400F0AEB9BDF841
:10C9B000000040BA05F03BFE02210320FAF765FEB5
:10C9C000012089F80100EFE79DF801109DF80000B3
:10C9D000A1E04FF0010A89F801A099F8000080BB9E
:10C9E000F6F705FA68B39DF8005089F800A0FAF749
:10C9F00031FE012808BF002515F0040F18BFFCF711
:10CA0000FAFB15F0020F06D01F20FBF749FDF9F7DE
:10CA100067F945F0010515F0010F10D0FAF71AFE7D
:10CA2000022802D106F002F848B1FAF713FE0528F1
:10CA300002D101F06AF910B10020F9F73DF989F847
:10CA4000006089F8016000F060B99DF80000401EA8
:10CA500001F086FCA8E79DF8000006F0B2F8A3E715
:10CA60009DF8000010F00F0018BF01200DF03BFAF8
:10CA700000F04BB99DF800000DF02BFA00F045B91D
:10CA8000D485001044AB0010BDE6000040860010C5
:10CA90009DF8000006F0A9F800F037B99DF80000F5
:10CAA00010B1012808D030E1002010F005FD002071
:10CAB00010F09DF8002006E0012010F0FDFC03209E
:10CAC00010F095F8012010F0C0F81EE19DF800006C
:10CAD000F8B1FAF7BFFD022818BF012406F056F896
:10CAE00001460220FAF7D1FD0FE10AE102E1FCE084
:10CAF000CAE0C4E0D5E071E0CBE009E127E021E045
:10CB00001BE00BE099E08AE083E06AE05BE030E064
:10CB100041E000210620FAF7B8FD45E79DF8000046
:10CB2000002818BF012006F01AF89DF80000002820
:10CB300018BF012001F0D4F8E7E09DF8000005F0EF
:10CB4000FAFFE2E0BDF8000006F0CDF82CE79DF812
:10CB5000000020B1012840D0022805D0D5E04FF4D4
:10CB60007F30F7F78BF9D0E001F062FE002104205E
:10CB7000D1E7F7F7E7FD00F008040820F7F7DDFD3F
:10CB800099F80300002808BF89F802602046F7F7EB
:10CB9000CFFD0121BEE79DF80000062805D2DFE8A1
:10CBA00000F004070A0C030FB3E702210846B2E7BE
:10CBB00002210520AFE7002103E000210420AAE7BD
:10CBC00004210320A7E79DF80300009A002360F3E7
:10CBD0001F626221072004F0ADFE96E0F9F784FBA6
:10CBE000E2E69DF800009DF80110000140EA1110F6
:10CBF0000BF04EFE9DF801109DF8020001F00F01B0
:10CC000040EA01200BF04AFE9DF803000BF052FEB3
:10CC100032E0BDF8000040BA0BF027FE75E09DF849
:10CC200000000BF05FFE9DF801000BF06EFEBDF8FA
:10CC3000020040BA0BF07CFE67E09DF800000BF0AC
:10CC40008CFE9DF801009DF80210000140EA1110D1
:10CC50000BF095FE9DF802109DF8030001F00F0106
:10CC600040EA01200BF07FFE9DF804000BF093FEDC
:10CC70009DF805000BF095FE0BF09FFE45E09DF83A
:10CC8000000006F0D8F88FE69DF8000006F0DBF80B
:10CC90008AE69DF80000002818BF0120FAF7D0FDB1
:10CCA00082E60DF028FD9DF8004006F095F8012C75
:10CCB00013D0022C14D0042C18BF082C7FF474AEAF
:10CCC00040F0005005F0C5FF042C18BF082C7FF47D
:10CCD0006BAE20460DF00AFD66E605F0BAFFF8E7F8
:10CCE00040F0805005F0B5FFF3E79DF8000010F02C
:10CCF00076FD0AE09DF800000DF0EFFC05F0CCFE9B
:10CD000003E09DF8000000F06FF934B1012742E024
:10CD10009DF8000006F064FF46E6D9F808006D466D
:10CD20004FF0FF3440B1D9F8082000230121084614
:10CD300004F000FEC9F80860F7F704FD00F0080AE7
:10CD40000820F7F7FAFC99F80300F0B199F805000C
:10CD50000BEBC001401CC0B289F80500202828BF99
:10CD600089F8056099F80300401E89F803004C78A3
:10CD700091F800800020002C05DD0A1892782A54D2
:10CD8000401C8442F9DC0E704E705046F7F7D0FC20
:10CD9000002CBFF6C7ADF7F7D5FC00F0080408205B
:10CDA000F7F7CBFC99F80310002908BF89F8026057
:10CDB0002046F7F7BDFC002F14BF0120002003B070
:10CDC000BDE8F08F02460020022928BF704752B10B
:10CDD000012A18BF704701EB4100C0EB4110FE492A
:10CDE00001EB8000704740F2DB104843FB49F7E756
:10CDF00070B5F7F7A7FC00F008060820F7F79DFCD0
:10CE0000F74C00256078FF2806D240F6D861F34839
:10CE100013F0C3F8E5702571E079FF2805D2E82109
:10CE2000ED4813F0BAF8257265723046BDE87040DF
:10CE3000F7F77EBCDFF8ACC300FB01F31CEB030C7F
:10CE400088BF7047E64B1A62C3E906017047DFF8F6
:10CE500090C30028DCF8183018BF0360E0480029B0
:10CE6000C06918BF0860002A1CBFDCF820101160E0
:10CE700058437047DA4801214171007840F2DB11D4
:10CE800080F001004843D54901EB80007047D44849
:10CE9000C278002132B1027922B9027882F001020F
:10CEA0000270C17041717047CD491E284A784870A0
:10CEB00008BF002003D01F2808BF012000D1087040
:10CEC00010467047C648007840F2DB1180F0010040
:10CED0004843C24901EB800070472DE9F007C04F7D
:10CEE00097F800C040F2DB140CFB04FCBB4CBE699D
:10CEF00004EB8C0C03FB06F40CEB440C8E4234BFA9
:10CF000035460D46FC69E31A934238BF1A46BB7892
:10CF1000012B16BF052B6C0800244FF00008002AD7
:10CF20009CBFBDE8F00770472346AC420FD297F88C
:10CF30000290B9F1050F30F8139006BFA3EB040A75
:10CF40002CF81A902CF813905B1CAB42EFD308F12D
:10CF500001080CEB460C00EB41009045E4D3BDE822
:10CF6000F00770472DE9F0419D4F14468C4601466D
:10CF70007A7806981D468A4218BFBDE8F0810121E3
:10CF80003971012802D0022824D029E0387840F2F3
:10CF9000DB1148439149BE6901EB8001A64234BFD1
:10CFA00032462246F869A84238BF05460023002DC4
:10CFB00016D90020002A06D91CF8007021F810703C
:10CFC000401C8242F8D85B1C01EB4601A444AB42F2
:10CFD000EFD305E000232A4621466046FFF77DFF98
:10CFE000BDE8F04100F0C7BC7D4A01281146D0726F
:10CFF000497808BF242004D0002806BF2429FF2038
:10D000007047507070477648C07A704770B4DFF848
:10D01000D8C1DCF800C0DCF818C01CF0040F1ABF3F
:10D02000012424EA0C060CF0010605680C68002EA9
:10D030001CBF1B1B5C1E1CF0020F1CBF521B551E8D
:10D040001CF0040F19BF04600D6005600C6070BC1B
:10D050007047002808BF70476149644B4A786449AB
:10D060001B78002A097818BF022A05D0042A18BFA5
:10D07000092A01D0012230E75E4A1278012A84BFD2
:10D080005D4A1378012200F090BC2DE9F041544C28
:10D090000F4601212171594A1578544A167828B152
:10D0A000A170002332462946FFF717FF3FB1052044
:10D0B000A0700023324629463846FFF70EFF00F0E5
:10D0C0005AFCFF20A070BDE8F0812DE9F04FDFF899
:10D0D00010918BB0012189F804104849454C464E07
:10D0E0000D784249DFF8F4B00F7899F80110112952
:10D0F00033D00CDC042920D004DC002918BF02291D
:10D1000011D11AE0092918D0102926D00BE02129C5
:10D110007AD004DC122918BF132904D11DE022297A
:10D1200072D0242971D0002800F0308100233A46C3
:10D130002946FFF7D2FE00F029B92178012902D94A
:10D140002F4937780D78002800F0208100233A46D7
:10D15000294600F02AFC00F019B9F5F736FDF5F77D
:10D160003BFC0090002818BFF5F7D1FE207801287D
:10D1700088BF3778F5F748FE10F0020F18BF7F1C04
:10D18000DFF8808099F8016099F8000040F2DB1127
:10D190004143D9F818000BEB8104A84238BF05467B
:10D1A000D9F81C00B84238BF0746F5F75DFF01907B
:10D1B0000020F6F7B1FB4FF0000A002F4EDD4FF0D4
:10D1C0000009002DC4BF0AEB4A0000EB0A1B3DDD3D
:10D1D000019810F9090019E01CBB001044AC0010C4
:10D1E000E48500104AFCFFFFC88600105E85001031
:10D1F000648500105F850010618500105D8500105A
:10D2000060850010000001303BE042E0262824BF8A
:10D21000002024F8190015D200F0010108EB81313B
:10D2200000EBD07001EB8B014010102E51F8200064
:10D230001AD0112E1FD0122E0CBFC0B2F6F772FBFF
:10D2400024F8190009F10109A945C1DBFE480AF1DA
:10D25000010ABA45806904EB4004B0DB009800285D
:10D2600018BFF5F757FE91E010F4003FC0F34230CD
:10D27000E6D04042E4E710F4803FC0F30420F8D148
:10D28000DEE700287ED00023BA1C2946FFF725FEE2
:10D290007CE000287AD00646EC480068007E10F05A
:10D2A000040F07BF2C46BA463C46AA46A1084FEADF
:10D2B0009A020592A4EB9400069200916208401E27
:10D2C000CDE901020391AAEB9A0104904FEA5A02B8
:10D2D000491ECDE9072109915346224605A9684612
:10D2E000FFF794FE5346224605AF06A9E84601A87B
:10D2F000FFF78CFE5346224607F1080108F10800AB
:10D30000FFF784FE5346224607F10C0108F10C009A
:10D31000FFF77CFE5346224607F1100108F110008A
:10D32000FFF774FE99F8000040F2DB114143002240
:10D330000BEB8100914620F8129058F82210A1F1D1
:10D34000010C491C61451CD357F822104B1E491C87
:10D3500099420FD303FB05C136F9114030F9121081
:10D360008C42C8BF20F8124057F822105B1C491CA1
:10D370009942EFD258F822100CF1010C491C61457A
:10D38000E2D200E002E0521C052AD4D30BB0BDE883
:10D39000F04F00F0F0BAAC4801218172807980F042
:10D3A000010000EB4001C1EB4010A94901EB8000F6
:10D3B0007047A548027A002132B1427A22B98279B7
:10D3C00082F0010282710172817270479E491E28AB
:10D3D000CA79C87108BF002003D01F2808BF0120E8
:10D3E00000D18871104670479748807980F001001D
:10D3F00000EB4001C1EB4010954901EB8000704704
:10D400002DE9F04F9349DFF8408285B00F789249BB
:10D410000E78012188F8091098F807108C4C4FF00D
:10D420000009102918BF11293AD0122918BF132951
:10D4300036D0F0B198F8061001EB4102C2EB411171
:10D4400004EB8102002116EB070C18BF7F4C10D0B3
:10D450002368002E5B8A03BF30F811500B4422F87A
:10D46000135030F8113018BF22F81130491C8C4588
:10D47000EED8F7F767F900F008040820F7F75DF930
:10D4800098F80A0000281CBF012188F808107CD0F9
:10D490002046F7F74DF988F8099005B0BDE8F08F00
:10D4A000F5F793FBF5F798FA0290002818BFF5F707
:10D4B0002EFD98F80750D8F82400009098F8060040
:10D4C00000EB4001C1EB401004EB800BF4F710FBC4
:10D4D00000286AD01120F3F70CFB00280CBF1220A3
:10D4E000112060F3070A0120F3F703FB002814BFA3
:10D4F0000120022060F30F2A0AF0FF000190F6F7E6
:10D500000BFAF5F7AFFD00240390002E1FD9039806
:10D510000257142AA8BF143A02DA0A2AA8BF123204
:10D52000262A28BF2BF814900ED2DDE90010F5F75B
:10D53000D5F8102D4AD0112D4FD0122D0CBFC0B2EE
:10D54000F6F7F0F92BF81400641CB442DFD30BEBB0
:10D550004606CAF3072B5846F6F7DEF9F5F784FDC1
:10D5600000248246002F1AD91AF90420262A28BF3F
:10D5700026F8149010D258460099F5F7AFF8102D00
:10D5800031D0112D36D0122D00E039E00CBFC0B2E1
:10D59000F6F7C8F926F81400641CBC42E4D30298DC
:10D5A000002818BFF5F7B6FC63E70120F3F7A1FAEE
:10D5B000002814BF0120022060F3070A1120F3F7AE
:10D5C00098FA002814BF1120122093E710F4003FAE
:10D5D000C0F34230B6D04042B4E710F4803FC0F30D
:10D5E0000420F8D1AEE710F4003FC0F34230D1D0B0
:10D5F0004042CFE710F4803FC0F30420F8D1C9E7E0
:10D6000098F8060080F0010088F8060088F8089075
:10D610003EE770B50D460C4901220A710F4A497860
:10D6200016780F4A212914781EBF2229232970BD9C
:10D63000002818BF002D20D0002322463146FFF7D6
:10D640004CFC631C01220DE0E4850010C88600102C
:10D650001CBB001062850010638500105D85001002
:10D660005E85001021462846FFF737FC05EB440095
:10D67000A31C01223146FFF730FCBDE8704000F0EA
:10D680007AB970B50446C068EA4D68B1697859B98D
:10D69000E949097801298CBFE849E9490B78E9494A
:10D6A0000122097800F081F9A06820B16978002989
:10D6B00008BFFFF70AFD6878102804BF0020FFF7B5
:10D6C00004FD6878112804BF0020FFF7FEFC68788D
:10D6D000122804BF0020FFF7F8FC6878132804BF65
:10D6E0000020FFF7F2FC206920B1E979002908BF8A
:10D6F000FFF786FEE879102804BF0020FFF780FEC0
:10D70000E879112804BF0020FFF77AFEE879122893
:10D7100004BF0020FFF774FEE879132818BF70BD1E
:10D720000020BDE870406BE62DE9F74F8046C64803
:10D730000D46002690F800A0C148BE49344690F836
:10D740000090BAFBF5F000FB09F701200871487B57
:10D750000978DFF8F8B288420ED0B64A40F2DB1101
:10D7600048430BEB8001107840F2DB1250430BEB87
:10D770008000920012F01BFC0298002888BFDFF89E
:10D78000B4B22DD99BF80EC00022BCFBF9F009FB06
:10D7900010C101FB0AF100FB0510002D12D938F869
:10D7A00014309BF8001040F2DB1E01FB0EFEA7496F
:10D7B000641C01EB8E0100EB020E521C21F81E309E
:10D7C0009542ECD80CF10100C0B28BF80E00B842C3
:10D7D00024BF00208BF80E00761C02988642D1D31D
:10D7E0009449887B401EC0B2887387429CBF781ED4
:10D7F00088730878487303B0BDE8F04F00F0BBB8F9
:10D80000934A30B41268B2F810C0538A0022BCF1B7
:10D81000000F07D99C1830F8144021F81240521C10
:10D820009445F7D80022002B9CBF30BC70479C1A4F
:10D8300044BF30BC704700EB44040CEB020534F8E5
:10D84000024C521C21F815409A42F0D330BC70476C
:10D850007848017800F1280281F0010132F81110B6
:10D86000002918BF7047017881F001010170002183
:10D870000182037822F81310764A00781154704719
:10D880006C49087370476B48007B704770B5694CF2
:10D890000025257025732582658240F6D8616B4886
:10D8A00012F07BFBA562A58270BD62490878002258
:10D8B0004A8280F001001431095C69B140F2DB1149
:10D8C000624A414332F82110A1F55062B63A02BFD4
:10D8D000614931F81000704700207047554B1878A7
:10D8E00003F1140C80F001014FF6FF701CF80120C9
:10D8F000012A18BF704740F2DB104843534A02EB3D
:10D9000080005A8A30F81200521C5A82524B33F867
:10D910001120521E1204120C23F8112004BF002201
:10D920000CF8012070474C49A1F12802137801EB53
:10D9300043010B8803440B8092F800C0012102F1DF
:10D94000140303F80C10118A084410827047394AF6
:10D95000138A03EB5000414B01445B1824BF0020A5
:10D960007047117840F2DB125143384A02EB8101D3
:10D9700001EB4000704770B5F6F7E4FE00F00806D2
:10D980000820F6F7DAFE2B4C60790025002801BF4D
:10D99000207880F001002070E5701CBF0120E0704D
:10D9A0003046F6F7C5FE257170BD2DE9F047994662
:10D9B00016460D460446F5F75CFB5FEA000C1CD0EA
:10D9C0001C49087840F2DB125043204AD1F81880F5
:10D9D00002EB800009FB08F200EB4200454594BFD2
:10D9E0002F464746C969A1EB0901B14238BF0E462F
:10D9F0000021002E09D8BDE8F0874B463246294663
:10DA00002046BDE8F047FFF768BA0023002F08D989
:10DA10001CF9032034F8122020F813205B1C9F42CD
:10DA2000F6D8491C00EB480004EB4504B142ECD3A6
:10DA3000BDE8F087E48500105F8500106185001067
:10DA40005E850010648500105D85001044AC0010F8
:10DA5000C8860010F88500100C8600104AFCFFFFF5
:10DA60003949002814BF002001200870704736484B
:10DA7000007800280CBF01200020704701203249A7
:10DA800048707047304800214170017800291ABF62
:10DA90004068002870472D48016821F001010160AD
:10DAA00070472948017821B128490A6842F00102EB
:10DAB0000A60002141608160C160016170472248B5
:10DAC000017821B121490A6842F001020A6000216F
:10DAD00041608160C1600161704700B501784278A2
:10DAE00083B0890141EA82018DF80010418809095B
:10DAF0008DF80110818809098DF80210817801F0F4
:10DB00000F02017962F31F118DF80310017A8DF86D
:10DB10000410417A8DF805108179C27901F03F0136
:10DB200002F00C0241EA02118DF80610C179807AE8
:10DB3000890100F0010041EA40108DF807006846B5
:10DB400012F09EFA03B000BD10860010144C004085
:10DB5000002818BF33483449886370473248806BC7
:10DB6000304988420CBF0120002070472E48704782
:10DB70002E4B4FF0000C1C681B1F1D682A4B1960B0
:10DB80005A602B49D963DC6214F0804F22D0290CF3
:10DB90005985290A83F8291083F82850598D19B11D
:10DBA000598D012242EA014C93F8291039B193F8BA
:10DBB0002910022242EA014C1E490C681C6393F8AA
:10DBC000281039B193F82810032242EA014C1A496F
:10DBD0000C685C6319490C60091DC1F800C0184A43
:10DBE00081691160B0E816109960DA601C61C3F8B1
:10DBF00014C090E807109861D9611A62C3F824C074
:10DC0000986B0849884202D10F490E480860FEE728
:10DC10000E49012804BF09607047022818BF7047E9
:10DC200008470000504D5544005F01102CED00E006
:10DC3000544C414638ED00E034ED00E0344C0040F7
:10DC40003C4C0040AD2007B0304C0040ADDEADDEB6
:10DC500070B50E460446F9F7FDFC042811D1A4F571
:10DC6000C87070280DD2A019A0F29110702808D2A7
:10DC700065020024002E04D92846F6F7FFF8012893
:10DC800001D0002070BD641C05F50075B442F3D3CB
:10DC9000012070BD70B50D460446F9F7DBFC042881
:10DCA0000AD1A4F5C870702806D260022946F6F79A
:10DCB00087F9012808BF70BD002070BD10B5074C62
:10DCC000FEF7D4FD012808BF10BD206800F060FEFB
:10DCD000002818BFF9F720FDF2E70000C886001001
:10DCE000FE4A0028516814BF41F0010021F00100F4
:10DCF00050607047F94B59680A0E120721F07F41B6
:10DD000042EA0060084358607047F4484068C0F336
:10DD100003607047F1484068000F7047EF483221B8
:10DD2000C0684843EE49A1FB001080087047EB48EB
:10DD300000697047E948006A7047E84901200862B5
:10DD40007047E649002008627047E4480078704751
:10DD5000002818BF0120E14908707047DF48406A79
:10DD60007047DE4800214162017070472DE9F041A3
:10DD700084B000270FF049FD0646A021D94812F0D3
:10DD800084F9002425464FF00308305D10F0800F21
:10DD900019D0601C8DF801008DF807508DF80080B7
:10DDA000ADF804508DF80850ADF802508DF80650CB
:10DDB0008DF809508DF80E5035550127002269461F
:10DDC000C848F2F729FC601CC4B20A2CDDD3C64C4B
:10DDD000E07A68B1012F0BD10021C248F2F7A8FA0E
:10DDE000E07C28B100231A4603210420F2F797FAB9
:10DDF00004B0BDE8F0410FF084BB2DE9F04186B0DE
:10DE000040F20F31F9F7AEFD002804BF06B0BDE8BF
:10DE1000F08112F03FF912F042F9F7F7F6FD5FEAF0
:10DE2000000872D1F3F774FBB048F4F720FE01202C
:10DE3000F4F710FEF6F7A8FCAD48F6F75AFDF6F732
:10DE400041FDF6F76AFDAB4E4000A44D3168B1F8D4
:10DE5000FA20B0FBF2F0401CC0F34F00688091F84C
:10DE6000FC1011F0FF0169700AD0F6F756FD316819
:10DE70004000B1F8F810B0FBF1F0401CC0F34F00C7
:10DE8000F6F7BBFC9C4F17203860306890F80A0109
:10DE9000A860F4F79AFEF4F79FFD002808BFF5F795
:10DEA0001AF8687838B1401E10F0FF00687004BF9F
:10DEB0006888F6F7A2FC6868C0F303642146052071
:10DEC000F2F70FFAFEF7D2FC012807D06868C0F31A
:10DED0000360A04208BFB8F1000F1FD0F5F70DFB9B
:10DEE00000203860F6F7D9FC40B1F6F7BEFCF6F733
:10DEF000F4FC0020F6F7FDFCF6F753FCF4F765FEA2
:10DF0000F4F76CFD0020F4F7B2FD12F0C8F812F03F
:10DF1000CBF8F9F79BFE06B0BDE8F0816846F5F74F
:10DF2000A4FA98B16846FFF7ACFBF9F793FB2146DA
:10DF3000009A07F0B3FF684612F0BBF8804608F07D
:10DF400023F8F5F7DAFAF9F7FDFBBBE73068D0F80C
:10DF50009C0010F0704F02D0F9F7DEFBB2E7F9F742
:10DF6000F8FBAFE770B50546002404F063FE70B11E
:10DF70000CF0C1FB08280AD0604800EB0510C1680E
:10DF80005648C26A91421CBF012101630124204608
:10DF900070BD5A4A014602EB01110020CA684F4980
:10DFA000CB6A9A4208BF70470120086370472DE989
:10DFB000F05FDFF840B1DBF80000B0F90211B0F912
:10DFC000000112F044F8F2F745FC0120F7F775FD67
:10DFD00000200CF099FB0FF0EFFB042000F0C4F8D8
:10DFE000F7F750FD002004F084FF0AF091FDDFF800
:10DFF000EC9000240120C9F81040C9F81440C9E988
:10E00000064012F05BF80020C9F80C40F8F737FE24
:10E01000F9F720FB052808BFDFF8E0A070D1D9F898
:10E020000400010FC0F30367B94206D00020C9F80D
:10E030001000C9F81400C9F81800DBF80000B90096
:10E040000024D0F8EC00A04620FA01F101F00F0501
:10E05000C0F30320854204BF0020C9F830002AD154
:10E06000DBF80000D0F8EC100AEB04100279920003
:10E07000D14001F00F060F2E04D08168204688475A
:10E08000012807D0641C022CEAD3D9F830000128FB
:10E090000BD102E03546A046F7E70AEB0810C0684E
:10E0A000C9F82C000020F7F708FDD9F82800A8428D
:10E0B00018BFC9F828503946052003F0FBFCE7B328
:10E0C000022F45D0042F4BD0D9F804000A2F4FEA75
:10E0D000106120F07F404FEA017112E024860010A9
:10E0E000ABAAAAAA34890010208900100B440010A2
:10E0F0004D3C0010C88600101048004058860010A3
:10E100000EE018BF41F000710843C9F80400FEF7A3
:10E11000ADFB012804D0F9F79DFA05283FF47FAF45
:10E120000FF0EFF9F7F7C8FC0FF04DFB33484168EB
:10E1300021F400714160002000E00DE0F8F7DCFC04
:10E140000020F8F780FDBDE8F05F0020F2F755B938
:10E150002846FFF752FEDAE7284611F0B4FFD6E76B
:10E16000284604F0AFFFD2E72DE9F047DFF890A092
:10E1700001468900DAF8000000242746D0F8EC00B8
:10E1800020FA01F101F00F05C0F30320854231D1DF
:10E19000DFF87090002009F13408C9F83000DAF88F
:10E1A0000000D0F8EC1008EB041002799200D14086
:10E1B00001F00F060F2E04D0816820468847012801
:10E1C00007D0641C022CEAD3D9F8300001280BD107
:10E1D00002E035462746F7E708EB0710C068C9F8A4
:10E1E0002C000020F7F769FCD9F82800A84218BFD6
:10E1F000C9F828502846BDE8F0870000001000400C
:10E20000C8860010248600107047002808BF704799
:10E2100080220146014811F0BBBE704704C40010C3
:10E22000704705283CBFFE49087070470020FC4934
:10E2300088604860FB48006890F8B900052838BF3E
:10E24000087070470020F64948607047F44800782D
:10E25000704770B5F34D0024286890F8A40010F0C2
:10E26000020F0BD0F9F7F6F9022807D1EC4829681C
:10E27000007801EB8000B0F8BC0084B2204670BD8D
:10E2800070B5E84D4FF48054286890F8A40010F061
:10E29000020F0DD0F9F7DEF9022809D1E04829680C
:10E2A000007801EB8000D0F8BC00000CC0F3130430
:10E2B000204670BDDA488078002818BF01207047DA
:10E2C0002DE9F041F9F7C6F9022803D104F0AEFBBD
:10E2D000022803D04FF48050BDE8F0814FF4805500
:10E2E0002E4604F06BFCDFF83C830446CC4FD8F894
:10E2F000000090F8A41011F0010F0CD0B0F8AE009F
:10E30000B9684042814206DC2CB10020641EB8602E
:10E31000204604F056FCD8F8001091F8A40010F044
:10E32000040F18BF002C0AD0B1F8B400621E904050
:10E33000B1F8B620824238BF1046C0F31306D1F8B8
:10E34000DC0010F0020F1CBFB978002902D0000CCD
:10E35000C0F31305B54298BF35462846BDE8F081A5
:10E360002DE9F04FDFF8BCA287B0DAF8001091F881
:10E37000A42012F0020F0DD0A94A91F8B890DFF84E
:10E38000A8B21778002809DB484503D2B84218BF65
:10E39000064643D107B00020BDE8F08F3E464FF05F
:10E3A000FF38F4F71BFBF5F736FB0025B9F1000F3A
:10E3B00034D9DAF80000002400EB8500B0F8BC0086
:10E3C00081B22046F3F7ABF9F4F785FD6846F5F71F
:10E3D0004CF8002866D0029878B1014693489BF823
:10E3E000002000785043421E07D331F9020B002869
:10E3F000B8BF40420444521EF7D2F5F77EF8F4F756
:10E40000EDFA002322469221072003F093FAA0455B
:10E4100084BF2E46A0466D1C4D45CAD3B74244D09A
:10E42000052E3CBF7E490E70DAF80000B0F8BA1035
:10E4300039B300EB870200EB8600B2F8BC20B0F8DD
:10E44000BC0092B280B2801A484340F30F34F6F712
:10E45000B5FF774B9BF80020002193F800C002FB2A
:10E460000CF2002A0DD930F81120224420F8112096
:10E470009BF8002093F800C0491C02FB0CF28A4272
:10E48000F1D84FF4800004F0E7FCDAF80000002334
:10E4900000EB86008021B0F8BC0082B2072003F0B8
:10E4A00049FA09E0F9F738F990E704F087FB032807
:10E4B0003CBF401C04F085FB012007B0BDE8F08F95
:10E4C000584857490068B0F8AE0042428868824216
:10E4D000BCBF401E886070472DE9F04F93B0934653
:10E4E0000E4604464FF0000A04F068FBDFF8348162
:10E4F0004B4F0500D14610D111F0EAFDD8F80010BD
:10E50000B1F8B010884208D30120C7F8089004F091
:10E5100058FB13B00120BDE8F08F002E1FDDB86856
:10E520000028B8BFC7F8089007DBD8F80010B1F88A
:10E53000AC108842BCBF401CB860D8F80000B96875
:10E54000B0F8AC00884215DC032D13D2681CC7F864
:10E55000089004F036FB13B00120BDE8F08F09D11C
:10E56000D8F80000B0F8AE004142B8688842C4BF95
:10E57000401EB860B87850B1D8F8000090F8DC00C0
:10E5800010F0040F1EBF002013B0BDE8F08FD8F8C4
:10E590000000B0F9AA108C420EDD79682144796040
:10E5A000B0F8A600884210DC4FF0FF30C7F80490A6
:10E5B000FFF7D6FE824608E07868002805DD002CCB
:10E5C000D4BF01212146401A7860DFF8689099F89D
:10E5D000000007283BD11848594600784200684699
:10E5E00011F0E5FCADF80040ADF80260ADF8045064
:10E5F0003889ADF80600B888ADF80800D8F80000F2
:10E60000B0F8AA10ADF80A10B0F8AC10ADF80C10C4
:10E61000B0F8A610ADF80E10B0F8AE000EE0000095
:10E62000B0860010C88600105D850010618500105E
:10E630005E850010E585001064850010ADF81000BF
:10E6400099F80000072804BF6846FEF702FD50460F
:10E6500013B0BDE8F08F474810B50068D0F8DC0073
:10E6600010F4807F06D0C0F30330012101FA00F0DE
:10E67000F5F786FD404900204870887010BD70B5E0
:10E680003D4D0024A878002814BF01260026687894
:10E6900028B904F0A2FA002808BF002100D0012107
:10E6A0008E4227D00A1C18BF0122AA703148006888
:10E6B000D0F8DC3013F0040F0ED021B1C3F30310F7
:10E6C000052808D206E00021A960696090F8B90029
:10E6D000052800D22870012413F0020F18BF01246E
:10E6E000002A18BF012200238221072003F022F90B
:10E6F000F1F727FE204670BD2DE9F0411D480027A7
:10E700000068D0F8DC1011F4807F30D01A4E707899
:10E71000051C18BF0125C1F30330184A52680123B4
:10E7200003FA00F0024011F4007F0AD092B10BF01E
:10E73000E2FF042818BF08280AD002200BF0D6FFF9
:10E7400006E03AB10BF0D7FF042818BF0828F4D12F
:10E75000012403E0002401200BF0C8FFA54206D0ED
:10E76000201C18BF01207070FFF789FF074638464C
:10E77000BDE8F081C8860010B0860010001000408F
:10E780007148007870477048406800F540707047E5
:10E790006D48406800F58070704770B56A4C4FF462
:10E7A00050306A4A60600168914204BF4168B1F527
:10E7B0000C7F3BD18168B1F5264F37D8644AC568D4
:10E7C000954223D04FF0000C03466246BCEB910FFC
:10E7D0000AD253F8046B521C86EA0C0CB2EB910F70
:10E7E000F7D3BCF1000F21D1026A7AB14FF0000CCF
:10E7F00003466246BCEB910F06D253F8046B521CE1
:10E80000B444B2EB910FF8D365450FD1012500F563
:10E81000807000F0BDF848B1606800F5407000F00D
:10E82000C6F800281EBF2570012070BD002070BDF5
:10E830004549002008704FF45030F5F71FBB42489F
:10E84000017841B14068414A0168914202BF416884
:10E85000B1F50C7F7047002070473B4B5B6803F5B8
:10E8600080731844F5F700BC374B5B6803F54073C1
:10E870001844F5F7F9BB3448406800F580607047EC
:10E88000314B5B6803F580631844F5F7EDBB2E4808
:10E890004068006970472C4949680A6982429CBFF8
:10E8A0000020704700EB400001EB001000F5A06075
:10E8B0007047254A526802EB8000436A406E1A4452
:10E8C00000FB012070472049886070471E4880681F
:10E8D00070472DE9F0011C4B00220127D3E90146C6
:10E8E0009046831893F92030002B12DB07FA02FCC4
:10E8F0001CEA060F0DD002F0FF0C04EB8C0CDCF8C8
:10E900002450DCF864C0254403FB0C5341F822304A
:10E9100001E041F82280521C102AE2D3BDE8F00148
:10E9200070470029B8BF704730B49446064A526811
:10E9300002EB8000446A406E224401FB002030BCA0
:10E940001A466146F5F790BBBC86001054465053FA
:10E95000EFBEADDE10B5FFF720FFA8B1FFF713FF44
:10E960000146E422174811F013FBFFF711FF164C84
:10E9700001464FF4DE72206811F00AFB2068806BBC
:10E98000BDE8104004F09EB80220F8F72BFFE2E744
:10E9900058B10E4A0168914207D1406820F00F003B
:10E9A000B0F5247F04BF012070470020704730B1CC
:10E9B000006820F00F00702804BF0120704700207D
:10E9C0007047000044330110C88600104150535274
:10E9D000FE4948607047FD4880687047FB494870B1
:10E9E0007047FA48407870470200F9484FF0080134
:10E9F0000068438A008A03FB00101CBFC01C20F083
:10EA000003007047F0B40446481E02280FD80125C1
:10EA100005FA04F010F08C0F18BF002C07D0032C5F
:10EA200005D8EB4B4FF4483001221B6802E0F0BCE4
:10EA300000207047A24214D005FA02FC1CF08C0F93
:10EA40000CD05E8A1F8A4FF0080C06FB07CC0CF135
:10EA5000030C2CF0030C0CEB4C0C6044521C032AEE
:10EA6000E8D901228A4204BFF0BC70474FF0080C7D
:10EA70005C8A1D8A521C04FB05CC0CF1030C2CF0A3
:10EA8000030C6044032AEDD9F0BC70472DE9F04F28
:10EA90000E4690F821A090F8209000F15005ADF2BC
:10EAA0000C4D1746012411463046FFF7ABFF012EEF
:10EAB00008BFDFF820B308D0022E08BFDFF818B374
:10EAC00003D0032E08BFDFF814B34FF0000830B1B5
:10EAD0000168594504BF4068CDE9001001D0CDE977
:10EAE00000B8BF48022E01680CBFB1F98A00B1F925
:10EAF0003A0086460CBFB1F98820B1F93820934618
:10EB000000230AFB09FCBCF1000F0ED935F91310E4
:10EB10007145D8BF8B4505DC9142C8BF0A4681428A
:10EB2000B8BF08465B1C9C45F0D8104400EBD07081
:10EB300042100023BCF1000F88BFE94616D935F911
:10EB40001300801A00EBD07041107F29C8BF7F21CD
:10EB500005DC11F1800FB8BF6FF07F0100DA0024EF
:10EB600009EB03005B1C01729C45E8D88DF804405A
:10EB70009DF80500FF283CBF401C8DF80500ADF84E
:10EB800006206C4639463046FFF73CFF78B1904985
:10EB9000082209684B8A098A03FB01222146F5F7FE
:10EBA00063FA01280CBF4FF001084FF000084046FF
:10EBB0000DF20C4DBDE8F08F2DE9F0479846154653
:10EBC0000E468146F8F743FD401E022888BFBDE887
:10EBD000F0877E4F834C3878814588BFBDE8F08749
:10EBE0000CD287F800904FF00000B8704FF0FF0291
:10EBF0004FF014017B4811F0EEF919E097F802C0CC
:10EC0000BCF1050F28BFBDE8F087BCF1000F18BFAD
:10EC100000200DDD14F82010B14206D104EB800174
:10EC20004978A94208BFBDE8F087401C6045F1DB88
:10EC3000B87804EB800104F820604D70A1F80280E0
:10EC4000401CB870BDE8F0874B1E022B9CBF431ED2
:10EC5000032B32BF022A0020704701EBC10149019A
:10EC600000EB400001EB401002EB420100EB011011
:10EC700000F5403000F53A5070472DE9F04FA1B053
:10EC8000002416460D4607461E94FF223021684692
:10EC90001F9411F0A0F9DFF850A14FF47F30CDF8A8
:10ECA00000A00168880A424211EB822218BF401C72
:10ECB000404201EB8000C01C20F0030000F5005032
:10ECC0004A49428A437C52BA007C63F31F4242EABB
:10ECD000006001900888A1F1040840BAADF80A006C
:10ECE0003869039098F800008DF818004FF000097B
:10ECF0004A4631462846FFF7A7FF8446012231469F
:10ED00002846FFF7A1FF0122012D04D0022D18BFD4
:10ED1000032D45D08CE0BCF1000F2AD0DCF80010A8
:10ED2000514526D19CF808109CF809300B4440B19D
:10ED3000D0F800B0D34504D190F8089090F809A01D
:10ED4000D1444B4506D9ADF87820ADF87C109CF83D
:10ED5000090005E0ADF87840017AADF87C10407A02
:10ED6000ADF87E00BDF87C00BDF87E100844ADF81B
:10ED70007A00BDF87C00BDF87E109DF81830C0B256
:10ED80008DF80800C9B29A408DF8091012F00E0FE4
:10ED900019BF401C8DF80800481C8DF8090047E099
:10EDA000BCF1000F2AD0DCF80010514526D19CF8A8
:10EDB000081020B10368534508BF90F808904945F2
:10EDC00084BFADF87820ADF87A1011E0CC86001041
:10EDD000C88600104654525946544D3246544D335D
:10EDE000E886001098EA001046464853D086001086
:10EDF0009EBFADF87840007AADF87A00022D18BFBA
:10EE0000032D15D1387C10F0300004BF21B0BDE8CF
:10EE1000F08FBDF87A003146401C8DF80800284676
:10EE2000FFF7F0FD00280CBF204640798DF809005F
:10EE30001494159416946B461794189419941A9474
:10EE40001B94FD481C940DF1300AB0E806128AE8C4
:10EE5000061290E807100DF1400989E807109DF8A7
:10EE60001800112813D20CA951F82000B0F1FF3F6F
:10EE70000DD007EBC000D0E90A10CDE9041098F8D6
:10EE80000200EE49820003F11C0011F090F8BDF879
:10EE90007810EC46CAB231462846FFF7D5FE38B1A5
:10EEA00030226146F5F7E0F801280CBF0124002468
:10EEB000204621B0BDE8F08F01220021824012F0EF
:10EEC0008C0F10D001281CBF0228032804D007286B
:10EED00008BF4FF4907106E0D94808210068428AC3
:10EEE000008A02FB001108467047012300B500228A
:10EEF000834013F08C0F0FD001281CBF0228032879
:10EF000002D0072803D007E0FFF77CFD03E00022D2
:10EF10000120FFF799FE0246104600BD2DE9F041A1
:10EF200005460126F8F793FB8046401E022884BF61
:10EF30000020BDE8F081C34F786810F4807F18BFCF
:10EF400002240DD00120A04010F08C0F05D04246C5
:10EF500021462846FFF79AFD0646286978B90BE056
:10EF600010F4007F18BF0324ECD110F0070018BF85
:10EF70000124E7D1BDE8F0813878112805D2424656
:10EF800021462846FFF779FE06463046BDE8F08167
:10EF9000AC49C8607047AB4810B4C068002808BFCF
:10EFA0004FF47C30A84A016891421CD14168B1F508
:10EFB000007F18D3836800228446B3F5056F88BFAD
:10EFC0004FF405630021B1EB930F24BF10BC7047D1
:10EFD0005CF82140491C2244B1EB930FF8D3002A7E
:10EFE00004BF10BC7047002010BC704770B50022F1
:10EFF000C260D0F808C0012113460446BCF5056F75
:10F0000088BF4FF4056C0022B2EB9C0F06D254F877
:10F010002250521C2B44B2EB9C0FF8D35A42C260D0
:10F02000884A127912F0800F07D14FF47C304FF4E8
:10F0300005622146F5F718F8014601290CBF0120A9
:10F04000002070BDFF2270B50025044605614FF415
:10F050000061503010F0BFFFA584E584E562A56231
:10F0600065632563E563A56365642564E564012044
:10F07000A56470BD2DE9F0414FF47C310446724E19
:10F080000868B04218D14868B0F5007F14D38A6888
:10F0900000230D46B2F5056F94BF94464FF4056CFE
:10F0A0000020B0EB9C0F26D255F82070401C3B444A
:10F0B000B0EB9C0FF8D3F3B1FF224FF4056120466B
:10F0C00010F089FF4FF40870C4E900604FF4056048
:10F0D000A0600020E06084F8200084F8210084F81B
:10F0E000220084F8230020616061A061E061204675
:10F0F000FFF7A8FF07E0B2F5056F88BF4FF4056280
:10F10000204610F045FF0120BDE8F08170B4026890
:10F110004FF408715160016801F1500291F821C06B
:10F1200091F820300CFB03F102EB41010022BCF10D
:10F13000000F08D900EB4204521CB4F8DE4021F85D
:10F14000024B9445F6D80022002B08D900EB42046C
:10F15000521CB4F8064121F8024B9342F6D8002223
:10F16000BCF1000F08D900EB4204521CB4F8644013
:10F1700021F8024B9445F6D80022002B08D900EB69
:10F180004204521CB4F88C4021F8024B9342F6D84A
:10F19000B0F8DA2021F8022BB0F8DC2021F8022B9D
:10F1A000B0F8D82021F8022B00240022BCF1000F77
:10F1B0000ED904EB440505EB041500EB850505EBC2
:10F1C0004206521CB6F8526121F8026B6245F6D332
:10F1D0000022002B0ED904EB440505EB041500EBCF
:10F1E000850505EB4206521CB6F8826221F8026BD7
:10F1F0009A42F6D3641C042CD7D370BC70472DE917
:10F20000F74F88B000250A992C462E4609680491CC
:10F2100001F150030999002984BF0C49D1F80080FD
:10F220002AD90022002888BFB8F93A701BD933F9CF
:10F23000021B00290CE00000F855020098EA0010BB
:10F24000C8860010CC86001053454C46E886001056
:10F25000B4BFC1F1000C8C46BC45BCBF0D44641C5E
:10F26000521C8242E3D30999761C8E42D9D3002CDA
:10F27000C8BF95FBF4FA08DC4908414301EB500292
:10F28000049901EB4201B1F950A0002102910191D2
:10F29000049950310091002103910999002969D9FD
:10F2A000F849009E069609684FF0000B4FF00109DF
:10F2B000B1F81CE091F824105F46D846CDF814B0A0
:10F2C0000791002829D9B6F900204FF0000C0699C3
:10F2D0009344634600280DD9B1F90040A51A48BFF0
:10F2E000151B7545B8BF0CF1010C01EB49015B1C06
:10F2F0008342F1D307998C4503D305997F1C1144B0
:10F30000059108F1010806EB49068045DBD3002F83
:10F31000C4BF059991FBF7F101DC9BFBF0F1039B66
:10F320000A9A09B202EB4302A2F86410D54A1268A5
:10F33000538BAAEB0303994209DD128B52448A4294
:10F3400005DD019A114401910299491C029100992D
:10F35000099A01EB400100910399491C03919142E4
:10F360009ED30299002905DDDDE9011291FBF2F13E
:10F37000019102E05146CDF804A00A9AA2F8DA10F1
:10F3800000210291039104995031009100210491D0
:10F39000002865D9BB49009F069709684FF0000B0C
:10F3A000099EB1F820E091F82510D846D946CDF84D
:10F3B00014B00791002E2BD9B7F900204FF0000CA4
:10F3C000069993446346002E0DD9B1F90040A51A61
:10F3D00048BF151B7545B8BF0CF1010C01EB40018E
:10F3E0005B1CB342F1D307998C4504D3059908F10E
:10F3F00001081144059109F1010907EB4007B145E6
:10F40000DAD3B8F1000FC4BF059991FBF8F101DC24
:10F410009BFBF6F1049B0A9A09B202EB4302A2F8A5
:10F420008C10984A1268538BAAEB0303994209DDAA
:10F43000128B52448A4205DD039A114403910299CA
:10F44000491C02910099891C00910499491C04915E
:10F4500081429FD302980028C4BF039991FBF0FA20
:10F460000A98A0F8DCA001980A99504400B200EB79
:10F47000D0704010A1F8D8000BB0BDE8F08F2DE996
:10F48000F74F8AB006460C980C99DFF8F8810768A8
:10F49000002008620C990546C8610C9988610C9996
:10F4A0004861711E0B980291411E0191002872D98A
:10F4B0000024002E6BD9E81705EBD06020F01F0167
:10F4C000691A012202FA01FB41110C9800EB810A32
:10F4D0000AF11C0905FB064007EB4000012DB0F9BD
:10F4E00050007DD0022D00F0CF80032D00F0DD8094
:10F4F000042D00F0EB80052D00F0F980012D70D077
:10F50000022D00F0C980032D00F0D780042D00F0FB
:10F51000E580052D00F0F38015B101998D4208D1E9
:10F52000002C19BF02998C42D8F80010B1F9A6102E
:10F5300003D0D8F80010B1F9A410002904BFD8F8FE
:10F540000010B1F9A41088421EDDDAF81C104FF04B
:10F55000010C41EA0B01C9F80010E11704EBD1637B
:10F560005A110C9923F01F0301EB820101F11402DF
:10F570004969E31A0CFA03F31943116083B2E2B24A
:10F58000E9B20720FFF718FB641CB442A2D30B9822
:10F590006D1C85428CD3D8F8000090F8C510002966
:10F5A0001CBF90F8C400002800F046820B9800258C
:10F5B000002840F24182801E0990B01E089000246D
:10F5C000002E40F23482A5F10108002108FB06104C
:10F5D00007EB40000790681C009000FB061001E05C
:10F5E0003FE046E007EB40000690E81705EBD060EF
:10F5F00020F01F01691A012202FA01F1059141115F
:10F600000C9800EB810004901C30039005FB064031
:10F6100007EB4009052DB9F9502079D8242C77DB68
:10F62000252C75DCB8F1040F98BF242C14BFB9F950
:10F630004E00B9F952008242CCBF11460146002962
:10F6400072D0111A6423594364D48242CCBF13464A
:10F6500003461944A1F1010100DD104691FBF0F3CE
:10F6600064E0242C04BFD8F80010B1F9AC103FF4CA
:10F6700064AF252C04BFD8F80010B1F9B6103FF4E0
:10F680005CAF4AE7E8860010242C04BFD8F80010CD
:10F69000B1F9AE103FF451AF252C04BFD8F80010DB
:10F6A000B1F9B8103FF449AF37E7242C04BFD8F8BC
:10F6B0000010B1F9B0103FF440AF252C04BFD8F8CA
:10F6C0000010B1F9BA103FF438AF26E7242C04BF7C
:10F6D000D8F80010B1F9B2103FF42FAF252C04BFB9
:10F6E000D8F80010B1F9BC103FF427AF15E7242C6F
:10F6F00004BFD8F80010B1F9B4103FF41EAF252CA8
:10F7000004BFD8F80010B1F9BE103FF416AF04E7FB
:10F7100022E009E08242CCBF13460346A1EB03017D
:10F7200001F101019ADD98E74FF0FF0355EA04006B
:10F7300000F00381112D08BF002C00F0FE80242C66
:10F7400000F00281252C00F00881242C73D0252C98
:10F7500000F0098100F009B9A4F12400012894BF48
:10F760004FF0060C4FF0000C0B98052DA0F1010A8C
:10F7700094BF2323731E00200146654508D0012D48
:10F780001ED008FB064107EB41010120B1F95010E2
:10F79000554531D0DDF824B05D4523D1002C14BF90
:10F7A0004FF0000B4FF0010BDDF808E074450CBF83
:10F7B0004FF0010E4FF0000E5BEA0E0B1CD111E072
:10F7C000002C14BF4FF0000B4FF0010BDDF808E0E8
:10F7D00074450CBF4FF0010E4FF0000E5BEA0E0BAC
:10F7E000D6D1CEE7DDF800B0401C0BFB064B07EB93
:10F7F0004B0BBBF950B059442CB1012C1CD0B9F9BA
:10F800004EB0401C59449C422CD0DDF820B05C45E1
:10F8100024D1002D14BF4FF0000B4FF0010BDDF889
:10F8200004E075450CBF4FF0010E4FF0000E5BEA8F
:10F830000E0B17D112E089E0002D14BF4FF0000B22
:10F840004FF0010BDDF804E075450CBF4FF0010EE1
:10F850004FF0000E5BEA0E0BD5D1D0E7B9F952900C
:10F86000401C4944654516D14CB1DDF80090401C60
:10F8700009FB064907EB4909B9F94E9049449C42F6
:10F8800009D0DDF80090401C09FB064907EB490947
:10F89000B9F952904944554512D13CB108FB06498B
:10F8A00007EB4909401CB9F94E9049449C4207D0E6
:10F8B00008FB064907EB4909401CB9F95290494435
:10F8C00074B9654518BF55450AD0DDF81C90801CF9
:10F8D000B9F952904944DDF81890B9F95290494469
:10F8E0009C4213D1654518BF55450FD008FB064310
:10F8F00007EB4303801CB3F94E301944009B03FB14
:10F90000064307EB4303B3F94E301944002818BFF0
:10F91000002A3FF409AF6423594391FBF0F002EB56
:10F92000C20101EB0211D0EB810059BF1044401E0F
:10F93000801A401C90FBF2F3F8E6FE48006890F94C
:10F94000C71090F9C60033E0012D14D0022D18BF66
:10F95000042D17D0032D1CD007E0022D18BF042D55
:10F9600009D0012D0ED0032D13D0CDB1112D08BF1C
:10F97000252C28D016E0EF48006890F9C91090F9BE
:10F98000C80015E0EB48006890F9CB1090F9CA0068
:10F990000EE0E848006890F9D11090F9D00007E037
:10F9A000252C09D0E348006890F9C51090F9C400EF
:10F9B00051EA000C14D10DE0DE48006890F9CD103A
:10F9C00090F9CC00F4E7DB48006890F9CF1090F98B
:10F9D000CE00EDE7D748006890F9C51090F9C40053
:10F9E0008B4201DC83421EDA04984FF0010CC1699E
:10F9F0000598014303980160E01704EBD0604311C0
:10FA00000C9920F01F0001EB830101F114034969F7
:10FA1000201A0CFA00F00843186093B2E2B2E9B27F
:10FA20000720FFF7C9F8641CB442FFF4EFAD0B9850
:10FA30006D1C8542FFF4C3AD0DB00120BDE8F08F11
:10FA40002DE9F04F146887B015460E468046A1F1A7
:10FA50002009202928BF4FF0FF3B05D24FF00100BD
:10FA600000FA06F0A0F1010B31BF0020012000FADE
:10FA700009F0401E0290B8F1200F3DBF012000FAAE
:10FA800008F0401E4FF0FF3038BF002207D3A8F126
:10FA900020024FF0010101FA02F1A1F10102C6F1C9
:10FAA000200A202E34BF20FA0AF100FA09F1B240F0
:10FAB0001143B040CDE90001206920F4FE602061CF
:10FAC0009D48406810F0010F79D010F4807F05D078
:10FAD0002A463146404601F04FFA8AE010F4007F92
:10FAE0002A463146404602D0FFF7C9FC81E001F0CA
:10FAF00023F90020A86107466861B8F1000F22D9F8
:10FB000005EB4700B0F98C000028B8BF404200B2B6
:10FB100088490968B1F93810814211DD7A0905EB8D
:10FB2000820C07F01F0301219940DCF8142083B2F6
:10FB30001143CCF81410FAB2FF210420FFF73CF86F
:10FB40007F1C4745DCD30027B8F1010F1CBFA8F18B
:10FB5000010003904DD005EB4700B0F98E30B0F9AD
:10FB60008C20991A48BFD11A09B2DFF8C8C1DCF855
:10FB700000C0BCF932C08C4537DAB5F9DC10B2EB05
:10FB8000010C48BFA1EB020C0FFA8CFC5A1A48BFBB
:10FB9000CA1A11B28C4513DB7A0905EB820107F012
:10FBA0001F0C01224B6902FA0CF21A434A61B0F8A9
:10FBB0008C30FAB2FF210420FEF7FEFF15E02BE0A7
:10FBC000791C4B0905EB830E01F01F0C0122DEF8B6
:10FBD000143002FA0CF21A43CEF81420B0F88E302A
:10FBE000CAB2FF210420FEF7E7FF03987F1C87427B
:10FBF000B1D36969E869B14008432063A969286AFB
:10FC0000B140084360636969202E34BF21FA0AF1CC
:10FC100001FA09F1084360634748007910F0040FC6
:10FC200000F0F581002028630746E862002E22D903
:10FC3000404905EB47000968B0F95201B1F95C2071
:10FC4000824203DCB1F95E10814211DA7A0905EBD8
:10FC5000820C07F01F0301219940DCF82C2083B2AD
:10FC60001143CCF82C10F9B2FF220220FEF7A4FFBA
:10FC70007F1CB742DCD30020A86207466862B8F157
:10FC8000000F22D92B4905EB47000968B0F9820221
:10FC9000B1F95C20824203DCB1F95E10814211DAD5
:10FCA0007A0905EB820C07F01F0301219940DCF86B
:10FCB000242083B21143CCF82410FAB2FF21022091
:10FCC000FEF77AFF7F1C4745DCD3002028640746F7
:10FCD000E863002E34D9174905EB47000968B0F9ED
:10FCE0009E01B1F960208242DCBFB1F962209042EE
:10FCF00010DD7A0905EB820C07F01F030121994002
:10FD0000DCF83C2083B21143CCF83C10FF22F9B25E
:10FD100001200BE0B1F96C208242DCBFB1F96E101A
:10FD2000884205DD83B2F9B2FF221020FEF744FFBE
:10FD30007F1C03E0E8860010CC860010B742CAD3CF
:10FD40000020A86307466863B8F1000F2FD905EBC0
:10FD50004700B0F9CE02FE490968B1F9602082423D
:10FD6000DCBFB1F96220904210DD7A0905EB820C0C
:10FD700007F01F0301219940DCF8342083B21143BE
:10FD8000CCF83410FF21FAB201200BE0B1F96C205D
:10FD90008242DCBFB1F96E10884205DD83B2FAB24F
:10FDA000FF211020FEF708FF7F1C4745CFD300201E
:10FDB0002865E864A86407466864002E22D9E449EF
:10FDC00005EB47000968B0F9EA01B1F96420824205
:10FDD00003DCB1F96610814211DA7A0905EB820C75
:10FDE00007F01F0301219940DCF84C2083B2114336
:10FDF000CCF84C10F9B2FF220320FEF7DDFE7F1C89
:10FE0000B742DCD30027B8F1000F22D9D04905EB67
:10FE100047000968B0F91A03B1F96420824203DC93
:10FE2000B1F96610814211DA7A0905EB820C07F00C
:10FE30001F0301219940DCF8442083B21143CCF820
:10FE40004410FAB2FF210320FEF7B6FE7F1C47459F
:10FE5000DCD3696AE86AB14040EA0107A763A96A8E
:10FE6000286BB1400843E063696A202E34BF21FA51
:10FE70000AF101FA09F141EA0000E0630590696BBB
:10FE8000E86B01FA06F140EA01022264A96B286CD2
:10FE900001FA06F140EA01006064696B34BF21FA9F
:10FEA0000AF101FA09F141EA000161646B6CE86C46
:10FEB00003FA06F340EA0300A0640390AB6C286DDC
:10FEC00003FA06F340EA0300E0646B6C34BF23FAE4
:10FED0000AF303FA09F343EA0000E0640690059888
:10FEE00032EA070521EA000C47EA0502256404927C
:10FEF00040EA0C0906EB0801C4F844C008BFBCF195
:10FF0000000F46D000231A461846002988BF4FF03C
:10FF100001083ED94FEA501A04EB8A0A00F01F0E7E
:10FF2000DAF840A008FA0EFE1AEA0E0F03D0864255
:10FF300094BF521C5B1C401C8142EBD8012B10D19A
:10FF400005EA0B003843A06302980CEA0003059809
:10FF50001843E06325EA0B00206402982CEA0000B5
:10FF60006064012A15D1206C009A00EA0203A26B9A
:10FF70001A43A263626C019BD4F83CC0134043EA6D
:10FF80000C03E363009B98432064019822EA00007D
:10FF90006064DDE903208243A264049840EA02051C
:10FFA000069820EA090049EA0007E06408BF002833
:10FFB00022D000231A461846002988BF4FF0010CB2
:10FFC00017D94FEA501804EB880800F01F09D8F839
:10FFD00048800CFA09F918EA090F03D0864294BF49
:10FFE000521C5B1C401C8142EBD8002B18BF002A1E
:10FFF00002D10020A064E0645648007910F0010F9F
:020000021000EC
:1000000005D0206BA8432063606BB8436063206B0E
:100010000099084203D1626B01990A4203D0216919
:1000200041F01001216110EA0B0F03D1616B0298BE
:10003000014203D0206940F020002061A06B0099AC
:10004000084203D1E26B01990A4203D0216941F0D1
:100050004001216110EA0B0F03D1E16B02980142CC
:1000600003D0206940F080002061206C0099084294
:1000700003D1626C01990A4203D0216941F4807175
:10008000216110EA0B0F03D1616C0298014203D089
:10009000206940F400702061A06C002804BFE06C6F
:1000A000002803D0206940F48060206107B001205F
:1000B000BDE8F08F2DE9F04FCBB017460D46044652
:1000C000F2F78CFC0120F0F714FD06461120F0F742
:1000D00010FD304314BF012002208DF8180014BF1A
:1000E000112012208DF81900F1F702FD38B19DF8AA
:1000F00018009DF819108DF818108DF819009DF84A
:100100001800F0F7F6FC002818BF284604909DF868
:100110001900F0F7EEFC002818BF20460590F2F712
:10012000A1FF0022002D88BF24A90BD98356142BD0
:10013000A8BF143B02DA0A2BA8BF12338B54521CFF
:10014000AA42F3D3F2F790FF0021002C04E0000054
:10015000E8860010CC86001088BF24AA07D9435C2B
:1001600002EB010C491C8CF826308C42F7D8F2F7D0
:100170004BFE0390FE480DF1180A007910F0200F95
:1001800055D007F1DE00009028300025E9460DF13A
:10019000100B01905BF825601AF80500F3F7BCFB23
:1001A0000024002E1AD905EB450000EB051024A908
:1001B00001EB400818F90420262A28BF002006D2A7
:1001C0001AF805000021F2F789FAF3F7ABFB59F8AA
:1001D000251021F81400641CB442EBD36D1C022DD1
:1001E000D8D3E44C26781D2E21D100210A460DF1EA
:1001F0001C085BF822500020002D88BF59F822C04F
:1002000007D93CF8103028F81130401C491C8542B1
:10021000F7D8521C022AECD31D2E08D14046FDF718
:10022000EFF820781D2804BF07A8FDF7E9F8D04DA6
:10023000287910F00C0F00F0B083039800F0F00064
:10024000F2F799FC9DF81800F1F755FA07909DF820
:100250001800F1F7BFFA002437901AF80400F2F7FB
:1002600085F944A941F824001AF80400F1F7EFFADF
:100270000EA941F824001AF80400F1F73CFC20A96B
:1002800041F824001AF80400F1F76DFC22A941F8A6
:1002900024001AF80400F0F76BFC46A918AA41F8EC
:1002A00024001CA81AA902EB840200EB840001EBD5
:1002B00084010092CDE9011016A800EB840314A874
:1002C00000EB840212A800EB84011AF80400F1F795
:1002D0002CFF1AF80400F2F75AF81EA941F824007E
:1002E0001AF80400F2F792F910A941F82400641CEE
:1002F000022CB2D3A04E3068B0F848109DF8180018
:10030000F1F70DFA002400211AF80400F2F714F9AD
:10031000994E306890F84A101AF80400F1F7ABFAD9
:100320001AF804000021F1F700FC1AF8040000217B
:10033000F1F733FC1AF804000121F0F7FFFB3068F5
:10034000B0F84C101AF80400F1F7ABFF1AF80400EB
:100350000021F2F723F9641C022CD4D384484FF017
:100360000009007910F0040F00F0DE8134462068A7
:1003700090F84B3090F85920B0F850100091CDE92A
:10038000012390F84F3090F84E2090F858109DF8C7
:100390001800F1F70EFD206890F84B3090F85920C6
:1003A000B0F850100091CDE9012390F84F3090F84B
:1003B0004E2090F858109DF81900F1F7FAFC9DF8BE
:1003C00018000021F2F7EAF89DF819000021F2F771
:1003D000E5F83AADF2F77FFDFCF748FA012806D0C0
:1003E0002846F3F742F800287DD0F3F786F8F2F7B5
:1003F000F5FA3E99002204AD002055F82230002B7A
:100400000ED902EB420C0CEB021C07EB0C1C31F872
:10041000026B0CEB4008401CA8F852618342F6D8EE
:10042000521C022AE8D35548D0E90010CDE90C103F
:100430009DF81800F0F75DFB48909DF81900F0F763
:1004400058FB49909DF8180040A9F1F7B1FA9DF8C2
:10045000190042A9F1F7ACFA9DF8180008A9F1F7C4
:1004600019FB9DF819000AA9F1F714FB424C20680A
:1004700090F84B3090F85920B0F852100091CDE927
:10048000012390F84F3090F84E2090F858109DF8C6
:100490001800F1F78EFC206890F84B3090F8592046
:1004A000B0F852100091CDE9012390F84F3090F848
:1004B0004E2090F858109DF81900F1F77AFC9DF83D
:1004C00018000CA9F1F7C4FA9DF819000CA9F1F76E
:1004D000BFFA00249DF818000021F2F75FF89DF89C
:1004E0001900002100E017E0F2F758F89DF8180015
:1004F0000021F0F7E4FA9DF819000021F0F7DFFA87
:100500001AF804000121F0F7DAFA1AF80400C0F32F
:10051000011001280AD102E0F7F7FEF85CE784F049
:10052000010001211AF80000F0F7C9FACDF8E090B7
:10053000CDF8E4909DF8180038A9F1F719FA9DF864
:10054000190038A9F1F714FA04A8002150F8248002
:100550001AF80400F2F768F900250190B8F1000FCD
:1005600056D904EB440024A900EB041008E0000075
:10057000CC860010EB850010E8860010F0550200D4
:1005800001EB400107EB001B0091009838AA002105
:100590004657CDF8E090CDF8E4901AF80400F2F751
:1005A00060F8202E06DBA6F1200101208840CDE96D
:1005B000389003E00120B040CDE938091AF8040072
:1005C00038A9F1F7D5F9389838AAC0433890399846
:1005D0000921C04339901AF80400F2F742F83AAE04
:1005E000F2F779FCFCF742F9012806D03046F2F721
:1005F0003CFF00287ED0F2F780FFF2F7EFF9019878
:1006000000880BEB45016D1CA1F89E014545BCD34C
:10061000CDF8E090CDF8E4901AF8040038AA002153
:10062000F2F71FF8641C022CFFF454AF9DF8180079
:1006300008A9F1F70DFA9DF819000AA9F1F708FACF
:100640009DF818004899F0F73AFA9DF81900499971
:10065000F0F735FA9DF8180040A9F1F789F99DF8EF
:10066000190042A9F1F784F9FE4C206890F84B304C
:1006700090F85920B0F854100091CDE9012390F87A
:100680004F3090F84E2090F858109DF81800F1F770
:1006900090FB206890F84B3090F85920B0F8541037
:1006A0000091CDE9012390F84F3090F84E2090F85A
:1006B00058109DF81900F1F77CFB9DF818000121F6
:1006C000F1F76CFF9DF819000121F1F767FF3AACD3
:1006D000F2F701FCFCF7CAF8012806D02046F2F731
:1006E000C4FE00287DD0F2F708FFF2F777F9002268
:1006F00004AC00E081E03E9954F822C00020BCF137
:10070000000F0ED902EB420303EB021307EB0313B6
:1007100031F8025B03EB4006401CA6F8EA51844521
:10072000F6D8521C022AE7D3CF48007910F0080F00
:100730007ED0CC4C206890F84B3090F85920B0F81F
:1007400056100091CDE9012390F84F3090F84E20DB
:1007500090F858109DF81800F1F72BFB206890F8DE
:100760004B3090F85920B0F856100091CDE9012394
:1007700090F84F3090F84E2090F858109DF81900DE
:10078000F1F717FB00210DF1100C00205CF821207F
:10079000002A0CD901EB410303EB011307EB031310
:1007A00003EB4005401CA5F836928242F8D8491C5C
:1007B0000229EAD32068002590F86800B5EB400FC5
:1007C00036DA206890F86800A842D4BF01210021E1
:1007D0009DF81800F1F7E2FE206890F86800A84242
:1007E00000E00DE0D4BF012100219DF81900F1F7D0
:1007F000D5FE3AAEF2F76FFB05E0F6F78DFFF1E6B6
:10080000F6F78AFF66E7FCF731F8012805D0304695
:10081000F2F72BFED8B3F2F770FEF2F7DFF83E994D
:100820004FF0000904AB0022104653F8296000E0A5
:1008300058E0002E05D931F91030401C1A44864288
:10084000F9D8B2FBF6F2701E3DD009EB490303EB79
:10085000091307EB031B31F9103001EB400C3CF995
:10086000028CB3EB080348BF5B4231F91080B8EB50
:10087000020831F910804CBFA2EB0808A8EB02086F
:100880003CF902EC3CF902CCBEEB020E00E00FE0BA
:100890004CBFA2EB0C0CACEB020CE0450BEB400C9C
:1008A00009DDBCF936824345C8BFACF8363208E0F2
:1008B000F6F732FFA7E7BCF934829845B8BFACF829
:1008C0003432401EC7D109F1010901EB4601B9F1EB
:1008D000020FA7D320686D1C90F86800B5EB400F9D
:1008E000FFF66FAF9DF818000799F0F718FF9DF815
:1008F00018003799F0F77DFF00241CAD1EAE20AF25
:100900000DF188080DF588790DF58C7B59F82410C8
:100910001AF80400F1F710FE0EA850F824101AF887
:100920000400F0F7A8FF57F824101AF80400F1F7B4
:10093000FCF858F824101AF80400F1F72EF95BF8C7
:1009400024101AF80400F0F7F9F81AA918A851F8B9
:10095000241055F8242050F82400CDE9000116A8F1
:10096000029250F8243014A850F8242012A850F80D
:1009700024101AF80400F1F71CFA56F824101AF89B
:100980000400F1F78EFC10A850F824101AF80400A7
:10099000F1F704FE641C022CB8D30398F2F7EBF8CD
:1009A0004BB0BDE8F08F304801218160112101700A
:1009B00000218170FDF775B82B49002088607047D1
:1009C0002DE9F04FDFF8A0A0ADF56F7D01271120D4
:1009D000CAF808704FF000088AF800008AF8028010
:1009E000FDF75FF8DAF804004FF4407131EA0000D7
:1009F00008BF002600F07C811D20FCF755FAED9021
:100A00001D20FCF7E3FCEE904FF46D716846DAF8B8
:100A10000C400FF0C2FA0094BAF8040010F4804FB2
:100A20001CBF2046FEF70EFB6A46009890F8203067
:100A300090F821C050300CFB03F100EB4100002185
:100A4000BCF1000F08D902EB410630F8025B491CEB
:100A5000A6F8DE508C45F6D80021002B0DD930F8D1
:100A6000025B03E0E8860010CC86001002EB410632
:100A7000491CA6F806518B42F1D80021BCF1000FA9
:100A800008D902EB410630F8025B491CA6F8645015
:100A90008C45F6D80021002B08D902EB410630F82E
:100AA000025B491CA6F88C508B42F6D830F8021B2A
:100AB000A2F8DA1030F8021BA2F8DC1030F8021BA2
:100AC000A2F8D81000250021BCF1000F0ED905EBCB
:100AD000450606EB051602EB860606EB410B30F8E1
:100AE000029B491CABF852916145F6D30021002BC3
:100AF0000ED905EB450606EB051602EB860606EB5E
:100B0000410B30F8029B491CABF882929942F6D314
:100B10006D1C042DD7D361461846FEF770FBDAF83A
:100B200004003E4610F4004F03D1694600F041FD39
:100B30000646ED98FCF7B8F9EE98FCF747FC94F8F8
:100B4000209094F82150002E1CBFB9F1000F002D09
:100B500000F0CE809AF8040010F0020F04D06A462C
:100B60002946484600F0CCFB9AF8040010F0050F27
:100B700004D06A4629464846FEF762FF9AF8040008
:100B800010F0080F79D0009ADFF8E4E668461169A2
:100B900021F4C05111610021CDF86080CDF85C8056
:100BA000002D19D9DEF800C000EB4103B3F936324D
:100BB000BCF96AC09C450CDA4B0900EB830301F0D9
:100BC0001F0BD3F85CC007FA0BFB4CEA0B0CC3F805
:100BD0005CC0491CA942E5D3C0F858800021C0F888
:100BE0005480B9F1000F19D9DEF800C000EB4103C1
:100BF000B3F96633BCF96AC09C450CDA4B0900EBCB
:100C0000830301F01F0BD3F854C007FA0BFB4CEA27
:100C10000B0CC3F854C0491C4945E5D3916BC36D17
:100C20001943436DAB4019439163D16B036E194374
:100C3000836DAB400B43D363416D202D39BFC5F1AC
:100C4000200C21FA0CF1A5F1200C01FA0CF119434A
:100C5000D163416D002904BF816D002903D0116962
:100C600041F400611161C16D002904BF006E0028CC
:100C700003D0106940F4805010619AF8040010F01D
:100C8000400F0FD16069401C60612069002814BFCB
:100C9000E069A06900F1010014BFE061A06168464D
:100CA000FEF734FAC4F80C80A36800222146A4465B
:100CB000B3F5056F88BF4FF405630020B0EB930FC9
:100CC00006D25CF82070401C3A44B0EB930FF8D386
:100CD0005042C8609AF8040010F0800F05D14FF41C
:100CE0007C304FF40562F3F7BFF92046FEF716F9A2
:100CF00041208DF8B403BEB1207C8DF8B503607C33
:100D00008DF8B603A07C8DF8B703E07C8DF8B803AE
:100D100000230522EDA9072000F095FECAF80880FF
:100D20000DF56F7DBDE8F08FFF208DF8B5038DF8D0
:100D3000B6038DF8B703E9E72DE9F74F84B04FF01C
:100D4000000AC2F820A00646C2F81CA00598DFF8E9
:100D50002085174654464FF00109002821D907EB9A
:100D60004400B0F964000028B8BF404200B2D8F88F
:100D70000010B1F9381081420FDD610907EB8101E4
:100D800004F01F03CA6909FA03F31A43CA6183B264
:100D9000E1B2FF220420FDF70FFF0598641C844296
:100DA000DDD3002401281CBF0598451E46D007EB63
:100DB0004403B3F96620B3F96410501A48BF881A87
:100DC00000B2D8F800C0BCF930C0844533DAB7F9B6
:100DD000DA00B1EB000C48BFA0EB010C0FFA8CFC61
:100DE000111A48BF811A08B2844511DB600907EB6C
:100DF000800004F01F02C16909FA02F21143C161C7
:100E0000B3F86430E1B2FF220420FDF7D5FE12E012
:100E1000601C410907EB810100F01F0CCA6909FA47
:100E20000CFC42EA0C02CA61C1B2B3F86630FF2280
:100E30000420FDF7C1FE641CAC42B8D3D8F8000012
:100E400090F8361000297DD090F837003D68814237
:100E500088BF084600240599002984BF401C0090E3
:100E600070D94FF0010E00984FF000090121CA46D9
:100E7000012852D9FE4800680390B0F93A3004FBCB
:100E8000066002900EFB0660019004FB061005EB65
:100E90004000B0F950C0BCF1000FB4BFCCF100006D
:100EA0006046834239DB0EFB061005EB4000B0F9CB
:100EB00050000028B4BF4242024693422DDB029A02
:100EC000521A05EB4202B2F94E80B8F1000FB4BFDE
:100ED000C8F10002424693421FDB019A521A05EB09
:100EE0004202B2F94E20002AB4BFC2F1000B934671
:100EF0009B4512DCA0EB0C0C0398B0F93400604564
:100F0000B8BF09F10109A2EB08028242C8BF0AF189
:100F1000010A491C00988142B7D3BAEB090048BFC7
:100F2000A9EB0A00D249096891F83610884214DB0F
:100F3000600907EB800004F01F030121C26999409A
:100F4000114300E014E0C16107EB4400E1B2B0F8E6
:100F50006430FF220420FDF72FFE0598641C8442B4
:100F600006D2002C18BFA4F1010E7FF47CAF78E705
:100F700007B00120BDE8F08F2DE9F04F07464FF094
:100F8000000087B0D2F800801062D061906150619B
:100F9000DFF8E0B216465FEA010947F6FF7A0090F3
:100FA000019002900546039050D00024002F4AD9AA
:100FB000E81705EBD06020F01F01691A012202FA40
:100FC00001F1401106EB8000CDE905011C300490D1
:100FD000A74905FB0740096808EB4000B0F950003D
:100FE000B1F98A20B1F988105845C4BF8346CDE9CC
:100FF00002455045BCBF8246CDE90045904201DC28
:1010000088421DDA05994FF0010CCA6906990A4316
:1010100004990A60E11704EBD1614A1106EB8203DF
:1010200003F1140221F01F015B69611A0CFA01F14E
:101030001943116083B2E2B2E9B20620FDF7BCFDAC
:10104000641CBC42C4D36D1C4D45AED3884C206893
:10105000B0F88E0000281CBFABEB0A01814241DDD5
:1010600003980399400906EB800001F01F03C26951
:10107000012101FA03F31A43C2610198019A400960
:1010800006EB800002F01F02C36901FA02F21A4364
:10109000C2610298029A400906EB800002F01F022A
:1010A000436901FA02F21A4342610098009A40092A
:1010B00006EB800002F01F02436991401943416131
:1010C00002981FFA8BF3C2B20398C1B20620FDF753
:1010D00073FD00981FFA8AF3C2B20198C1B20620CC
:1010E000FDF76AFD6248006890F88C00002800F067
:1010F00003814FF0000BA9F1010A002F84BFA9F171
:101100000200049077D908EB4B000024B0F950009E
:10111000B9F1010F6BD04FEAEB710BEBD16121F00C
:101120001F02ABEB0202012303FA02F2491106EBA4
:101130008101CDE9021214310191611C009101FB82
:1011400007B108EB4101B1F95050002DC8BF00288C
:1011500049DD291A48BF411B8542CCBF2A460246B9
:101160004FF44843594391FBF2F101F2FF114A0A4F
:10117000002C1ABF04998C42BBF1000F3C4909684E
:1011800014BF91F88C1091F88D1019B9384909687D
:1011900091F88C108A4226DDE11704EBD1614A11E7
:1011A00006EB820221F01F0102F11C03A4EB010CEB
:1011B000D269012101FA0CF111431960029983B23D
:1011C00006204A6903990A4301990A600BF0FF025D
:1011D000E1B2FDF7F1FC0098ABB2C1B20BF0FF0237
:1011E0000620FDF7E9FC641C28465445A5D30BF105
:1011F000010BBB4587D30025B9F1000F84BF781ED2
:10120000039079D905FB07F008EB40000024B0F902
:101210005000012F6DD0E91705EBD16121F01F02BD
:10122000AA1A012303FA02F2491106EB8101CDE962
:1012300001121C31009105FB074108EB4101B1F996
:1012400052B0BBF1000FC8BF00284DDDBBEB000161
:1012500048BFA0EB0B018345CCBF5A4602464FF472
:101260004843594391FBF2F101F2FF114A0A03E0AE
:10127000E88600100080FFFF002D14BF5545002CAC
:10128000FE49096814BF91F88C1091F88D1019B9B6
:10129000FA49096891F88C108A4225DD01994FF0CE
:1012A000010CCA6902990A4300990A60E11704EB2C
:1012B000D1614A1106EB820303F1140221F01F01F0
:1012C0005B69611A0CFA01F11943116083B2E2B251
:1012D000E9B20620FDF770FC601CC2B21FFA8BF366
:1012E000E9B20620FDF768FC0399641C58468C425D
:1012F000A1D36D1C4D4585D307B00120BDE8F08F0B
:101300002DE9F04FD2F80080074689B0D8F81000D8
:1013100047F6FF7B20F00F00C8F8100008F15000DE
:1013200004904FF000001061D060906015465FEAB5
:1013300001096FEA0B0A0446506069D0049804FB67
:1013400007F14FF0000C30F91120012113461E4621
:10135000012F1CD904FB071E049830F91E0090428F
:10136000C4BF0246CDE90241B042BCBF0646CDE94A
:101370000041B0EB030E48BFA3EB000E0FFA8EF353
:101380006345C8BF9C460346491CB942E2D3524557
:1013900004DD029808900398924607905E4504DAAF
:1013A000009806900198B3460590901B48BFB01A6C
:1013B00001B2B2480068B0F91C308B4203DBB0F9CF
:1013C0001E00844521DDE01704EBD060411105EBE0
:1013D000810120F01F0001F10C03A4EB000CC9688F
:1013E000012000FA0CF008431860039893B2C2B2CF
:1013F0000298C1B20520FDF7DFFB0198B3B2C2B27B
:101400000098C1B20520FDF7D7FB641C4C4595D36D
:101410000026002F5BD9049801224FF0000C30F910
:101420001610B9F1010F0B461C4618D902FB076EC6
:10143000049830F91E008842C8BF0146A042B8BFD8
:101440000446B0EB030E48BFA3EB000E0FFA8EF379
:101450006345C8BF9C460346521C4A45E6D35145E6
:10146000C8BF8A465C45B8BFA346081B48BF601A80
:1014700002B282480068B0F92030934203DBB0F931
:101480002200844520DDF01706EBD060421105EB09
:10149000820220F01F00131DA6EB000C52680120F1
:1014A00000FA0CF01043186003988BB2C2B2029895
:1014B000C1B20520FDF780FB0198A3B2C2B200982B
:1014C000C1B20520FDF778FB761CBE42A3D3E868C5
:1014D000002804BF2869002805D0D8F8100040F083
:1014E0000800C8F810006868002804BFA868002831
:1014F00005D0D8F8100040F00400C8F81000696862
:10150000E86801FA09F10843C8F82800A9682869C1
:1015100001FA09F10143C8F82C106868B9F1200FED
:1015200039BFC9F12002D040A9F120029040084300
:10153000C8F82C00A8F824B0A8F826A0B5F9D8104F
:10154000BAEB010048BFA1EB0A004C4C2168B1F98D
:10155000181088420EDDD8F810001FFA8AF340F008
:101560000200C8F810000798C2B20898C1B205205E
:10157000FDF722FBB5F9D810B1EB0B0048BFABEB80
:1015800001002168B1F91A1088420EDDD8F8100068
:101590001FFA8BF340F00100C8F810000598C2B2A2
:1015A0000698C1B20520FDF707FB09B00120BDE890
:1015B000F08F2DE9F04F0446314887B00F460068A0
:1015C0004FF0000890F8E40000F00F0500F0C4FAB6
:1015D00001280BD040F20F312846F6F7C3F9012855
:1015E00013D0002000F0B5FA00F092B900210846AF
:1015F000F1F7F7FAEFF7D6FC50B12248D0F84013D4
:1016000041F48031C0F8401302E0012000F0A1FA5B
:101610001D4806781D480578002D18BF002E00F0E3
:1016200075813868002180F8206080F8215080F8AA
:10163000221080F82310F2F7C2F9F1F7E5FB0090D1
:10164000002014F0030F18BF114814F0200F1CBF26
:1016500040F0F00040F00050DFF82080002877D004
:10166000009940F47F00084014F4407F18BF20F434
:101670007F00F1F780FA04200CE00000E8860010FB
:10168000C8860010005000405D8500105E85001087
:1016900007000010F7F75AFD60F30F09824600219A
:1016A0000420F7F74AFD0220F7F750FD60F31F49C9
:1016B00000210220F7F741FD14F4407F17D00020ED
:1016C000F0F719F806900020F0F784F80590002054
:1016D000F0F7BDF804900020F0F70DFA0390002019
:1016E000F0F741FA02900020F0F7D3FD019014F4D6
:1016F000807F4FF0FF3B2CD0D8F80000B0F884106A
:1017000000291CBF0020F0F70AF8D8F8000090F874
:10171000861000291CBF0020F0F7ADF8D8F80000B3
:1017200090F8870010F00F0F05D000F00F00411E59
:101730000020F0F7FAF9D8F8000090F8870010F0D0
:10174000F00F38D00BEB10110020F0F726FA32E042
:101750005DE014F4007F2ED0D8F80000B0F8A0109F
:1017600000291CBF0020EFF7DAFFD8F8000090F83E
:10177000A21000291CBF0020F0F77DF8D8F8000067
:1017800090F8A30010F00F0F05D000F00F00411EDD
:101790000020F0F7CAF9D8F8000090F8A30010F084
:1017A000F00F04D00BEB10110020F0F7F6F9002138
:1017B0000846F0F761FD1F20F6F772FEF1F70EF90B
:1017C00014F4407F17D000200699EFF7A8FF0020FF
:1017D0000599F0F70EF800200499F0F74CF8002076
:1017E0000399F0F7A2F900200299F0F7D6F900204A
:1017F0000199F0F741FD51460420F7F79EFC4FEAAE
:1018000029410220F7F799FC0098F1F7B4F914F098
:101810002C0F04D03A4629463046FEF74BFC14F014
:10182000030F71D000973F68AA46B14607F15005F3
:10183000F1F71AFC8346F1F7D1F8374CA08810F481
:10184000407F03D00020F0F702F801903248406852
:1018500010F4807F05D0D8F8000090F8861059B1B8
:1018600007E010F4007F07D0D8F8000090F8A2102D
:1018700011B10020EFF7FFFF0020F2F74DF800262E
:10188000BAF1000F23D906EB4600002400EB06183E
:1018900016E01BF90400262811D2C107490C00EB01
:1018A000D07001EB8801401001EB800000F1405046
:1018B00000F580300068F2F735F825F8020B641C5B
:1018C0004C4501D2262CE4DB761C5645DBD312486E
:1018D000808810F4407F03D000200199EFF7CBFF00
:1018E0000E4C20781D280AD107F15000FBF7EDFBC4
:1018F00020781D2804BF07F15000FBF7E6FB514696
:101900004846009AFDF77BFC4FF00108F1F73FFADB
:1019100007B04046BDE8F08FCC860010E58500108A
:1019200070474FF0FF3070477848406870477749FC
:101930004860704710B582B007280BD14FEA111CE0
:10194000012404FA0CFC714C64681CEA040F04BF07
:1019500002B010BD9B0100F00F0043EA800040F090
:1019600001008DF800008DF801108DF80220100A9A
:101970008DF80300100C8DF80400100E8DF8050092
:1019800000208DF806008DF8070068460EF0FBFA7F
:1019900002B010BD2DE9F04F0E464FF0000183B0AC
:1019A0005FEA020800914FF001024FF002070D4676
:1019B0000C46019104BF03B0BDE8F08FEB467B01FC
:1019C00000F0070943EA890040F0030A16F8140002
:1019D0000BF80200501C36F81420C0B2120A0BF8A3
:1019E0000020401CC2B2481CC1B2B9420ED1681CD2
:1019F00085B28DF800A0FF2D94BF2846FF208DF8FA
:101A0000050068460EF0BFFA00210122601C84B276
:101A10004445DBD3002904BF03B0BDE8F08F480183
:101A200040EA890040F003008DF80000681C80B295
:101A3000FF2888BFFF208DF8050068460EF0A3FA46
:101A400003B0BDE8F08F10B582B007280DD191F832
:101A500000C001244FEA1C1C04FA0CFC2B4C6468E7
:101A60001CEA040F04BF02B010BD9B0100F00F0080
:101A700043EA800040F001008DF80000072A88BF8B
:101A8000072200206B46002A09D911F800C01C1853
:101A9000401C84F801C09042F7D3072805D20021EA
:101AA0001A18401C51700728FAD318460EF06BFA2A
:101AB00002B010BD70B5154E40EA012502283488E9
:101AC000224618BF052803D1002918BF022900D1DA
:101AD0002C46A24209D051B17088002344EA00424A
:101AE00090210720FFF726FF3480758070BDF2F744
:101AF00014FF4FF47A71B0FBF1F044EA0042002386
:101B000090210720FFF716FFEEE70000DC860010AB
:101B1000FE4908707047FD480078704710B50446CC
:101B2000FCF7A9FE0146D42220460EF031FAF74810
:101B3000446010BD58B1F64A0168914207D140682F
:101B400020F00F00B0F5807F04BF01207047002017
:101B50007047EE4948707047EC484078704710B5C0
:101B6000EC48EA4C86B000686178808F0429C0F3A5
:101B7000032008D00421F5F7F5FE01281CBF002042
:101B800060700FD043E000210846F1F72AF8EFF724
:101B900009FA88B1E048D0F8401341F48031C0F828
:101BA000401309E00420607005210020EFF7B7FD25
:101BB00000210846F0F785F81F20F6F771FC0EF0BB
:101BC00069FA0EF06CFA0020F4F72FF8EFF7EAF953
:101BD00010F0010F04BF0120EFF79AFCF1F742F972
:101BE000FAF744FE01280CD06846F1F73EFC28B114
:101BF0006846FBF746FDF1F780FCF1E7F5F78CFD51
:101C0000EEE7F0F7EBFE0EF04AFA0EF04DFAF1F7C0
